:100000000C9419090C9468090C9468090C946809FB
:100010000C9468090C9468090C9468090C9468099C
:100020000C9468090C94A81C0C9468090C94680939
:100030000C9449380C9468090C9468090C9468096C
:100040000C9468090C9468090C94DC180C946809E9
:100050000C943A0F0C9468090C94040F0C946809E2
:100060000C94981F0C9468090C94BF330C94680985
:100070000C94AB970C9468090C94A28D0C946809AD
:100080000C9468090C9468090C946809BF1FC41F7C
:10009000C91FD21FE91F0020102020205B20EA2268
:1000A000002077218821B721D521F2214C22A722D7
:1000B00079253C26E226592791273428432AA42A69
:1000C0001E2B4F2BA72BD52B022C652CAF2CF92CDC
:1000D000F22DDE3312345534C534DD341E35D535BA
:1000E0009C369C369C369C369C369C369C369C3680
:1000F0009C369C369C36513653365836703672369E
:10010000CE70BF7144726F719672C3720B719E7123
:10011000C07E647FE97F4B809F80088159888981F8
:10012000BB81BB81BB81BB81BB81BB81BB81BB81EF
:10013000BB81E9816482F5821A835D83B583408443
:10014000298590859085908590859085908590856E
:1001500090859085C885E6850B866786A386078788
:100160003487D487598834883488348834883488EC
:10017000348834883488E995EC95EC95EC95F595C0
:10018000F895FB950D960A960A0D3D3D3D3D3D3D8A
:100190003D3D3D3D3D3D3D3D3D3D3D3D3D3D3D3D8F
:1001A0003D3D3D3D3D3D3D3D3D3D3D3D3D000A0D1F
:1001B000426174743A002025642043656C6C73209E
:1001C00000204C6F77207761726E696E673A202548
:1001D000642E2564000A0D466F756E6420424C2D16
:1001E0004374726C3A20002564000A0D0A0D212127
:1001F000204D495353494E4720424C2D4354524CB5
:100200003A202564202121000A0D43616C69627245
:100210006174696E6720707265737375726520739F
:10022000656E736F722E2E004F4B0A0D000A0D463D
:100230006C696768742D74696D65202575206D691A
:100240006E20546F74616C3A2575206D696E0041A3
:100250006E676C654E69636B202020202020204152
:100260006E676C65526F6C6C20202020202020412E
:1002700063634E69636B20202020202020202041D2
:100280006363526F6C6C2020202020202020205996
:1002900061774779726F2020202020202020204184
:1002A0006C746974756465205B302E316D5D20411E
:1002B00063635A2020202020202020202020204757
:1002C0006173202020202020202020202020204377
:1002D0006F6D706173732056616C756520202056B8
:1002E0006F6C74616765205B302E31565D20205243
:1002F00065636569766572204C6576656C2020477C
:1003000079726F20436F6D70617373202020204DD0
:100310006F746F7220312020202020202020204D5B
:100320006F746F7220322020202020202020204D4A
:100330006F746F7220332020202020202020204D39
:100340006F746F7220342020202020202020203144
:100350003620202020202020202020202020203176
:100360003720202020202020202020202020203165
:100370003820202020202020202020202020203154
:100380003920202020202020202020202020205321
:100390006572766F202020202020202020202048F9
:1003A0006F76657267617320202020202020204313
:1003B000757272656E74205B302E31415D20204372
:1003C00061706163697479205B6D41685D202048CC
:1003D000656967687420536574706F696E74203244
:1003E00035202020202020202020202020202032E6
:1003F00036202020202020202020202020202043C4
:100400006F6D7061737320536574706F696E74499A
:1004100032432D4572726F7220202020202020420E
:100420004C204C696D69742020202020202020471A
:1004300050535F4E69636B202020202020202047EE
:1004400050535F526F6C6C202020202020202021F0
:10045000212120494E434F4D50415449424C4520A3
:10046000212121002A002E000A0D20444143206F43
:100470007220493243204552524F52212043686531
:10048000636B204932432C2033567265662C20441E
:10049000414320616E6420424C2D4374726C005BBA
:1004A00025695D005B25695D002B204D696B726FCE
:1004B0004B6F70746572202B0048573A5625642E96
:1004C00025642053573A25642E256425632056342D
:1004D0000053657474696E673A2564202573004D76
:1004E00069786572204572726F72210045525225FB
:1004F00032643A00486172647761726520457272B5
:100500006F7220313A2564202121004D697373698F
:100510006E6720424C2D4374726C3A256421210091
:10052000493243204552524F5221212100486569EA
:100530006768743A202025356900536574706F69C7
:100540006E743A2535690050726573737572653A39
:10055000253569004F66667365743A202025356934
:10056000002841290048656967687420636F6E74CC
:10057000726F6C0044495341424C454400616374BE
:100580002E2062656172696E67004E69636B3A2066
:10059000202020202025356900526F6C6C3A2020E5
:1005A0002020202025356900436F6D706173733AF8
:1005B000202020253569004B25693A253469202003
:1005C0004B25693A25346920004E693A2534692063
:1005D00020526F3A253469200047733A2534692048
:1005E0002047693A253469200050313A2534692082
:1005F0002050323A253469200050333A253469209E
:100600002050343A25346920004779726F202D201C
:1006100053656E736F72004E69636B2534692028D1
:100620002533692E25692900526F6C6C25346920A9
:10063000282533692E2569290047696572253469A3
:10064000202825336929004E69636B2025346920F1
:10065000282533692E25782900526F6C6C202534AB
:100660006920282533692E257829005961772020B3
:10067000253469202825336929004E69636B2025BC
:100680003469202825336929282533692900526FC8
:100690006C6C202534692028253369292825336985
:1006A00029005961772020253469202825336929BC
:1006B000282533692900414343202D2053656E735B
:1006C0006F72004E69636B202534692028253369D9
:1006D0002900526F6C6C2025346920282533692944
:1006E000005A20202020253469202825336929003C
:1006F000566F6C746167653A2020202533692E257A
:100700003169560043757272656E743A2020202557
:1007100033692E2531694100506F7765723A202088
:10072000202020253469570044697363686172672B
:10073000653A202535696D416800526563656976C3
:1007400065720052432D5175616C6974793A2025A8
:1007500034690052432D4368616E6E656C733A25AF
:10076000346900436F6D70617373004D61676E652E
:10077000743A202020253569004779726F3A20208D
:1007800020202025356900536574706F696E743AB6
:100790002025356900506F746925693A202025337A
:1007A0006900506F746925693A2020253369005328
:1007B0006572766F202000536574706F696E7420C7
:1007C0002025336900506F736974696F6E3A202574
:1007D00033690052616E67653A2533692D253369A7
:1007E00000424C2D4374726C204572726F727320FC
:1007F00000253364202533642025336420253364A9
:100800002000424C2054656D70657261747572658C
:100810000025336420253364202533642025336488
:100820002000424C2D4374726C20666F756E6420FC
:100830000020256320202025632020202563202000
:1008400020256320002025632020202563202020F0
:100850002563202020256320002025632020202DD3
:100860002020202D2020202D20003130003131008B
:10087000313200466C696768742D54696D652020BB
:1008800000546F74616C3A2535756D696E00416373
:10089000743A20202535756D696E00287265736580
:1008A0007429000A0D2D2D3E204861726477617213
:1008B000652056657273696F6E20427974652043B6
:1008C00068616E676564203C2D2D000A0D47656EDA
:1008D00065726174696E672064656661756C742009
:1008E000506172616D657465722053657420256472
:1008F000000A0D5573696E6720506172616D6574F1
:10090000657220536574202564000A0D47656E6585
:10091000726174696E672064656661756C74204DE0
:1009200069786572205461626C65000A0D4D6978C2
:1009300065722D436F6E6669673A202725732720FD
:10094000282575204D6F746F727329000A0D41437D
:1009500043206E6F742063616C69627261746564B8
:10096000210D0A0000008F001E01AD013B02CA02EA
:100970005803E603740402058F051B06A706330718
:10098000BE074808D2085B09E3096B0AF20A780B34
:10099000FD0B810C040D860D070E870E060F840FCC
:1009A00000107B10F5106E11E5115B12CF1242138F
:1009B000B31323149214FE146A15D3153B16A11613
:1009C00005176717C81727188318DE1837198E19E7
:1009D000E319361A871AD61A231B6E1BB61BFD1B8A
:1009E000411C831CC31C001D3C1D751DAB1DE01D5F
:1009F000121E421E6F1E9A1EC31EE91E0D1F2E1FC1
:100A00004D1F691F841F9B1FB01FC31FD31FE11FF2
:100A1000EC1FF51FFB1FFF1F002000000500050055
:100A2000040106010800060102000400040007009A
:100A30000700070007000700070007000301030184
:100A4000050017010F01060009010A01190105013E
:100A5000050119011A010F0100004E6F2045727245
:100A60006F722020202020202020004E6F742063F1
:100A70006F6D70617469626C652020004D4B334D61
:100A80006167206E6F7420636F6D7061004E6F2020
:100A9000464320636F6D6D756E6963617400436FCB
:100AA0006D7061737320636F6D6D756E6963004760
:100AB000505320636F6D6D756E69636174696F006B
:100AC000636F6D706173732076616C756520202093
:100AD000005243205369676E616C206C6F73742001
:100AE0002000464320737069207278206572726F0F
:100AF0007220004E6F204E4320636F6D6D756E69DE
:100B0000636174004643204E69636B204779726FBE
:100B10002020202000464320526F6C6C20477972C1
:100B20006F202020200046432059617720477972AA
:100B30006F2020202020004643204E69636B204117
:100B40004343202020202000464320526F6C6C201D
:100B50004143432020202020004643205A2D41437A
:100B600043202020202020202000507265737375C0
:100B700072652073656E736F7220004932432046A0
:100B8000432D3E424C2D4374726C2000426C204D2C
:100B9000697373696E67202020202020004D6978DA
:100BA0006572204572726F72202020202000436100
:100BB000726566726565204572726F72202000470B
:100BC000505320466978206C6F73742020202000D9
:100BD0004D61676E6574204572726F72202020200F
:100BE000004D6F746F72207265737461727420208F
:100BF0002000424C204C696D69746174696F6E20ED
:100C00002020004750532052616E6765202020202D
:100C1000202020004E6F2053442D43617264202019
:100C2000202020200053442D4C6F6767696E672099
:100C30006572726F7200466C79696E672072616EC0
:100C4000676521202020004D617820416C74697413
:100C500075646521202020004E6F20475053206688
:100C6000697820202020202000636F6D70617373ED
:100C7000206E6F742063616C2E0053657420203ADF
:100C800000202121204C69506F20766F6C746167C1
:100C90006520212120200020202020204D696B721A
:100CA0006F4B6F7074657220202020200020202060
:100CB0002020202020202020202020202020202034
:100CC00020200020202532692E2531695620200061
:100CD00020202532692E25316956202000414C54B0
:100CE0003A2534696D20256300414C543A25346916
:100CF0006D202000414C543A2D2D2D2D2000202018
:100D00002532693A253032692020002020253269B9
:100D10003A253032692020004449523A2025336474
:100D20002563004300200020202535692020002075
:100D300020253569202000493A2532692E25316960
:100D40004120003A003A003A002D2D2D2D2D2D2D59
:100D50002D2D2B2D2D2D2D2D2D2D2D2D2D2D002DF2
:100D60002D2D2D2D2D2D2D2D2D2D2D2D2D2D2D2DB3
:100D70002D2D2D2D003A005341543A253264200088
:100D8000444953543A2533646D00442000334400F1
:100D90002121004D41473A25337525252000484D36
:100DA0003A253364256320256300696E636C3A2518
:100DB000326425632825326929002020202025322D
:100DC000756D2F733A2020484D3A253364256320F2
:100DD0002563004552523A202532642021004552B5
:100DE000523A20002121204C69506F20766F6C749C
:100DF00061676520212100207777772E4D696B721E
:100E00006F4B6F707465722E646520200020253250
:100E1000693A2530326920202532692E25316956FC
:100E2000202534696D416800202532693A25303229
:100E30006920202532692E25316956202534696DB7
:100E40004168004449523A253364256300414C54BB
:100E50003A2534696D00414C543A2534696D00419E
:100E60004C543A2D2D2D2D2000256300484D3A2558
:100E7000336425632020444953543A2533646D205C
:100E80002563005057523A2532692E253169412099
:100E90002825695729200043460020200047505349
:100EA0003A2532756D2F73205341543A2564200042
:100EB0002020334420004E4F4649580044475053A9
:100EC00020002020204E6F204E6176694374726CA2
:100ED00020202020202020002532692E2569202571
:100EE00032692E2569202532692E2569202532692F
:100EF0002E25694100253369202533692025336972
:100F000020253369256343002532692E2569202574
:100F100032692E256941002532692E256920253246
:100F2000692E2569202532692E2569202532692EF2
:100F30002569410025336920253369256343202035
:100F400020202020202000253369202533692025FA
:100F5000336920253369256343004552523A2025E1
:100F600032642021004552523A20002121204C6950
:100F7000506F20766F6C74616765202121002077A7
:100F800077772E4D696B726F4B6F707465722E643C
:100F90006520200053657474696E673A25752025B5
:100FA0007320004D696E3A2532692E25316956202D
:100FB00025732000414C543A00504F54493A253390
:100FC000752000284F4E29202000284F4646292012
:100FD000004C494D495400564152494F0044495331
:100FE00041424C45440043463A0044495341424C37
:100FF00045440020284F4E29200020284F464629EE
:1010000000205445414348004750533A0044495357
:1010100041424C4544002846524545290028484F46
:101020004D4529002841494429200028484F4C4477
:1010300029002046533A257573656B2000484F4DB3
:101040004520414C543A0025756D00484F4C4420D2
:10105000004E693A25346920526F3A25346920439D
:101060003A2533690047733A2534692059613A2596
:101070003469200050313A2534692050323A253401
:101080006920333A2533690050343A2534692050B9
:10109000353A25346920363A25336900434F555097
:1010A0004C494E47204F46462120004C4F4F504957
:1010B0004E472120004848212000434F4D504153C6
:1010C00053204F4646212000004F50515253545355
:1010D000565748005859005A554546474841004917
:1010E000424A4A0000000000000000000000444C9A
:1010F0004D00000000004E0000004B00430A0D7739
:1011000077772E4D696B726F4B6F707465722E64BA
:10111000652028632920486953797374656D7320AD
:10112000476D6248000A0D74686520757365206F0D
:1011300066207468697320736F66747761726520C6
:101140006973206F6E6C79207065726D6974746557
:1011500064200A0D6F6E206F726967696E616C2082
:101160004D696B726F4B6F707465722D486172645C
:1011700077617265005573657200486F545420564C
:1011800034004143542044534C004A657469005371
:1011900070656B7472756D0050504D000A0D52658C
:1011A0006365697665723A2000532E427573007547
:1011B0006E6B6E6F776E2E205573696E6720505080
:1011C0004D2E2E2E006E6F7420737570706F7274BA
:1011D00065642062792068617264776172652100BC
:1011E0000A0D466C69676874436F6E74726F6C0A9F
:1011F0000D48617264776172653A25642E25640A30
:101200000D536F6674776172653A5625642E2564B6
:10121000256320000A0D202D204C4942204E4F54BA
:1012200020434F4D50415449424C4520212121211A
:10123000000011241FBECFEFD0E4DEBFCDBF12E00F
:10124000A0E0B1E0E6E2F5E301E00BBF02C00790E9
:101250000D92AC3DB107D9F71CE0ACEDB2E001C096
:101260001D92A83AB107E1F77AEAE2E0F0E081E204
:1012700080935700D4907E010894E11CF11C20EF6C
:1012800037EF41E050E087016FE0DA01C9012F5FDD
:101290003F4F4F4F5F4FABBFFC018791F8018193E8
:1012A0008F01615067FFF1CFF7016EE081917827E0
:1012B0007095615067FFFACF8889781729F0F7E9B0
:1012C000DF1611F40000FECF0E94340A0C94929AAB
:1012D0000C94000088E891E09F938F9383EB95E155
:1012E0009F938F93E0918405F091850509950F9068
:1012F0000F900F900F90089580912908E82FFF27F5
:10130000EE0FFF1FE25AF64F808191818D5E9F4F55
:1013100014F010920301808191818A5B9F4FCCF47D
:10132000809103018823A9F481E0809303018091D7
:10133000B8058F5F8093B805853038F088EE93E06C
:101340009093120380931103089566E970E00E9460
:10135000B73B08951F93CF93DF93182F882389F00D
:101360008EEA91E09F938F9383EB95E19F938F9308
:10137000E0918405F091850509950F900F900F90ED
:101380000F9080914C08823308F044C084EF91E0C4
:101390000E94BE19EC01112329F0CE010E94C71949
:1013A0008823D9F3C2E0D0E026E530E08091200127
:1013B000909121018217930730F02196255D3F4FD0
:1013C000C730D10598F380914C089927C89F9001A8
:1013D000C99F300DD89F300D112420930101112396
:1013E000D9F068EC70E08C2F0E94B73BDF93CF936D
:1013F00086EB91E09F938F9383EB95E19F938F937F
:10140000E0918405F091850509958DB79EB7069604
:101410008DBF02C080930101112311F18091010160
:101420006AE00E94E599892F99279F938F93809175
:1014300001010E94E59999279F938F9381EC91E098
:101440009F938F9383EB95E19F938F93E091840516
:10145000F091850509952DB73EB7285F3F4F2DBF09
:10146000DF91CF911F910895CFEFD0E4DEBFCDBFC4
:1014700088249924C1E07C2E14B815B88AE08AB972
:101480008FE58BB9B7EEEB2EB3E0FB2E2EEC3FEFE2
:10149000E20EF31EF7FEFACF6624199B08C04C9BA0
:1014A00004C085E18093020108C086E101C087E1A4
:1014B0008093020181E08093F70381E887B93E9A27
:1014C0008FEF88B98BE184B981E085B9469A84B7FA
:1014D000877F84BF80916000886180936000109254
:1014E000600084EC99E090931203809311031092B2
:1014F00045041092440410926309109262091092FC
:101500004704109246041092490410924804209116
:101510000201243128F084EC94E0A0E0B0E004C0A3
:101520008BE095E0A0E0B0E080933C0190933D011A
:10153000A0933E01B0933F012A3011F0243110F006
:10154000289801C0289A2C3010F0273111F4299ADC
:1015500001C029980E94271A0E94F8190E94BB1501
:101560000E9410380E94291E81E00E9473330E945D
:10157000746F0E94047983E00E9461968091020159
:101580008C3010F0873111F4299A01C02998789491
:101590000E945A3280915A03826080935A031092BB
:1015A0005D030E94844784EF91E00E94BE197C0194
:1015B00080915A0380FD05C0C7010E94C719882386
:1015C000B9F385ED91E09F938F93A3EBAA2EA5E14C
:1015D000BA2EBF92AF92E0918405F09185050995EE
:1015E00080EA9FE00E94BE197C01C0E0D0E00F902D
:1015F0000F900F900F9000E019E0F4EBCF2EF8E081
:10160000DF2E0E94844780915A0380FD05C0C701E8
:101610000E94C7198823B9F3F60180811816ACF42B
:101620000BC00E94844780915A0380FD05C0C7010A
:101630000E94C7198823B9F3C7010E94C7198823DC
:1016400021F4F8018081882364F7F801808187FF05
:1016500019C02196DF93CF93219787EE91E09F9356
:101660008F93BF92AF92E0918405F0918505099523
:101670008091DD028F5F8093DD022DB73EB72A5F38
:101680003F4F2DBF219684E090E0C80ED91E085F21
:101690001F4FCC30D10508F4B4CFC0E0D0E00DEF3F
:1016A00018E0E4EBEE2EE8E0FE2EF801838187FDE2
:1016B0001DC0F70180811816CCF42196DF93CF93DB
:1016C00021978AEE91E09F938F9383EB95E19F930F
:1016D0008F93E0918405F0918505099582E08093D0
:1016E0000F032DB73EB72A5F3F4F2DBFF80183810F
:1016F00080788383219624E030E0E20EF31E085FB9
:101700001F4FCC30D10588F20E946A0990912708BA
:101710008091DD02981728F480919E058061809366
:101720009E0588E092E09F938F93C3EBD5E1DF9312
:10173000CF93E0918405F0918505099588EE93E0BB
:101740000E94BE197C010E942F1E0F900F900F90D7
:101750000F90C7010E94C7198823D9F388E292E04D
:101760009F938F93DF93CF93E0918405F09185054C
:10177000099580E00E949B3C809102010F900F90A0
:101780000F900F908A3011F0843110F0289801C02A
:10179000289A80ED97E0909312038093110385E5DA
:1017A0008093BA058EE090E00E947A309927182F36
:1017B00000278FE090E00E947A30080F111D1093EF
:1017C000E3020093E2028AE090E00E947A309927D7
:1017D000182F00278BE090E00E947A30080F111D2F
:1017E0001093E1020093E0020F5F1F4F39F08091E8
:1017F000E2029091E3028F5F9F4F41F41092E30267
:101800001092E2021092E1021092E0028091E00256
:101810009091E1029F938F938091E2029091E30275
:101820009F938F938DE292E09F938F93DF93CF935B
:10183000E0918405F091850509950E94EB2488E8E4
:1018400093E19093370180933601C1E0C093B905CD
:101850008C2F0E94AA0980914F080E94AD950E948A
:101860006A0980ED97E00E94BE197C018AEF90E042
:101870000E94BE1983E0809381071092DC02809160
:1018800098082DB73EB7285F3F4F2DBF84FF02C099
:10189000C093E40212BC11BC8091E602882311F0CF
:1018A0004798FECF80911503882309F49EC280914A
:1018B0001201882309F499C2109215038091B8058A
:1018C000882319F00E947C0902C00E940B4B0E94E1
:1018D0008447209102012A3011F0243110F0289819
:1018E00001C0289A80913804882331F0809138040F
:1018F0008150809338040EC080916F008062809385
:101900006F0010925F0910925E0980919E058860B9
:1019100080939E05809136019091370101979093B5
:101920003701809336018091360190913701892BE0
:1019300021F080915B038823C9F180913601909159
:101940003701892BD9F40E949D3385E090E0909374
:101950003701809336018091BB079091BC070196B7
:101960009093BC078093BB0780919E058160809314
:101970009E058091820782608093820780910A0190
:1019800090910B018F5F9F4FC1F4809137048823A2
:10199000A1F088EA91E6909312038093110380E806
:1019A00090E090930B0180930A0107C02A3011F058
:1019B000243110F0289801C0289A0E942E97809117
:1019C0001503882309F00FC280915105882319F06F
:1019D0000E94D98808C280911001882311F00E94CA
:1019E000801A0E9404160E948A11C7010E94C7191A
:1019F000882309F4F4C184E190E0E80EF91E0E9406
:101A00003E1A80914F08863019F40E94847E04C0EB
:101A1000843011F40E94A9898091F703882331F161
:101A20008091C8079091C9078C52914074F08091C1
:101A300091079091920780509240C4F48091C8071A
:101A40009091C907835593408CF0639432E3361527
:101A500070F480913704882331F080919D05806275
:101A600080939D0504C08093230401C06624809167
:101A70005B03882349F080919E05826080939E05D8
:101A80008091820782600FC08091110390911203B0
:101A9000892B59F48091360190913701079728F0EE
:101AA000809182078D7F809382078091E402882352
:101AB00061F080913804873940F01092E40288E8A0
:101AC00093E1909312038093110380910501882381
:101AD00021F08150809305012EC08093C40510929F
:101AE0000B0410920A041092090410920804109238
:101AF000070410920604809138048823E1F4809151
:101B00000A0190910B018F5F9F4FA9F42091E4028D
:101B1000223089F088E99AE39093120380931103AD
:101B200080E09CE090930B0180930A01222319F03E
:101B300082E08093E40280919E01893C70F08150A4
:101B400080939E0180919E058B7F80939E0580915E
:101B5000A10581608093A10551C08091640A88230A
:101B6000F9F080919E05846080939E0589E08093C2
:101B7000160580910A0190910B018F5F9F4F81F4B0
:101B800080913704882361F088E99AE390931203E7
:101B90008093110380E098EA90930B0180930A01EF
:101BA000109208051092070510920605109205057F
:101BB000109204051092570A8FEF8093CC0A10926E
:101BC000960A1092950A1092980A1092970A8FEF2F
:101BD0009FEF9093940A8093930A10922704109297
:101BE00028041092290410922A0410922B04809148
:101BF000A1058E7F8093A10510929E018091010125
:101C0000282F33278091200190912101821793077B
:101C1000CCF48091FF0380628093FF0380910A01DE
:101C200090910B018F5F9F4FC1F480E797E19093F4
:101C300012038093110380E093E090930B01809353
:101C40000A010BC08091110390911203892B29F492
:101C50008091FF038F7D8093FF0383E080931003C7
:101C600012BC11BC8091E5028F5F8093E502813345
:101C700009F06CC01092E50280913E05882319F0AE
:101C8000815080933E058091FF0381FF0AC08091BF
:101C9000DE029091DF0201969093DF028093DE02D4
:101CA00004C05AEA852E55E0952E8091000490914B
:101CB00001048050944008F049C02091CA07309137
:101CC000CB074091CC075091CD078091180190919E
:101CD0001901A0911A01B0911B01281739074A0771
:101CE0005B0764F48091CA079091CB07A091CC0761
:101CF000B091CD070596A11DB11D20C02091CA0746
:101D00003091CB074091CC075091CD0780911801BD
:101D100090911901A0911A01B0911B0182179307AC
:101D2000A407B5079CF48091CA079091CB07A091B6
:101D3000CC07B091CD070597A109B1098093CA07D7
:101D40009093CB07A093CC07B093CD070894811C48
:101D5000911C82E788168BE0980609F040C0882421
:101D600099242091E2023091E3022F5F3F4F30939C
:101D7000E3022093E2028091E0029091E102019659
:101D80009093E1028093E002832F9927682F8EE0E1
:101D900090E00E9482308091E2029091E302907084
:101DA000682F8FE090E00E9482308091E002909155
:101DB000E102892F9927682F8AE090E00E94823003
:101DC0008091E0029091E1029070682F8BE090E0AA
:101DD0000E94823084E190E00E94BE197C010E9442
:101DE000B9740E941B7971107A94772029F40E94AB
:101DF00082748CE0782E50CD80911003882309F0F6
:101E00004BCD0E94956F48CD1F920F920FB60F9247
:101E100011248F939F93EF93FF9380910701882361
:101E2000E1F48091000390910103019690930103E6
:101E300080930003FC01EB55F94FE081ED3019F080
:101E40008C3D910539F4109201031092000381E05A
:101E500080930701E093C60004C010920103109222
:101E60000003FF91EF919F918F910F900FBE0F9004
:101E70001F9018951F920F920FB60F9211242F9357
:101E80003F934F935F936F937F938F939F93AF9302
:101E9000BF93CF93EF93FF9390E08091E602813060
:101EA00029F48091C6008093CE00CCC08091E602D8
:101EB000823029F48091C6008093C705C3C0809109
:101EC000C6008093F802509106035C3D10F0909399
:101ED00007038091F8028D3009F065C080910703F7
:101EE000823009F060C090930703852F99278953AA
:101EF0009A4FFC01329740812091020330910303F5
:101F0000241B3109DC0111978C91281B3109C9016F
:101F10009F70909303038093020346E09695879504
:101F20004A95E1F7982F935C909304032F733070D8
:101F3000235C209305038081981729F48C9128173E
:101F400011F491E006C090E08091F5028F5F8093DC
:101F5000F502C091F702CC2309F074C0992309F46B
:101F600071C081E08093F702580F5093F4025150F2
:101F7000E52FFF27E953FA4F8DE080838091C90553
:101F8000823509F05FC00E94EB2488E190E02CE0EC
:101F90000FB6F894A895809360000FBE2093600060
:101FA000C0930F034FC020910703822F99278130E0
:101FB0009105F9F0823091051CF4892B21F040C085
:101FC000029711F13DC08091F802833239F480917B
:101FD000F702882319F481E0809307038091F802C7
:101FE0008093C70581E0809306038091F8029927CA
:101FF00022C02F5F20930703E52FFF27E953FA4FF5
:102000008091F802808309C0E52FFF27E953FA4F3A
:102010008091F80280835C3D20F45F5F509306035B
:1020200002C0109207032091F80280910203909160
:102030000303820F911D909303038093020302C058
:1020400010920703FF91EF91CF91BF91AF919F91B4
:102050008F917F916F915F914F913F912F910F9051
:102060000FBE0F901F901895AC01A0E0B0E09D014D
:10207000A817B90748F4E5EAF6E08191280F311D69
:102080001196A417B507C8F33F70FD01EB55F94F42
:10209000C90156E0969587955A95E1F7835C808350
:1020A0001196FD01EB55F94F2F733070822F835C31
:1020B0008083AA55B94F8DE08C93109207018091CF
:1020C000A5068093C6000895A0E0B0E0EAE6F0E13E
:1020D0000C945E9A2C859D850E85BB2483E28093AB
:1020E000A5069F599093A6062093A70633E0E32EFA
:1020F000F12C002309F49EC0CF84D888BE016D5E08
:102100007F4FA989BA890150109709F493C010979D
:10211000B9F0F601EB0DF11DB3949081119791F494
:10212000002349F1FB016E5F7F4FDB01C080D1804E
:102130006E5F7F4F0D90BC91A02DBB24015002C05B
:1021400090E019C01097B9F0F601EB0DF11DB394B2
:102150004081119791F4002341F1FB016E5F7F4FA5
:10216000DB01C080D1806E5F7F4F0D90BC91A02DB0
:10217000BB24015002C040E018C01097B1F0F60136
:10218000EB0DF11DB3941081119781F4002371F0D0
:10219000FB013296DB01CD90DC90BF016E5F7F4F7B
:1021A000A081B181BB24015001C010E0F701EB55C3
:1021B000F94F892F86958695835C80830894E11C6E
:1021C000F11CF701EB55F94F892F99278370907017
:1021D00024E0880F991F2A95E1F755279A0194E08A
:1021E000369527959A95E1F7822B835C8083089436
:1021F000E11CF11CF701EB55F94F4F705070440F83
:10220000551F440F551F812F992726E096958795D6
:102210002A95E1F7842B835C80830894E11CF11CF0
:10222000F701EB55F94F1F73135C10830894E11C01
:10223000F11C6ACFC7010E943410E9E00C947A9A2D
:10224000A3E07A2F4091F4024650442309F458C089
:10225000E72FFF27E953FA4F80818D537F5FE72FE8
:10226000FF27E953FA4F20812D537F5FE72FFF2788
:10227000E953FA4F30813D537F5FE72FFF27E95342
:10228000FA4F60816D537F5F9927880F991F880FE0
:10229000991F522F52955F70582B822F99278F705C
:1022A0009070F4E0880F991FFA95E1F7232F269597
:1022B0002695282B832F992783709070E6E0880F4E
:1022C000991FEA95E1F7682B41504F3FC9F0EA2F7B
:1022D000FF27E953FA4F5083AF5F41504F3F81F0E2
:1022E000EA2FFF27E953FA4F2083AF5F41504F3F5A
:1022F00039F0EA2FFF27E953FA4F6083AF5FA5CF8C
:102300008AEC95E09093F3028093F202A350A0939D
:10231000F1020895A2E0B0E0E0E9F1E10C94649AE2
:102320008091F702882309F41AC40E942011809139
:10233000C805823609F0E6C28091C9059927803721
:10234000910509F4ABC081379105C4F48A36910533
:1023500009F443C28B36910544F48B34910571F135
:102360008636910509F470C1CDC28D36910509F408
:1023700069C08E36910509F44DC0C4C284379105F9
:1023800041F1853791054CF48137910509F48DC0F1
:102390008337910509F4E0C0B5C28737910509F488
:1023A000DEC1883791052CF48537910509F49AC16F
:1023B000A9C28937910509F47FC1A4C2E091F20254
:1023C000F091F3028081918190938B0180938A0137
:1023D00099C28091F402A091F202B091F30285318A
:1023E00040F080E1E2EAF5E00D9001928A95E1F794
:1023F0000DC08D919D910D90BC91A02D8093A20553
:102400009093A305A093A405B093A50580EF8093B6
:10241000EF0247C0809107018823E1F38DE490E04B
:102420009F938F9387EA98E09F938F9381E08F9398
:102430008F938EE48F930E9464108DB79EB707969A
:102440008DBF60C2A091F202B091F3021C911130D5
:1024500081F48DE4E7EAF8E00D9001928A95E1F7C6
:102460000E949531198380919E058F7E80939E05F1
:1024700001C01982809107018823E1F381E090E097
:102480009F938F93CE0101969F938F9381E08F93BB
:102490008F938DE48F930E94641009C181E0809333
:1024A000FA028FEF809305012DC2809137048823B3
:1024B00009F028C2E091F202F091F302E0818E2F40
:1024C0008A508A3058F48983882311F481E003C04C
:1024D000863010F085E0898361E00EC08E2F845134
:1024E0008A3070F48983882311F481E003C0863038
:1024F00010F085E0898360E089810E94173212C064
:10250000E983EF3F19F40E94F83189838981882398
:1025100011F481E003C0863010F085E08983898161
:102520000E949830809107018823E1F38EE790E0C4
:102530009F938F9388E298E09F938F9381E090E040
:102540009F938F93CE0101969F938F9382E08F93F9
:1025500081E08F9381E539C12091F2023091F3023D
:10256000D9018C918150853008F045C0F9018181F5
:102570008F3509F040C0809137048823E1F52F5F43
:102580003F4F8EE7E8E2F8E0D9010D9001928A957D
:10259000E1F7F90182910E9405318091690899273C
:1025A000AA27BB27BC01CD0124EC39E040E050E074
:1025B0000E94C699DC01CB01809382019093830134
:1025C000A0938401B093850180916A089927AA2776
:1025D000BB27BC01CD010E94C699DC01CB018093D1
:1025E0007E0190937F01A0938001B09381010E94AE
:1025F000F831898301C01982809107018823E1F3B2
:1026000081E090E09F938F93CE0101969F938F93EB
:1026100081E08F938F9383E58F930E9464108DB731
:102620009EB707968DBF80913704882329F46EE604
:1026300070E089810E94B73B80E00E94AA098091E6
:102640004F080E94AD955EC180913704882309F040
:1026500059C1E091F202F091F302E0818E2F815096
:10266000853018F48E2F0E9498300E94F8318983AB
:10267000809107018823E1F381E090E09F938F939D
:10268000CE0101969F938F9381E08F938F9386E481
:102690008F930E9464106EE670E089810E94B73BC0
:1026A00080E00E94AA0980914F080E94AD95ADB7C5
:1026B000BEB71796ADBF26C119822981A091F2023B
:1026C000B091F302EEE5F9E08D91992787FD9095A1
:1026D00093A382A3822F8F5F8983282F32968C3019
:1026E00098F310C1E091F202F091F30280810E9410
:1026F00069378A83882319F481E0898301C01982AC
:10270000809107018823E1F388E090E09F938F9305
:1027100085EF98E09F938F9321E030E03F932F93D4
:102720008091F2029091F3029F938F933F932F93A6
:10273000CE0102969F938F933F932F93CE01820FEA
:10274000931F9F938F9384E08F9381E08F9385E510
:102750008F930E946410EDB7FEB773963CC08091D2
:10276000F102893008F4CEC02091F2023091F302D8
:102770002F5F3F4F88E0A5EFB8E0F90101900D927F
:102780008A95E1F7D9018E910E94BF368A8388230A
:1027900019F481E0898301C019828091070188239F
:1027A000E1F321E030E03F932F93CE0102969F9317
:1027B0008F933F932F93CE01820F931F9F938F93FD
:1027C00082E08F9381E08F9387E58F930E9464105E
:1027D000EDB7FEB73B96EDBF95C0809137048823D7
:1027E00009F090C00E9464958983823019F084308A
:1027F00009F088C020E430E0F8948091C1008F7324
:102800008093C1008091C9008F738093C90080912B
:10281000C100877E8093C1008091C900877E80932C
:10282000C9008091C80087FF03C08091CE00F9CF16
:102830008091C00087FF03C08091C600F9CFE0916E
:10284000F202F091F302E081E13021F482E0809322
:10285000E6022EC0E43611F421E830E081E08093F6
:10286000E602832F99278093CD002093CC0080919E
:10287000CD008093C5008091CC008093C4008091EE
:10288000CA008F7D8093CA008091CA008F7E80939A
:10289000CA008091C9008B7F8093C9008091CA00D3
:1028A00084608093CA008091CA0082608093CA00CD
:1028B0008091CA00877F8093CA008091C200877F81
:1028C0008093C2008091C9008E7F8093C90080915F
:1028D000C10088618093C1008091C90088618093A4
:1028E000C9008091C10080688093C1008091C900B7
:1028F00080688093C90010926E0010926F00109251
:10290000700078948091C90599278436910509F45F
:10291000BBC085369105ACF48136910509F46FC0D2
:10292000823691052CF48B34910509F45DC00FC1FA
:102930008236910509F470C08336910509F47FC091
:1029400006C18C36910509F4EDC08D3691054CF425
:102950008736910509F4F8C08836910509F4B2C0AC
:10296000F6C08437910529F08637910509F4E8C04F
:10297000EEC08091F402A091F202B091F302803196
:1029800040F080E1E2EAF5E00D9001928A95E1F7EE
:102990000DC08D919D910D90BC91A02D8093A205AD
:1029A0009093A305A093A405B093A505809107017A
:1029B0008823E1F31F92809104018F9384E58F9324
:1029C0000E9464108AEF8093EF028FEF80930501DD
:1029D00080EA9FE00E94BE199093E8028093E7028C
:1029E0000F900F900F90B3C0E091F202F091F302BC
:1029F0008081918190938B0180938A01A8C0E0919E
:102A0000F202F091F302808180930601803298F007
:102A10008FE1809306010FC0A091F202B091F30202
:102A20008BE0EAEBF5E00D9001928A95E1F7809159
:102A3000C3058093C3078FEF8093050188C0809101
:102A4000EB029091EC02892B89F4E091F202F09173
:102A5000F302E081EE2351F08AE0E89FC0011124E7
:102A60000E94BE199093950580939405E091F2021F
:102A7000F091F30290818AE0989FC0011124909315
:102A8000EC028093EB0215C08FEF80930501E0917B
:102A9000F202F091F30290818AE0989FC001112424
:102AA0009093EE028093ED02892B19F081E08093E0
:102AB000FC0280EA9FE00E94BE199093E802809396
:102AC000E70245C08FEF80930501E091F202F0919B
:102AD000F302908197FD08C082E08093F902109282
:102AE000EA021092E9021AC0909580915303892B53
:102AF0008093530391818AE0989FC00111249093A1
:102B0000EA028093E90284E08093F90280EA9FE080
:102B10000E94BE199093E8028093E70281E08093BF
:102B2000FD0215C08FEF80930501E091F202F09154
:102B3000F30280818093540381E08093FE0207C0FA
:102B400081E08093FB0203C081E08093FF0210923A
:102B5000F7021092F3021092F2021092F102E3E0F7
:102B6000CE5F0C94809A982F8091C00085FFFCCF97
:102B70009093C60008950F931F9388E18093C1003E
:102B80008091C00082608093C0008091C100806805
:102B90008093C1008091C10080648093C10000E0F7
:102BA00010E00093C5008AE290E08093C400809119
:102BB000ED029091EE020E94BE19909397058093CA
:102BC00096058CED90E00E94BE199093C605809307
:102BD000C50582E0809398051092990510929C0596
:102BE0008BE080939A0510929B051092A00580912E
:102BF000020180939F051093F3020093F20210925A
:102C0000F1021F910F910895A0E1B0E0EAE0F6E132
:102C10000C94619A80910701882309F4C9C28091BC
:102C2000E7029091E8020E94C719882361F0109290
:102C3000EA021092E9021092EE021092ED02109256
:102C4000EC021092EB028091E9029091EA02892B4A
:102C500041F08091A3069091A4060E94C719882391
:102C600029F48091FD02882309F460C08091070156
:102C7000882309F45BC08091F90207ED17E08430E6
:102C8000A8F00E94012580E590E09F938F931F9309
:102C90000F9381E08F938F9388E48F930E94641049
:102CA0002DB73EB7295F3F4F2DBF34C0109255035B
:102CB0008FE494E09F938F9384EF94E29F938F939C
:102CC000E0918405F0918505099584E190E09F935A
:102CD0008F931F930F9381E090E09F938F9389EFE1
:102CE00092E09F938F9382E08F9381E08F9388E4AB
:102CF0008F930E9464108091F902982F8F5F8093C8
:102D0000F9022DB73EB7215F3F4F2DBF943010F031
:102D10001092F9028091E9029091EA020E94BE1994
:102D20009093A4068093A3061092FD028091FE0268
:102D3000882351F180910701882331F10E940125F8
:102D400080E590E09F938F9387ED97E09F938F931B
:102D500021E030E03F932F9382E291E09F938F93A5
:102D60003F932F9384E593E09F938F9383E08F931A
:102D700081E08F938CE48F930E9464101092FE0286
:102D80008DB79EB70F968DBF8091FB028823D1F03F
:102D9000809107018823B1F08AE090E09F938F93A0
:102DA00088E995E09F938F9381E08F938F9386E5D9
:102DB0008F930E9464101092FB022DB73EB7295FDB
:102DC0003F4F2DBF8091FF028823D9F080910701EA
:102DD0008823B9F08BE090E09F938F938AEB95E086
:102DE0009F938F9381E08F93809104018F9387E469
:102DF0008F930E9464101092FF028DB79EB70796C2
:102E00008DBF8091ED029091EE02892B41F080916F
:102E10009605909197050E94C719882321F4809107
:102E2000FC02882341F180910701882321F10E944F
:102E3000993A82E490E09F938F9381E897E09F9383
:102E40008F9381E08F938F9384E48F930E9464101B
:102E50001092FC022DB73EB7295F3F4F2DBF8091E6
:102E6000ED029091EE02009731F00E94BE1990930E
:102E70009705809396058091EB029091EC02892B47
:102E800009F4B7C080919405909195050E94C719E7
:102E9000882309F4AEC080910701882309F4A9C0F2
:102EA000809144089927880F991F880F991F7C01EA
:102EB0000027F7FC0095102F8091920490919304C5
:102EC000A0919404B0919504BC01CD01A801970193
:102ED0000E943A9A309387052093860580918A0450
:102EE00090918B04A0918C04B0918D04BC01CD0114
:102EF000A80197010E943A9A30938905209388058A
:102F000020914C0A30914D0A40914E0A50914F0A3F
:102F1000DA01C90163E0880F991FAA1FBB1F6A95D8
:102F2000D1F7820F931FA41FB51F820F931FA41FF9
:102F3000B51F20913C0130913D0140913E015091DF
:102F40003F01BC01CD010E943A9A30938B0520933A
:102F50008A0580915A0490915B04A0915C04B09121
:102F60005D0459E0B595A795979587955A95D1F742
:102F700080938C058091560490915704A091580439
:102F8000B091590449E0B595A795979587954A95CD
:102F9000D1F780938D058091620490916304A09194
:102FA0006404B091650439E0B595A7959795879528
:102FB0003A95D1F780938E058EE090E09F938F93A2
:102FC00086E895E09F938F9381E08F938F9383E4BE
:102FD0008F930E9464108091EB029091EC020E940A
:102FE000BE1990939505809394058DB79EB707966B
:102FF0008DBF809106018F3F79F1992724E0880FDA
:10300000991F2A95E1F7815B9D4F40E150E0BC019B
:10301000CE0101960E94109880E190E09F938F93DB
:10302000CE0101969F938F9381E090E09F938F93C1
:1030300086E091E09F938F9382E08F9381E08F935E
:1030400081E48F930E9464108FEF809306012DB767
:103050003EB7255F3F4F2DBF8091C3078823C9F03E
:10306000809107018823A9F081E090E09F938F93DE
:1030700083EC97E09F938F9381E08F938F9382E40B
:103080008F930E9464101092C3078DB79EB7079666
:103090008DBF8091FA028823D1F0809107018823A7
:1030A000B1F086E490E09F938F938EE599E09F9333
:1030B0008F9381E08F938F9380E58F930E946410AC
:1030C0001092FA022DB73EB7295F3F4F2DBF809176
:1030D000C5059091C6050E94C719882309F468C0E8
:1030E00080910701882309F463C0809144089927DF
:1030F000880F991F880F991F7C010027F7FC009506
:10310000102F8091920490919304A0919404B09117
:103110009504BC01CD01A80197010E943A9A309311
:10312000B3052093B20580918A0490918B04A091FD
:103130008C04B0918D04BC01CD01A80197010E94BF
:103140003A9A3093B5052093B40580911404809386
:10315000B605809113048093B70588E090E09F93B3
:103160008F9382EB95E09F938F9381E08F9383E021
:103170008F938BE68F930E9464108091B8052DB7D2
:103180003EB7295F3F4F2DBF853018F086E0809312
:10319000B80580919E01882319F483E690E002C06F
:1031A00087EE93E00E94BE199093C6058093C505F3
:1031B000E6E0C05F0C947D9A1F920F920FB60F92BB
:1031C00011242F933F935F936F937F938F939F93DC
:1031D000AF93BF93EF93FF9380911003882329F05F
:1031E0008091100381508093100380912A058823D9
:1031F00019F0815080932A058091180381508093A3
:1032000018038F3F09F04BC089E080931803809129
:10321000160390911703019690931703809316035A
:10322000809111018F5F817080931101882319F4BF
:1032300081E080931503349903C081E080930E03ED
:103240008091110390911203892B11F18091110348
:10325000909112030B9750F08091110390911203FB
:103260000A97909312038093110304C010921203E3
:1032700010921103809111039091120320910A0181
:1032800030910B0182239323892B41F0479A07C089
:103290008FEF9FEF90930B0180930A0147988091E5
:1032A0000E03882309F45AC020919E01222309F0BD
:1032B00055C080913C0A83FF51C086B19927FC011B
:1032C000E071F07084FF13C0809113039091140398
:1032D00001969093140380931303809113039091AC
:1032E0001403895E9340D0F120930E0337C0809180
:1032F000130390911403892B69F18091130390912A
:1033000014038A56914030F5809113039091140371
:1033100069E270E00E94F199809113039091140387
:10332000860F971F909314038093130380911303C8
:10333000909114030B9750F0809113039091140314
:103340000A9790938B0180938A0104C0F0938B01BC
:10335000E0938A011092140310921303FF91EF91EE
:10336000BF91AF919F918F917F916F915F913F91AD
:103370002F910F900FBE0F901F901895209116035C
:1033800030911703280F391FC90101960895209124
:10339000160330911703821B930B892F992786956B
:1033A000807490700895CF93DF930E94BE19EC0152
:1033B000CE010E94C7198823D9F3DF91CF910895D8
:1033C000CF93DF930E94BE19EC0109C080911201D6
:1033D000882329F0909312018FEC80937A00CE011C
:1033E0000E94C719982F882389F3DF91CF91089500
:1033F0009FB7F8945F983E9A469A8091B0008F707C
:103400008093B0008091B00083608093B000809181
:10341000B1008B738093B1008091B1008B60809379
:10342000B1001092B2008FEF8093B3008091B00092
:1034300080688093B000809170008A7F80937000D4
:10344000809170008260809370009FBF08958AE031
:1034500090E00E94BE199093C5078093C40782E054
:1034600085BD83EA84BD17BC84EB88BD86E086BD3C
:1034700080916E00816080936E000895809197081E
:103480002091690182FF30C0909158088CE3989F89
:10349000B00111249091570880E5989FA001112454
:1034A000922F905897FD9D5F9595959586E098028F
:1034B000C00111242091080130910901281B390B0A
:1034C0003093090120930801421753072CF05093C1
:1034D00009014093080108952617370784F0709377
:1034E0000901609308010895822F992736E0880F1B
:1034F000991F3A95E1F79093090180930801089587
:10350000A0E0B0E0E6E8FAE10C94609A80915F08F0
:10351000E82FFF27EE5BFE4F9681D080809110014F
:10352000A92FBB27A7FDB095CB2FDB2F813009F04A
:1035300017C12091920430919304409194045091CA
:103540009504BD01CE010E94C69997FF04C0615841
:103550007F4F8F4F9F4F7B018C01C7E015950795DB
:10356000F794E794CA95D1F78D2D992787FD90950B
:10357000A92FB92F20918A0430918B0440918C049B
:1035800050918D04BC01CD010E94C69997FF04C0E3
:1035900061587F4F8F4F9F4FB7E0959587957795EF
:1035A0006795BA95D1F7F801E701C61BD70BE80B71
:1035B000F90B20910F0530911005C901A3E0880F88
:1035C000991FAA95E1F7821B930BAA2797FDA09557
:1035D000BA2FC81BD90BEA0BFB0B80916701992707
:1035E000AA27BB27BC01CD019E01AF010E94C6994D
:1035F00097FF04C061507E4F8F4F9F4FFC01EB013E
:1036000079E0F595E795D795C7957A95D1F710911B
:103610009708609108017091090112FF05C070932D
:103620000F0160930E0118C040910E0150910F01DF
:1036300080915E08282F3327CB01841B950BB9019D
:103640000E94059A80910E0190910F01860F971F9D
:1036500090930F0180930E0110FF14C080910E0112
:1036600090910F0197FD0F9664E0959587956A9567
:10367000E1F7AA2797FDA095BA2FC80FD91FEA1F17
:10368000FB1F15C080910E0190910F0197FD0F96C1
:1036900054E0959587955A95E1F7AA2797FDA0954F
:1036A000BA2F8C1B9D0BAE0BBF0BFD01EC012091C3
:1036B0009208222321F1332780910A0390910B0372
:1036C000829FA001839F500D929F500D1124CA012B
:1036D000AA2797FDA095BA2F8C0F9D1FAE1FBF1F65
:1036E0002F5F3F4F442737FD4095542FBC01CD013C
:1036F0000E943A9A30930B0320930A0304C0D0939C
:103700000B03C0930A0380915708282F3327220FF9
:10371000331F220F331F80910A0390910B038217EE
:1037200093077CF080915808282F3327220F331FEE
:10373000220F331F80910A0390910B03281739073A
:1037400024F430930B0320930A0380910201843107
:1037500008F4F7C0809110018F5F80931001F3C0CF
:1037600020918A0430918B0440918C0450918D04F7
:10377000BD01CE010E94C69997FF04C061587F4FDA
:103780008F4F9F4F7B018C0187E015950795F7942C
:10379000E7948A95D1F78D2D992787FD9095A92FCC
:1037A000B92F209192043091930440919404509148
:1037B0009504BC01CD010E94C6999B01AC0197FF05
:1037C00004C021583F4F4F4F5F4FC7E05595479575
:1037D00037952795CA95D1F72E0D3F1D401F511FD4
:1037E000809166019927AA27BB27BC01CD010E94C1
:1037F000C69997FF04C061507E4F8F4F9F4FFC01C9
:10380000EB01B9E0F595E795D795C795BA95D1F74E
:10381000809168019927A6E0880F991FAA95E1F782
:1038200040910C0150910D0120915E083327841BBB
:10383000950BB9010E94059A80910C0190910D01A0
:10384000860F971F90930D0180930C01809197082C
:1038500081FF14C080910C0190910D0197FD0F968E
:1038600074E0959587957A95E1F7AA2797FDA0953D
:10387000BA2FC80FD91FEA1FFB1F15C080910C017A
:1038800090910D0197FD0F9664E0959587956A9547
:10389000E1F7AA2797FDA095BA2F8C1B9D0BAE0BC5
:1038A000BF0BFD01EC0120919308222321F1332766
:1038B0008091080390910903829FA001839F500D7E
:1038C000929F500D1124CA01AA2797FDA095BA2FE7
:1038D0008C0F9D1FAE1FBF1F2F5F3F4F442737FD2B
:1038E0004095542FBC01CD010E943A9A30930903B0
:1038F0002093080304C0D0930903C0930803809168
:103900005B08282F3327220F331F220F331F80918C
:10391000080390910903821793077CF080915C085B
:10392000282F3327220F331F220F331F80910803C4
:10393000909109032817390724F430930903209341
:10394000080310921001E7E0CDB7DEB70C947C9A23
:103950001F920F920FB60F9211242F933F934F9304
:103960005F938F939F93EF93FF93809102019091C8
:103970001903843108F04CC0992309F029C18091C2
:10398000B00086FF24C08091B0008F7B8093B00090
:1039900080910A0390910B0387559E4F90930D03DE
:1039A00080930C0325E08D3D920718F08CED95E097
:1039B00005C08757914030F487E791E090930D035D
:1039C00080930C0380910C0390910D03C2C08091F1
:1039D000B00080648093B00080915D08282F332769
:1039E0008DED96E0289FA001299F500D389F500D26
:1039F0001124CA0120911A0330911B03821B930BDF
:103A000090930D0380930C0381E080931001DDC03F
:103A1000992309F0DDC08091B00086FF9FC080919E
:103A2000B0008F7B8093B000E0911C0320915D0873
:103A3000EE23D9F433278DED96E0289FA001299F2E
:103A4000500D389F500D1124CA0120911A03309156
:103A50001B03821B930B90930D0380930C03109216
:103A60001B0310921A03469AB0C02E1738F48AE04E
:103A700090E090930D0380930C03A7C089EA93E034
:103A800090930D0380930C038E2F9927833091051B
:103A9000D9F08430910534F48130910549F00297D2
:103AA00061F020C08430910591F0059799F01AC01B
:103AB00080910A0390910B0304C0809108039091B8
:103AC000090387559E4F1DC08091170A05C080913C
:103AD000F00902C08091200A9927880F991F880F4A
:103AE000991FEFCFFF27EE0FFF1FE25AF64F2081FD
:103AF0003181220F331F80910C0390910D03820FAF
:103B0000931F90930D0380930C0380910C0390916D
:103B10000D0355E08D3D950718F08CED95E005C03F
:103B20008757914030F487E791E090930D0380939D
:103B30000C0320910C0330910D032C5B304030932B
:103B40000D0320930C0380911A0390911B03820FA5
:103B5000931F90931B0380931A0337C08091B0008A
:103B600080648093B0008CEB90E090930D03809381
:103B70000C0380911A0390911B0384549F4F9093E0
:103B80001B0380931A0380910F03882321F08091F7
:103B90003804882321F480910F03823011F4469871
:103BA00001C0469A80911C038F5F80931C03282FCD
:103BB000332780915D0899270196821793072CF48B
:103BC00081E08093100110921C0381E0809319031F
:103BD00020910C0330910D0341E02F37340730F072
:103BE0008FEF8093B3002F5F30400FC02F3F310520
:103BF000C9F0C0F0A9014F5F50404F37510550F454
:103C000080E88093B3002058304030930D03209318
:103C10000C0312C08FEF8093B30050930D034093B9
:103C20000C030AC080910C038093B30010920D0323
:103C300010920C0310921903FF91EF919F918F91B5
:103C40005F914F913F912F910F900FBE0F901F905A
:103C5000189510927C008FEC80937A000895CF9392
:103C6000DF931092250386E987BD83E090E00E94F0
:103C70007A30C82F863E08F4C65FC8BD84E690E05F
:103C80000E94E01980911601909117018152934092
:103C900010F0C0EF02C0C530F8F0C8BD82E390E07C
:103CA0000E94E01984E694E09F938F9383EB95E163
:103CB0009F938F93E0918405F091850509958091FC
:103CC0001601909117010F900F900F900F90815255
:103CD000934010F4C550DFCF6C2F83E090E00E943A
:103CE0008230CF3018F0CCE8D0E002C0C0E0D0E0A5
:103CF000CA3FD105F8F4C7BD82E390E00E94E01905
:103D000086E694E09F938F9383EB95E19F938F9347
:103D1000E0918405F09185050995809116019091B7
:103D200017010F900F900F900F908052934010F05A
:103D30002196DECFC093D4078091350880FF09C05B
:103D40008C2F8A508B3E28F080919D058064809353
:103D50009D05C7BD8CE291E00E94E019DF91CF91F3
:103D60000895EF92FF921F93CF9310E080ED97E0BC
:103D70000E94BE197C01CCE8133019F4CB3008F056
:103D8000C9E010E080913403909135038C5F93403B
:103D900024F48091150181500AC0809134039091E0
:103DA00035038750944034F0809115018F5F8093E4
:103DB000150101C011E080913203909133038C5FB3
:103DC000934024F48091140181500AC08091320301
:103DD000909133038750944034F0809114018F5FA9
:103DE0008093140101C01F5F8091300390913103D3
:103DF0008C5F934024F48091130181500AC080911C
:103E000030039091310387509440C4F080911301A6
:103E10008F5F8093130113C088E694E09F938F9384
:103E200083EB95E19F938F93E0918405F091850555
:103E300009950F900F900F900F905FC01F5F82E168
:103E40008093600380915A038E7F80935A0385EAA2
:103E50008093BC00809115018A3040F480919D05CB
:103E6000816080939D058AE0809315018091150102
:103E7000863F40F080919D05816080939D0585EF90
:103E800080931501809114018A3040F480919D0542
:103E9000826080939D058AE08093140180911401D3
:103EA000863F40F080919D05826080939D0585EF5F
:103EB00080931401809113018A3040F480919D0514
:103EC000846080939D058AE08093130180911301A3
:103ED000863F40F080919D05846080939D0585EF2D
:103EE0008093130180916003882339F0C7010E94F9
:103EF000C719882309F090CFF5CF109212018FECEB
:103F000080937A00809112018823E1F3CA3020F473
:103F10008AE090E00E94E019C15009F02DCF86E4BC
:103F200090E00E94E019CF911F91FF90EF900895CB
:103F30001F920F920FB60F921124EF92FF920F93E0
:103F40001F932F933F934F935F936F937F938F9321
:103F50009F93AF93BF93EF93FF9380913D03282FDF
:103F60003327442755278F5F80933D03F901223182
:103F7000310508F00BC5EA5BFF4F0C948C9A8091D9
:103F800078009091790046C08091780090917900F6
:103F9000B8C180917800909179009093410380930B
:103FA0004003E3C180919C0490919D04209178008E
:103FB00030917900821B930B9093C7078093C607BB
:103FC0008091C6079091C70790934B0380934A0353
:103FD000EAC1809178009091790020919E043091FF
:103FE0009F04821B930B9093D3078093D2078091F9
:103FF000D2079091D30790934D0380934C03C8C48C
:10400000809144039091450320917800309179008C
:10401000820F931F909345038093440381E0B9C4BA
:104020008091420390914303209178003091790070
:10403000820F931F909343038093420384E0A9C4AB
:104040008091980883FF1AC08091200190912101EE
:104050009C01220F331F280F391F40917800509187
:1040600079008BE090E0489FB001499F700D589F08
:10407000700D1124CB016EE170E00FC08091200122
:10408000909121019C01220F331F280F391F80912D
:1040900078009091790063E070E00E94F199260F1A
:1040A000371F369527953695279530932101209314
:1040B000200185E06EC48091780090917900909302
:1040C000C9078093C8078091C8079091C90740919C
:1040D000980450919904841B950B60919704262FA6
:1040E000332727FD3095821B930B90932B038093EE
:1040F0002A038091F703882309F071C080912A0375
:1041000090912B0302977CF172E04E3E57070CF022
:10411000A7C020913E0330913F032B5F3F4F309368
:104120003F0320933E03255030408091000490913E
:104130000104845F914030F4215F3F4F30933F038F
:1041400020933E0380913E0390913F038536910575
:104150000CF486C04F5F5F4F5093990440939804CE
:104160008456904037C080912A0390912B038F5F33
:104170009F4F0CF075C082E0473258070CF470C0B6
:1041800020913E0330913F032550304030933F0350
:1041900020933E032B5F3F4F8091000490910104D8
:1041A000845F914030F42F50304030933F03209390
:1041B0003E0380913E0390913F037FEF8C39970738
:1041C0000CF04EC0415050405093990440939804D5
:1041D0008C599F4F90933F0380933E0341C0809141
:1041E0000C0A90910D0A8F5C9F41D4F180912A03B3
:1041F00090912B030297ACF020913E0330913F0346
:10420000C901019690933F0380933E0389589341DF
:104210003CF166301CF46F5F60939704275833417C
:104220001BC080912A0390912B038F5F9F4FC4F492
:1042300020913E0330913F03C901019790933F03C2
:1042400080933E0388579C4E5CF46B3F1CF061509A
:104250006093970429573C4E30933F0320933E03CD
:1042600080912A0390912B039C01442737FD4095B0
:10427000542F8091520490915304A0915404B09112
:104280005504820F931FA41FB51F8093520490936F
:104290005304A0935404B0935504209152043091D8
:1042A0005304409154045091550457FF04C02150C9
:1042B0003C4F4F4F5F4F7AE055954795379527957F
:1042C0007A95D1F78091520490915304A0915404AF
:1042D000B0915504821B930BA40BB50B8093520431
:1042E00090935304A0935404B09355042EC180912D
:1042F0004203909143032091780030917900820F1E
:10430000931F909343038093420310923C0343C353
:10431000809102018A3071F4809178009091790047
:104320002091400330914103820F931F019696958F
:10433000879517C04091400350914103843158F054
:104340002091780030917900240F351F8FEF97E08E
:10435000821B930B06C08091780090917900840FA6
:10436000951F909331038093300386E012C38091B0
:104370009C0490919D042091780030917900821BDB
:10438000930B9093C7078093C6078091C6079091BF
:10439000C70720914A0330914B03820F931F9093DC
:1043A0002F0380932E0387E0F4C2809178009091D0
:1043B000790020919E0430919F04821B930B90936F
:1043C000D3078093D2078091D2079091D307209191
:1043D0004C0330914D03820F931F90932D038093D4
:1043E0002C03D6C22091440330914503809178007C
:1043F00090917900280F391F30934503209344038F
:10440000809102018A3019F4220F331F04C0220F59
:10441000331F220F331F3093450320934403209111
:10442000440330914503C90137FD079643E0959554
:1044300087954A95E1F790933503809334038091F3
:10444000460390914703820F931F97FD0196959520
:10445000879590934703809346032091A804309159
:10446000A904821B930B90931F0180931E0120913E
:104470003A0330913B0380911E0190911F01280F58
:10448000391F37FF02C02F5F3F4F35952795309377
:104490003B0320933A03C2CD209142033091430362
:1044A0008091780090917900280F391F3093430351
:1044B00020934203809102018A3019F4220F331FA6
:1044C00004C0220F331F220F331F30934303209366
:1044D00042032091420330914303C90137FD0796FF
:1044E000B3E095958795BA95E1F790933303809360
:1044F00032038091480390914903820F931F97FDE7
:104500000196959587959093490380934803209150
:10451000A6043091A704821B930B90931D018093F6
:104520001C01209138033091390380911C01909136
:104530001D01280F391F37FF02C02F5F3F4F3595F0
:104540002795309339032093380383E022C280916A
:10455000F703882309F180E00E9439949B01AC01A4
:1045600020503F4F4F4F5F4F57FF06C09B01AC019C
:1045700021503D4F4F4F5F4FE9E055954795379597
:104580002795EA95D1F720931D0330931E0340939E
:104590001F035093200310C0809132049091330484
:1045A000A0913404B091350480931D0390931E03B1
:1045B000A0931F03B093200310923D0381E08093EA
:1045C000120180912103909122030196909322037E
:1045D0008093210380917800909179009093170146
:1045E000809316018091F703882309F47EC080919F
:1045F0001601909117017C01002711278091250356
:10460000992787FD9095A92FB92FBC01CD012BE0EB
:1046100032E040E050E00E94C699DC01CB01E81A8C
:10462000F90A0A0B1B0BE0924E03F0924F03009322
:1046300050031093510320911801309119014091BA
:104640001A0150911B0157FF04C0215F3F4F4F4F8C
:104650005F4F74E055954795379527957A95D1F733
:104660008091180190911901A0911A01B0911B013C
:10467000821B930BA40BB50B809318019093190127
:10468000A0931A01B0931B01809118019091190118
:10469000A0911A01B0911B018E0D9F1DA01FB11F8B
:1046A0008093180190931901A0931A01B0931B01F4
:1046B0008091CA079091CB07A091CC07B091CD070C
:1046C000209118013091190140911A0150911B015C
:1046D000821B930BA40BB50B80933204909333048D
:1046E000A0933404B093350453C180911601909186
:1046F0001701AA27BB2720914E0330914F03409109
:10470000500350915103280F391F4A1F5B1F2093FC
:104710004E0330934F0340935003509351038091C5
:1047200052038F5F80935203803108F431C180912E
:10473000180190911901A0911A01B0911B017C01FF
:104740008D0163E0EE0CFF1C001F111F6A95D1F76D
:10475000E81AF90A0A0B1B0BE20EF31E041F151FC1
:1047600080912503992787FD9095A92FB92FBC012A
:10477000CD0120EB30E240E050E00E94C699DC0120
:10478000CB01E81AF90A0A0B1B0BD801C7010496E2
:10479000A11DB11DB7FF05C0D801C7010B96A11D12
:1047A000B11D23E0B595A795979587952A95D1F7E3
:1047B0008093180190931901A0931A01B0931B01E3
:1047C000E090CA07F090CB070091CC071091CD077D
:1047D0008091180190911901A0911A01B0911B01CB
:1047E000E81AF90A0A0B1B0BE0923204F092330428
:1047F000009334041093350420912603309127034D
:10480000409128035091290357FF04C0215F3F4F77
:104810004F4F5F4F84E055954795379527958A957B
:10482000D1F78091260390912703A0912803B0919E
:104830002903821B930BA40BB50B80932603909343
:104840002703A0932803B093290380912603909116
:104850002703A0912803B09129038E0D9F1DA01F4F
:10486000B11F8093260390932703A0932803B0934E
:1048700029038091260390912703A0912803B091EA
:104880002903B7FF03C00F96A11DB11D14E0B59514
:10489000A795979587951A95D1F720913204309175
:1048A0003304281B390B64E0213036071CF020E06C
:1048B00034E006C07CEF2030370714F420E03CEFF2
:1048C00080912303909124038091230390912403EA
:1048D00097FF03C0909581959F4FA901F3E0440F86
:1048E000551FFA95E1F78D5B9240C4F08091230348
:1048F000909124039C01E4E0220F331FEA95E1F735
:10490000281B390B240F351F37FF02C0215F3F4F93
:1049100074E0359527957A95E1F717C080912303C8
:10492000909124039C0165E0220F331F6A95E1F703
:10493000281B390B240F351F37FF02C0215E3F4F64
:1049400045E0359527954A95E1F730932403209368
:10495000230380914E0390914F03A0915003B09197
:104960005103B7FF03C00196A11DB11DB595A795D1
:104970009795879580934E0390934F03A093500390
:10498000B093510388E08093520302C010923D031C
:1049900082E080933C0380913C0380937C00809173
:1049A0003D03882319F08FEC80937A00FF91EF91FB
:1049B000BF91AF919F918F917F916F915F914F9137
:1049C0003F912F911F910F91FF90EF900F900FBE8D
:1049D0000F901F90189590E2E7EDF7E08FE4919328
:1049E000815087FFFCCF089590915503903540F496
:1049F000E92FFF27E952F84F80839F5F909355037B
:104A00000895AF92BF92CF92DF92FF920F931F93C0
:104A1000CF93DF932091530320FF0AC0809154036A
:104A2000882311F0815002C08091220180935403A9
:104A300021FF0CC09091540380912201981719F422
:104A40001092540303C09F5F90935403822F9927C1
:104A500080FF04C081FF02C0109254030E94EB2427
:104A600080915403282F332794EFC92E94E2D92E36
:104A7000C0918405D09185058A3098F481E18093B6
:104A800055033F932F938FE994E09F938F93DF9289
:104A9000CF92FE0109952DB73EB72A5F3F4F2DBF3C
:104AA00011C080E1809355033F932F9384EA94E0F3
:104AB0009F938F93DF92CF92FE0109958DB79EB79A
:104AC00006968DBF20915403822F9927AA27BB27D2
:104AD000FC01419710F00C94522EE85AFF4F04EF5E
:104AE000C02E04E2D02EC0918405D09185050C948F
:104AF0008C9A1092550389EA94E09F938F9304EF68
:104B000014E2DF92CF92FE01099584E18093550370
:104B10000F900F900F900F9081E690E09F938F93EE
:104B20001F921F9282E090E09F938F9380910201E9
:104B30006AE00E94E599892F99279F938F9380912E
:104B400002010E94E59999279F938F9389EB94E046
:104B50009F938F93DF92CF92E0918405F09185052A
:104B6000099588E280935503EDB7FEB73E96EDBFF9
:104B700088EA98E09F938F938091000199279F93F3
:104B80008F9381ED94E09F938F93DF92CF92E0918A
:104B90008405F0918505099580919E0599272DB78B
:104BA0003EB7285F3F4F2DBFEC01C071D07084FF2E
:104BB00006C08CE3809355038FED94E0FEC0909186
:104BC0001605992359F18CE380935503892F992772
:104BD0009F938F938CEE94E09F938F931F930F93EB
:104BE000E0918405F09185050995DF93CF9390912D
:104BF000160581E1989FC0011124865A954F9F9315
:104C00008F931F930F93E0918405F091850509958B
:104C10008DB79EB70C968DBF0C945B2E90919D0521
:104C2000992351F08CE380935503892F99279F9303
:104C30008F9384EF94E038C190915B03992371F0D6
:104C40008CE380935503892F99279F938F938BE053
:104C500095E09F938F931F930F93E6C48091360145
:104C600090913701069710F00C945B2E8CE38093A3
:104C7000550380E295E0A8C780913C0A14EFC12E4D
:104C800014E2D12EC0918405D091850580FF82C0A9
:104C9000109255038091320490913304A091340412
:104CA000B0913504BC01CD0125E030E040E050E09A
:104CB0000E943A9A3F932F938DE295E09F938F93B2
:104CC000DF92CF92FE01099584E1809355038DB761
:104CD0009EB706968DBF80912E0490912F04A091CF
:104CE0003004B0913104BC01CD0125E030E040E05A
:104CF00050E00E943A9A3F932F938AE395E09F9366
:104D00008F93DF92CF92E0918405F091850509950C
:104D100088E280935503EDB7FEB73696EDBF8091DC
:104D20001601909117019F938F9387E495E09F93CD
:104D30008F93DF92CF92E0918405F09185050995DC
:104D40008CE3809355032DB73EB72A5F3F4F2DBFAD
:104D500087B599279F938F9384E595E09F938F93D1
:104D6000DF92CF92E0918405F091850509958DB78A
:104D70009EB706968DBF8091F703882309F49BC7E1
:104D80008DE48093550387B599279F938F9381E690
:104D900095E0CFC41092550385E695E09F938F93DD
:104DA000DF92CF92FE01099584E1809355030F9025
:104DB0000F900F900F9084E795E09F938F93DF9271
:104DC000CF9206C7109255038DE795E09F938F937E
:104DD00004EF14E2DF92CF92FE01099584E1809303
:104DE00055030F900F900F900F9080919204909127
:104DF0009304A0919404B0919504B7FF04C081502E
:104E00009C4FAF4FBF4FCAE0B595A7959795879533
:104E1000CA95D1F7BF93AF939F938F938AE895E09C
:104E20009F938F931F930F93E0918405F0918505D5
:104E3000099588E2809355032DB73EB7285F3F4F11
:104E40002DBF80918A0490918B04A0918C04B09125
:104E50008D04B7FF04C081509C4FAF4FBF4FFAE0A5
:104E6000B595A79597958795FA95D1F7BF93AF9389
:104E70009F938F9389E995E09F938F931F930F934F
:104E8000E0918405F091850509958CE380935503A5
:104E90008DB79EB708968DBF8091F8099091F9095A
:104EA0009F938F9388EA95E09F938F931F930F931F
:104EB00044C4E1E0FE2EC1E0D0E000E619E09F2D01
:104EC000969584E1989FC001112480935503F801C1
:104ED000828193819F938F932196DF93CF93219724
:104EE000808191819F938F93DF93CF9387EB95E0A0
:104EF0009F938F9384EF94E29F938F93E091840527
:104F0000F091850509952DB73EB7245F3F4F2DBF22
:104F100032E0F30E22960C5F1F4F88E08F1578F673
:104F2000CAC61092550380912A08E82FFF27EE0F7A
:104F3000FF1FE25AF64F808191819F938F9380915A
:104F40002908E82FFF27EE0FFF1FE25AF64F808156
:104F500091819F938F9389EC95E09F938F93DF923C
:104F6000CF92FE01099584E180935503EDB7FEB71A
:104F70003896EDBF80912C08E82FFF27EE0FFF1F1A
:104F8000E25AF64F808191819F938F9380912B08F5
:104F9000E82FFF27EE0FFF1FE25AF64F8081918125
:104FA00081589F4F9F938F9389ED95E09F938F93A7
:104FB000DF92CF92E0918405F0918505099588E212
:104FC000809355032DB73EB7285F3F4F2DBF80918B
:104FD0002E08E82FFF27EE0FFF1FE25AF64F8081C1
:104FE000918181589F4F9F938F9380912D08E82F37
:104FF000FF27EE0FFF1FE25AF64F80819181815803
:105000009F4F9F938F9389EE95E09F938F93DF92AD
:10501000CF92E0918405F091850509958CE380930A
:1050200055038DB79EB708968DBF80913008E82F45
:10503000FF27EE0FFF1FE25AF64F808191818158C2
:105040009F4F9F938F9380912F08E82FFF27EE0F9C
:10505000FF1FE25AF64F8081918181589F4F9F93A5
:105060008F9389EF95E06BC21092550389E096E02B
:105070009F938F9304EF14E2DF92CF92FE01099584
:10508000809102010F900F900F900F908A3009F0DD
:10509000A9C084E1809355038091A8049091A9044C
:1050A0009C0197FF02C0295F3F4F287F821B930B13
:1050B0009F938F938091A8049091A90497FD0796E0
:1050C00073E0959587957A95E1F79F938F9320915B
:1050D000A8043091A90437FF02C0295F3F4F63E065
:1050E000359527956A95E1F78091340390913503C2
:1050F000821B930B9F938F9387E196E09F938F93EF
:105100001F930F93E0918405F0918505099588E23E
:10511000809355032DB73EB7265F3F4F2DBF80913B
:10512000A6049091A7049C0197FF02C0295F3F4FFE
:10513000287F821B930B9F938F938091A60490915D
:10514000A70497FD079653E0959587955A95E1F743
:105150009F938F932091A6043091A70437FF02C03C
:10516000295F3F4F43E0359527954A95E1F78091B8
:10517000320390913303821B930B9F938F9388E2AA
:1051800096E09F938F931F930F93E0918405F09186
:10519000850509958CE3809355038DB79EB70A96D4
:1051A0008DBF8091A4049091A5049F938F938091CB
:1051B000A4049091A5042091300330913103821B07
:1051C000930B9F938F9389E396E09F938F931F9305
:1051D0000F93E0918405F09185050995EDB7FEB731
:1051E0003896B3C28B3019F0843108F4A9C084E139
:1051F000809355038091A8049091A9049C0197FF86
:1052000002C0215F3F4F207F821B930B97FD0196C9
:10521000959587959F938F938091A8049091A90469
:1052200097FD0F9624E0959587952A95E1F79F9332
:105230008F932091A8043091A90437FF02C0295F01
:105240003F4FC3E035952795CA95E1F78091340328
:1052500090913503821B930B9F938F9387E496E085
:105260009F938F931F930F93E0918405F091850591
:10527000099588E2809355032DB73EB7265F3F4FCF
:105280002DBF8091A6049091A7049C0197FF02C0B6
:10529000215F3F4F207F821B930B97FD01969595D1
:1052A00087959F938F938091A6049091A70497FD73
:1052B0000F96A4E095958795AA95E1F79F938F9314
:1052C0002091A6043091A70437FF02C0295F3F4F09
:1052D000F3E035952795FA95E1F7809132039091A7
:1052E0003303821B930B9F938F9389E596E09F93E3
:1052F0008F931F930F93E0918405F0918505099595
:105300008CE3809355038DB79EB70A968DBF80912D
:10531000A4049091A50497FD0196959587959F9378
:105320008F938091A4049091A50420913003309133
:105330003103821B930B9F938F938BE696E045CFAF
:105340008D3009F0B8C484E1809355038091150134
:1053500099279F938F938091A8049091A90497FD1A
:105360000F9674E0959587957A95E1F79F938F93C3
:105370002091A8043091A90437FF02C0295F3F4F54
:1053800063E0359527956A95E1F780913403909114
:105390003503821B930B9F938F938AE796E09F932D
:1053A0008F931F930F93E0918405F09185050995E4
:1053B00088E2809355032DB73EB7265F3F4F2DBF40
:1053C0008091140199279F938F938091A6049091C7
:1053D000A70497FD0F9654E0959587955A95E1F7A8
:1053E0009F938F932091A6043091A70437FF02C0AA
:1053F000295F3F4F43E0359527954A95E1F7809126
:10540000320390913303821B930B9F938F938EE80B
:1054100096E09F938F931F930F93E0918405F091F3
:10542000850509958CE3809355038DB79EB70A9641
:105430008DBF8091130199279F938F938091A4042E
:105440009091A50497FD0196959587959F938F93CD
:105450008091A4049091A5042091300330913103F0
:10546000821B930B9F938F9382EA96E09F938F9377
:105470001F930F93E0918405F09185050995EDB791
:10548000FEB73A9662C11092550386EB96E09F9361
:105490008F93DF92CF92FE01099584E180935503AB
:1054A0000F900F900F900F9080919E0490919F0409
:1054B0009F938F9380912C0390912D039F938F93B3
:1054C00083EC96E09F938F93DF92CF92E0918405D7
:1054D000F0918505099588E2809355032DB73EB775
:1054E000285F3F4F2DBF80919C0490919D049F9316
:1054F0008F9380912E0390912F039F938F9382ED32
:1055000096E09F938F93DF92CF92E0918405F09184
:10551000850509958CE3809355038DB79EB7089652
:105520008DBF80919804909199049F938F9380915F
:105530002A0390912B039F938F9381EE96E09F9384
:105540008F93DF92CF9245CE109255038091200128
:10555000909121016AE070E00E94059A9F938F93D9
:1055600080912001909121016AE070E00E94059AEB
:105570007F936F9380EF96E09F938F93DF92CF920C
:10558000FE01099584E1809355032DB73EB7285F4E
:105590003F4F2DBF8091DC0A9091DD0A6AE070E0F8
:1055A0000E94F1999F938F938091DC0A9091DD0A7C
:1055B0006AE070E00E94F1997F936F9384E097E036
:1055C0009F938F93DF92CF92E0918405F0918505B0
:1055D000099588E2809355038DB79EB708968DBFD5
:1055E0008091DE0A9091DF0A9F938F9388E197E084
:1055F0009F938F93DF92CF92E0918405F091850580
:1056000009958CE380935503EDB7FEB73696EDBF51
:105610008091E00A9091E10A9F938F9388E297E04E
:105620009F938F93DF92CF92E0918405F09185054F
:1056300009952DB73EB72A5F3F4F45C110925503DC
:105640008AE397E09F938F93DF92CF92FE010995B3
:1056500088E2809355030F900F900F900F908091E8
:10566000380499279F938F9383E497E09F938F93B8
:10567000DF92CF92E0918405F091850509958CE346
:10568000809355038DB79EB706968DBF80915D09B7
:10569000992701979F938F9383E597E04AC01092D3
:1056A000550383E697E09F938F93DF92CF92FE019D
:1056B000099584E1809355030F900F900F900F9000
:1056C00080918A0190918B019F938F938BE697E055
:1056D0009F938F93DF92CF92E0918405F09185059F
:1056E000099588E2809355032DB73EB72A5F3F4F57
:1056F0002DBF8091F8099091F9099F938F9389E7C5
:1057000097E09F938F93DF92CF92E0918405F09181
:10571000850509958CE3809355038DB79EB7069652
:105720008DBF80915004909151049F938F9387E88F
:1057300097E09F938F93DF92CF92E0918405F09151
:1057400085050995EDB7FEB73696EDBFB4C2C9E33E
:10575000CC2EC4E0DC2E20E030E0E901B3E0FB2EEB
:10576000C0935503F60181916F0199279F938F9301
:1057700089010F5F1F4F1F930F9385E997E09F9358
:105780008F9384EF94E29F938F93E0918405F0913F
:10579000850509952DB73EB7285F3F4F2DBFFA9479
:1057A00064969801F7FEDCCF86C2ADE3CA2EA4E072
:1057B000DA2EC0E0D0E08E01F3E0FF2E0093550317
:1057C000F60181916F0199279F938F932596DF931F
:1057D000CF9382EA97E09F938F9384EF94E29F9315
:1057E0008F93E0918405F091850509952DB73EB71B
:1057F000285F3F4F2DBFFA940C5E1F4F2497F7FE92
:10580000DDCF59C2109255038FEA97E09F938F9393
:1058100004EF14E2DF92CF92FE01099584E18093B8
:1058200055030F900F900F900F9080916901992769
:105830009F938F9387EB97E09F938F93DF92CF9205
:10584000E0918405F0918505099588E280935503E0
:105850008DB79EB706968DBF80910A0390910B037A
:1058600097FD039695958795959587959F938F932B
:1058700085EC97E09F938F931F930F93E09184059E
:10588000F091850509958CE380935503EDB7FEB73C
:105890003696EDBF8091580899279F938F938091FA
:1058A000570899279F938F9383ED97E09F938F934A
:1058B0001F930F93E0918405F091850509952DB70D
:1058C0003EB7285F3F4F2DBFF6C11092550381EEC2
:1058D00097E09F938F9374EFA72E74E2B72EDF9219
:1058E000CF92FE0109950F900F900F900F90CDEF82
:1058F000D8E000E010E062E0F62E802F8C5E80930E
:1059000055038B8D99278F7790709F938F938B89F9
:1059100099278F7790709F938F938B8599278F7797
:1059200090709F938F938B8199278F7790709F931F
:105930008F9381EF97E09F938F93BF92AF92E09107
:105940008405F091850509958DB79EB70C968DBF9E
:10595000FA940C5E1F4FA096F7FECFCFACC1109209
:10596000550382E098E09F938F9354EFA52E54E265
:10597000B52EDF92CF92FE0109950F900F900F90F8
:105980000F90CDEFD8E000E010E042E0F42E802F41
:105990008C5E809355038F8D992787FD90959F93FB
:1059A0008F938F89992787FD90959F938F938F85EC
:1059B000992787FD90959F938F938F81992787FDD6
:1059C00090959F938F9381E198E09F938F93BF92DF
:1059D000AF92E0918405F09185050995EDB7FEB78A
:1059E0003C96EDBFFA940C5E1F4FA096F7FECFCF0A
:1059F00062C11092550382E298E09F938F9304EF67
:105A000014E2DF92CF92FE01099584E18093550361
:105A10000F900F900F900F9080911809881F882782
:105A2000881F97E0899FC00111248D969F938F93C3
:105A300080911009881F8827881F96E0899FC001E0
:105A400011248D969F938F9380910809881F882732
:105A5000881F95E0899FC00111248D969F938F9395
:105A600080910009881F8827881F9927880F991F10
:105A7000880F991F8D969F938F9381E398E09F9352
:105A80008F93DF92CF92E0918405F091850509957F
:105A900088E2809355032DB73EB7245F3F4F2DBF5B
:105AA00080913809881F8827881F9BE0899FC00143
:105AB00011248D969F938F9380913009881F88279A
:105AC000881F9AE0899FC00111248D969F938F9320
:105AD00080912809881F8827881F99E0899FC00125
:105AE00011248D969F938F9380912009881F88277A
:105AF000881F992723E0880F991F2A95E1F78D9633
:105B00009F938F9385E498E09F938F93DF92CF923A
:105B1000E0918405F091850509958CE38093550308
:105B20008DB79EB70C968DBF80914009881F88273E
:105B3000881F9CE0899FC00111248D969F938F93AD
:105B400089E598E09F938F93DF92CF92E09184054F
:105B5000F0918505099580914809EDB7FEB7369615
:105B6000EDBF87FF12C080E4809355038AE698E07A
:105B70009F938F93DF92CF92E0918405F0918505FA
:105B800009950F900F900F900F908091500987FF0B
:105B900012C084E4809355038DE698E09F938F9321
:105BA0001F930F93E0918405F091850509950F905F
:105BB0000F900F900F908091580987FF7CC088E468
:105BC0008093550380E798E09F938F931F930F93E3
:105BD000E0918405F091850509950F900F900F9045
:105BE0000F9069C01092550383E798E09F938F93BD
:105BF000DF92CF92FE01099584E1809355030F90C7
:105C00000F900F900F908091E0029091E1029F938E
:105C10008F9381E898E09F938F93DF92CF92E091EA
:105C20008405F0918505099588E2809355032DB789
:105C30003EB72A5F3F4F2DBF8091E2029091E30271
:105C40009F938F938EE898E09F938F93DF92CF92EC
:105C5000E0918405F0918505099589E480935503C9
:105C60008DB79EB706968DBF8BE998E09F938F9373
:105C7000DF92CF92E0918405F0918505099580919E
:105C800053030F900F900F900F9083FF14C010924A
:105C9000E3021092E20260E070E08EE090E00E9489
:105CA000933009C080912201281719F421502093C4
:105CB00022011092540310925303DF91CF911F9150
:105CC0000F91FF90DF90CF90BF90AF900895F9991A
:105CD000FECF92BD81BDF89A80B599270895F999B4
:105CE000FECF1FBA92BD81BD60BD0FB6F894FA9A7F
:105CF000F99A0FBE08954AEA20E030E026173707E8
:105D000040F4FC018191480F2F5F3F4F2617370762
:105D1000C8F3842F99270895EAEA40E050E0461737
:105D2000570778F49C01F999FECF32BD21BDF89A4E
:105D300080B5E80F4F5F5F4F2F5F3F4F4617570704
:105D400090F38E2F9927089581E080932B0882E0AD
:105D500080932A0883E08093290884E080932C08AC
:105D600085E080932D0886E080932E0887E080935D
:105D70002F0888E08093300889E0809331088AE01A
:105D8000809332088BE0809333088CE08093340852
:105D900008958FE5809328088CE0EAE9F8E01192F5
:105DA0008A95E9F780910201843150F08AE080936E
:105DB000480810926C088BE1809344088EE40AC076
:105DC00083E08093480880E280936C088EE18093A2
:105DD000440885E58093690880936A0880E280938F
:105DE0006B08109296088AE68093350882E68093C5
:105DF000980886E080934F0810928C0810928908CA
:105E000048E04093420886EE8093430830E43093A4
:105E100045082EE12093360885E08093380890915C
:105E2000F7039923A9F084E18093390888E28093ED
:105E3000370820933B0881E080933C0810923D088E
:105E40008FE780933E083093990820938F0812C003
:105E50008FE0809339082093370890933B08409354
:105E60003C0884E180933D0890933E083093990864
:105E700090938F088FE080933A08109294088CE0FA
:105E8000809395081092510810925208109253086E
:105E90001092540810926E0810926F0810927008B9
:105EA0001092710890E89093550842E34093560889
:105EB00072E07093970888E18093570886EE80938C
:105EC000580884E080935D085DE750936008509324
:105ED0006108509362089093590865E560935A08E9
:105EE00086E480935B088CED80935C088CE3809360
:105EF0005E0810925F088FE58093720883EF8093AD
:105F000074088AEA809376088093770898E29093E1
:105F100073089093750810927808409363082AE5F7
:105F2000209364084093650836E03093790884E64E
:105F300080937A0880937B0820937C0888E780937D
:105F40007D08909381088BE480937E0860937F089E
:105F5000809380083093820888E080938308409380
:105F600084088AE28093850885EF809386088CE810
:105F7000809387087093880810928A0810928B0883
:105F800081E280934C0881E480934D0820934E0871
:105F900010928D0810928E0886E980939008509395
:105FA000660884E380936708109291081092920823
:105FB0001092930808950E94C92E8AE080933F08AA
:105FC00080E18093400826E0209341089AE5909371
:105FD000460888E7809347089093490880934A08C9
:105FE00020934B0880E2809350088CE380936808EC
:105FF0008BE480936D0886E491E6A3E7B4E7809391
:106000009A0890939B08A0939C08B0939D086EE714
:1060100070E088E298E00E947B2E8093A6080895A5
:10602000CF93DF930E94C92E88E080933F0830E130
:106030003093400826E02093410894E69093460868
:1060400088E7809347089093490880934A082093F3
:106050004B083093500886E48093680880936D085D
:10606000AAE9B8E085E0E3E2F1E0ED0101900992F0
:106070008A95E1F76EE770E0CD01825790400E946B
:106080007B2E8093A608DF91CF9108950E94C92EA0
:1060900026E020933F088AE08093400884E08093C4
:1060A000410894E69093460888E7809347089093C8
:1060B000490880934A0820934B0880E18093500858
:1060C00086E48093680880936D0885E491E6A3E7F1
:1060D000B9E780939A0890939B08A0939C08B0938B
:1060E0009D086EE770E088E298E00E947B2E809326
:1060F000A6080895F999FECF92BD81BDF89A80B5A2
:1061000099270895F999FECF1FBA92BD81BD60BD50
:106110000FB6F894FA9AF99A0FBE089567E67EE2F0
:106120000E94549808954FE65EE20E948E9808956A
:10613000EF92FF920F931F93CF93C82F815085301A
:1061400008F0C3E08FE7C89F8001112485EEE82E98
:106150008FEFF82EE00EF11E6EE770E0C7010E948F
:106160008C2E682F98012D593F4F8FB39927AC0182
:106170004270507081FDF9CF32BD21BDF89A80B5D3
:10618000861711F0CA0123C08FB399279C01227092
:10619000307081FDF9CFF2BCE1BCF89A80B58F3543
:1061A00011F0C90114C08FE7C89FC00111244B979B
:1061B00027E63EE24FE750E0BC0188E298E00E940B
:1061C0002F980E94AA740E94D49281E090E0CF910F
:1061D0001F910F91FF90EF900895282F863010F0B7
:1061E00025E003C0882309F421E020930001F999F8
:1061F000FECF1FBA82E090E092BD81BD20BD0FB6F8
:10620000F894FA9AF99A0FBE0895CF93C82F809107
:1062100028088F3509F051C0C63010F0C5E003C022
:10622000CC2309F44AC00E9418978091990882FFF4
:1062300007C080914D08843618F080E580934D08A2
:106240006EE770E088E298E00E947B2E8093A608BB
:106250008FE7C89FC00111242FE63EE24FE750E0D0
:1062600068E278E04B970E946C982FE63EE24CE0A3
:1062700050E069E278E080E590E00E946C986CE084
:1062800070E089E298E00E947B2E282FF999FECFDA
:106290001FBA8CE590E092BD81BD20BD0FB6F89489
:1062A000FA9AF99A0FBE8C2F0E94ED300E94AA74C0
:1062B0000E94D49281E090E002C080E090E0CF9113
:1062C00008956DE470E088EE93E00E948C2E482FD4
:1062D0008FB399279C012270307081FDF9CF85E33F
:1062E00094E092BD81BDF89A80B5841779F48FB39C
:1062F00099279C012270307081FDF9CF88EE93E0E0
:1063000092BD81BDF89A80B5813011F0C901089520
:1063100027E63EE24EE450E068EE73E087EA98E05C
:106320000E942F9881E090E008958091A708813025
:10633000A9F46DE470E087EA98E00E947B2E8093D8
:10634000F4082FE63EE24EE450E067EA78E088EE9B
:1063500093E00E946C9881E090E0089580E090E0E6
:106360000895CF93DF9381E08093A708E7EAF8E0F0
:106370008FE0158616861786108A8150349687FF1F
:10638000F8CF80E48093B4088093B5081092B608E3
:106390008093B7088093B80890EC9093B908109256
:1063A000BA088093BB088093BC081092BD089093F4
:1063B000BE089093BF088093C0081092C1088093D4
:1063C000C2089093C308A8EAB8E08CE0E9E2F1E0E3
:1063D000ED01019009928A95E1F76DE470E0CD013D
:1063E00001970E947B2E8093F408DF91CF9108954E
:1063F000F999FECF82E090E092BD81BDF89A80B518
:10640000282F863078F023E0322FF999FECF1FBA7B
:1064100082E090E092BD81BD30BD0FB6F894FA9A4B
:10642000F99A0FBE20930001822F992708951F9398
:10643000CF93C82F162F863010F0C5E003C08823F5
:1064400009F4C1E08C2F99278230910541F0833007
:10645000910544F4019731F40E94DB2F05C00E949E
:10646000103002C00E9446301123E1F06CE070E071
:1064700080E590E00E948C2E282FF999FECF8CE5C4
:1064800090E092BD81BDF89A80B5821759F427E655
:106490003EE24CE050E060E570E089E298E00E9466
:1064A0002F9802C00E94A42E8C2F0E940531CF91FC
:1064B0001F910895DF92EF92FF920F931F93CF9356
:1064C000FF24DF2CEF2C81E190E00E947A30909144
:1064D0000201981791F1963169F481E190E00E94F0
:1064E0007A30853139F44C9905C06F2D81E090E008
:1064F0000E9482306091020181E190E00E9482302E
:1065000088E190E028E00FB6F894A89580936000A9
:106510000FBE2093600083EA98E09F938F9383EBF4
:1065200095E19F938F93E0918405F09185050995FE
:106530000F900F900F900F90FFCF81E090E00E949E
:106540007A308F3511F031E0E32E6CE070E080E5B9
:1065500090E00E948C2EC82FF999FECF8CE590E038
:1065600092BD81BDF89A80B58C1711F421E0D22E2E
:10657000C1E001E010E0EE2029F48C2F0E94983059
:106580008823B9F591E0F92E1F930F938BEC98E0D7
:106590009F938F9383EB95E19F938F93E091840575
:1065A000F091850509952DB73EB72A5F3F4F2DBF66
:1065B0000130110521F00230110521F006C00E94C2
:1065C000DB2F05C00E94103002C00E944630DD2043
:1065D00059F027E63EE24CE050E060E570E089E2E9
:1065E00098E00E942F9802C00E94A42E8C2F0E9437
:1065F0000531CF5F0F5F1F4FC63008F4BCCFFF20BF
:1066000019F083E00E94ED300E94F831C82F0E94FB
:1066100098308C2F99279F938F9381EF98E09F93C9
:106620008F9303EB15E11F930F93E0918405F09195
:106630008505099581E090E00E947A302DB73EB73C
:106640002A5F3F4F2DBF8F3F21F00E946131882389
:1066500099F48AE099E09F938F931F930F93E091B1
:106660008405F091850509950E94B1310E9495310C
:106670000F900F900F900F90EE2029F06FE581E0C2
:1066800090E00E9482301092270890E0E4EBF8E05E
:10669000CFE08081349618160CF49F5FC150C7FF7D
:1066A000F8CF90932708892F99279F938F9388EA93
:1066B00098E09F938F938BE299E09F938F931F9322
:1066C0000F93E0918405F091850509950E946A0970
:1066D0008DB79EB708968DBFCF911F910F91FF90F8
:1066E000EF90DF900895982F2FB7F8943998389A43
:1066F00088B1836088B98091B9008C7F8093B9009C
:106700008AE28093B8001092600310925E031092A8
:106710005D03992379F0EDEFF8E08BE010821182B0
:106720001282138214821582168217828150389643
:1067300087FFF4CF78942FBF08951092600384E907
:106740008093BC0080E88093BC001092BD00109242
:10675000BA001092BB001092B9001092B8001092CB
:106760005C0380E00E9473331092BB0085E8809345
:10677000BC0080915A03826080935A0308951F924F
:106780000F920FB60F9211242F933F934F935F9365
:106790008F939F93EF93FF9380916003282F33276C
:1067A000442755278F5F80936003F9012731310516
:1067B00008F0C2C2E759FF4F0C948C9A81E0809395
:1067C0005C0309C080915E038C3090F480915E037D
:1067D0008F5F80935E0380915E03E82FFF27EE0FAB
:1067E000FF1FEE0FFF1FE955F74F8585181654F769
:1067F00080915E038C3070F0109259031092580310
:1068000010925E0385E08093600380915D03880FA2
:106810008D5A04C080915E03880F8E5A8093BB000E
:1068200085E87FC280915E03E82FFF2783E0EE0FAB
:10683000FF1F8A95E1F7E350F74F81818093BB00FA
:1068400085E88093BC0080915E03E82FFF27EE0F60
:10685000FF1FEE0FFF1FEE0FFF1FE350F74F80816A
:1068600080FF91C080915E03E82FFF27EE0FFF1F8E
:10687000EE0FFF1FEE0FFF1FE350F74F82818823BB
:1068800029F080912708873008F46CC28091580362
:1068900090915903892B09F065C28091560390911C
:1068A0005703892B09F05EC26EC080915E0321E020
:1068B00030E002C0220F331F8A95E2F78091560321
:1068C0009091570328233923232B79F080915E037D
:1068D000E82FFF27EE0FFF1FEE0FFF1FEE0FFF1F2A
:1068E000E350F74F80E184830DC080915E03E82F71
:1068F000FF27EE0FFF1FEE0FFF1FEE0FFF1FE350EE
:10690000F74F148280915E03E82FFF2753E0EE0FCC
:10691000FF1F5A95E1F7E350F74F8481282F332763
:1069200043E0220F331F4A95E1F780915E03E82F81
:10693000FF2793E0EE0FFF1F9A95E1F7E350F74F23
:1069400082818770822B8093BB0085E88093BC0096
:1069500020915E0381E090E002C0880F991F2A9584
:10696000E2F7209158033091590382239323892B16
:1069700051F085EF98E0909364038093630388E07F
:1069800080936503EFC184E089C1E0916303F091D6
:10699000640381918093BB0085E88093BC00F093F1
:1069A0006403E093630380916503815080936503E2
:1069B000882309F4D7C183E071C18091B900803385
:1069C00051F580916103882329F480915E038F5FE4
:1069D0008093610380915E03E82FFF2783E0EE0F31
:1069E000FF1F8A95E1F7E350F74F838199278F774F
:1069F00090708F3791057CF480915E03E82FFF271C
:106A0000EE0FFF1FEE0FFF1FEE0FFF1FE350F74FBC
:106A100083818F5F83831092600384E98093BC003D
:106A20008AE090E0909337018093360180915E0375
:106A30008F5F80935E03109260036DC18091B900F7
:106A40008034C9F180915D03E82FFF27EE0FFF1F0F
:106A5000EE0FFF1FEE0FFF1FE350F74F83818F777D
:106A6000838380915D038F5F80935D0380915D03DD
:106A70008C30A0F010925D031092570310925603D1
:106A8000809162038F5F809362038C3038F01092A4
:106A9000620380915A038D7F80935A0380915A0339
:106AA000816080935A031092600384E98093BC0054
:106AB00010925C0373C080915D03E82FFF27EE0FF7
:106AC000FF1FEE0FFF1FEE0FFF1FE350F74F8381F5
:106AD0008068838380915D03E82FFF27EE0FFF1FFF
:106AE000EE0FFF1FEE0FFF1FE350F74F808180FF77
:106AF0002FC080915D03E82FFF2753E0EE0FFF1FAB
:106B00005A95E1F7E350F74F84819927009751F0A8
:106B10004097D9F585EF98E09093640380936303E1
:106B200088E031C080915D03992743E0880F991F69
:106B30004A95E1F78E5F964F9093640380936303C9
:106B400090915D03809162039817E1F483E01BC08C
:106B500080915D03992733E0880F991F3A95E1F7FB
:106B60008E5F964F909364038093630380915A03E2
:106B700081FD06C090915D0380916203981711F426
:106B800082E001C081E080936503809165038130DC
:106B900011F485E801C085EC8093BC00809161030D
:106BA00080935B0310926103DDC0E0916303F09179
:106BB00064038091BB0080838091630390916403A0
:106BC00001969093640380936303809165038150E1
:106BD00080936503823010F085EC5DC0813011F444
:106BE00085E859C080915A0381FF2DC08091FF0331
:106BF00080FD1DC080915D03E82FFF2723E0EE0F8D
:106C0000FF1F2A95E1F7E350F74F86818A3F79F419
:106C100080915D03E82FFF2793E0EE0FFF1F9A9509
:106C2000E1F7E350F74F8081816080830CC0809151
:106C30005D03E82FFF2783E0EE0FFF1F8A95E1F742
:106C4000E350F74F108280915D038F5F80935D0367
:106C500080915D038C30A0F010925D031092570379
:106C600010925603809162038F5F809362038C3091
:106C700038F01092620380915A038D7F80935A03FB
:106C80001092600384E98093BC0080915A03816074
:106C900080935A0365C08093BC0086E080936003B4
:106CA00061C088E9BBCD80915F03880F805FB6CD5E
:106CB00080915F0399278130910561F082309105C1
:106CC0001CF4892B21F04EC0029739F04BC0809103
:106CD0001501A4CD80911401A1CD809113019ECD09
:106CE00080E89CCD1092600384E98093BC001092F0
:106CF0005C038AE090E090933701809336018091A5
:106D00005F03823088F480915F038F5F80935F031D
:106D100082E18093600380915A038E7F80935A03AF
:106D200085EA8093BC001EC010925F0380915A03D5
:106D3000816080935A0316C01092600384E98093A7
:106D4000BC0080915A03816080935A038AE090E0EE
:106D5000909337018093360110925E0310925D0389
:106D600010925C03FF91EF919F918F915F914F91F2
:106D70003F912F910F900FBE0F901F9018951F936A
:106D8000CF93DF93182F80913704882321F48091CB
:106D9000EF02882319F081E090E097C01D3008F0E1
:106DA00092C01123B1F0E12FFF2723E0EE0FFF1F68
:106DB0002A95E1F7E350F74F359780813596882380
:106DC0000CF081C03897808180FD03C083E090E0A3
:106DD0007CC08091F508823019F084E090E075C0A5
:106DE00067E070E085EF98E00E947B2E9091FC08B0
:106DF000891719F085E090E068C080ED97E00E9467
:106E0000BE19EC0180915A0380FD05C0CE010E949D
:106E1000C7198823B9F3112319F48FEF90E00BC041
:106E2000212F33272150304081E090E002C0880FAD
:106E3000991F2A95E2F79093590380935803A1E094
:106E4000B0E0EDEFF8E040E050E06BE0CD01042E63
:106E500002C0880F991F0A94E2F7209158033091DD
:106E6000590382239323892B11F0118212826150DE
:106E70004F5F5F4F389667FFE9CF10925E03109225
:106E8000600380915A038E7F80935A0385EA809332
:106E9000BC0080915A0380FD05C0CE010E94C71935
:106EA0008823B9F38091580390915903892B29F0D5
:106EB000CE010E94C719882311F380915803909145
:106EC0005903009711F082E090E0DF91CF911F917C
:106ED00008950F931F93CF93DF93982F80913704DA
:106EE000882321F48091EF02882319F081E090E05B
:106EF00092C09D30A0F4992319F486E090E08BC0F5
:106F0000C92FDD27FE0133E0EE0FFF1F3A95E1F7B1
:106F1000E350F74F35978081359687FD03C082E0B7
:106F200090E079C03897808180FD03C083E090E0D5
:106F300072C080ED97E00E94BE198C0180915A03C7
:106F400080FD05C0C8010E94C7198823B9F32197A5
:106F500021E030E0C90102C0880F991FCA95E2F70D
:106F60009093570380935603D901EDEFF8E040E08A
:106F700050E06BE0CD01042E02C0880F991F0A94E7
:106F8000E2F7209156033091570382239323892BF4
:106F900011F01182128261504F5F5F4F389667FF88
:106FA000E9CF10925D031092F5081092FC08109240
:106FB000600380915A038E7F80935A0385EA809301
:106FC000BC0080915A0380FD05C0C8010E94C7190A
:106FD0008823B9F38091560390915703892B29F0A8
:106FE000C8010E94C719882311F38091F5088230E7
:106FF00019F084E090E00FC067E070E085EF98E062
:107000000E947B2E9091FC08891719F085E090E092
:1070100002C080E090E0DF91CF911F910F91089521
:10702000CF93DF9380E021E83FEFC4EAD9E0EEE5BB
:10703000F9E0DF01853020F411961C921E9202C007
:10704000318320831982188222968F5F129632969E
:10705000833280F38FE790E090939D0980939C09A1
:1070600081E89FEF90939B0980939A0910929F0962
:1070700010929E091092A5041092A4041092A704E5
:107080001092A6041092A9041092A804DF91CF9147
:1070900008951F920F920FB60F9211240F931F9312
:1070A0002F933F934F935F936F937F938F939F9310
:1070B000AF93BF93CF93DF93EF93FF9380919808A3
:1070C00082FDC2C040918600509187008091670385
:1070D00090916803481B590B80918600909187001E
:1070E0009093680380936703CA018D549440A091E4
:1070F0006903B0916A03835F9A4158F480916903F0
:1071000080935D09149714F010923A0181E090E0A9
:1071100096C0A131B1050CF0F7C1CA018B5F904058
:10712000845B914008F086C08091380190913901CC
:10713000481B590BE0919108EE2351F0FF27EE0F09
:10714000FF1FE25AF64F8081918184369105ECF45D
:10715000FD01EA0FFB1FE25AF64F80819181FA018F
:10716000E81BF90BCF01F7FF03C0909581959F4F66
:1071700006975CF480913804883C20F480913804B0
:10718000865F01C088EC80933804FD01EA0FFB1F85
:10719000E25AF64F808191819C01220F331F280F04
:1071A000391F240F351F37FF02C02D5F3F4FE90104
:1071B000D595C795D595C795CA0101968C179D079A
:1071C00014F4219706C041505040C417D5070CF461
:1071D000219680913804833CE0F08D010A0F1B1F3B
:1071E000F801E25AF64F808191819E01281B390BEC
:1071F000C90163E070E00E94059ACB01880F991FD6
:10720000860F971F0C55164FD80111969C938E939D
:1072100007C0AA0FBB1FAC55B64F11961C921E9209
:10722000E0916903F0916A03EE0FFF1FE25AF64FF7
:10723000D183C0838091690390916A0301969093F2
:107240006A038093690360C1409186005091870072
:1072500080916B0390916C03481B590B80918600C1
:107260009091870090936C0380936B03CA018D54B7
:1072700094406091F503835F9A4108F07AC060936F
:10728000660380916603843008F453C090915D09D1
:1072900080916603981709F04CC05091F6035B305B
:1072A00008F43FC010923A011092F50340E05F31BC
:1072B000C0F0E42FFF27EE0FFF1F9F012F543C4F1C
:1072C000DF01A25AB64F8D919C91D9018D939C9369
:1072D000DF01AC55B64F8D919C91ED52FC4F9183DF
:1072E0008083E42FFF27EE0FFF1F9F01225A364FA6
:1072F000DF01A359BC4F8D919C91D90111969C93AC
:107300008E93DF01A157BC4F8D919C91EC55F64FA8
:1073100091838083842F8F5F482F813140F2809347
:10732000F5038091F6038F3FB9F08F5F8093F603EA
:1073300013C08091F603853620F08AE08093F6032F
:1073400002C01092F603809102018A3011F084315C
:1073500010F0289A01C0289881E08093F50380916D
:107360003704882309F0D0C08091660380935D09BB
:10737000CBC0613108F0A0C0CA018B5F9040845B34
:10738000914008F090C08091380190913901481BDC
:10739000590BE62FFF27EE0FFF1FE359FC4F8081AB
:1073A0009181FA01E81BF90BCF0105960B9720F5A7
:1073B000E0919108EE2351F0FF27EE0FFF1FE25AF4
:1073C000F64F8081918184369105B4F48091F60363
:1073D0008A3120F080913804865F05C08B3028F018
:1073E000809138048E5F8093380480913804893C02
:1073F00018F088EC80933804E62FFF27EE0FFF1F6C
:10740000E359FC4F808191819C01220F331F280F8B
:10741000391F240F351F37FF02C02D5F3F4FE90191
:10742000D595C795D595C795CA0101968C179D0727
:1074300014F4219706C041505040C417D5070CF4EE
:107440002196809138048E3BD8F0E62FFF27EE0F6F
:10745000FF1FDF01A359BC4F8D919C919E01281BFA
:10746000390BC90163E070E00E94059ACB01880FD7
:10747000991F860F971FE157FC4F9183808308C0A7
:10748000E62FFF27EE0FFF1FE157FC4F11821082FE
:107490008091F503E82FFF27EE0FFF1FE359FC4F04
:1074A000D183C08309C0809102018A3011F08431F8
:1074B00010F0289A01C028988091F503843120F4B7
:1074C0008F5F8093F50320C08431F1F48091020135
:1074D0008A3011F0843110F0289A01C028988EE18A
:1074E0008093F50320E1C4EAD9E0A1EBB3E0EEE537
:1074F000F9E08D919D919183808332961982188253
:107500002296215027FFF5CFFF91EF91DF91CF9188
:10751000BF91AF919F918F917F916F915F914F91AB
:107520003F912F911F910F910F900FBE0F901F90C1
:107530001895EF92FF920F931F938091440899271B
:10754000880F991F880F991F7C010027F7FC009571
:10755000102F8091920490919304A0919404B09183
:107560009504BC01CD01A80197010E943A9A30937D
:1075700084072093830780918A0490918B04A091C3
:107580008C04B0918D04BC01CD01A80197010E942B
:107590003A9A30938607209385078091400A90910C
:1075A000410A97FD039695958795959587959093B4
:1075B0008807809387078091500A9091510A97FD20
:1075C0000396959587959595879590938A078093CF
:1075D00089078091A4049091A504209130033091F3
:1075E0003103821B930B90938C0780938B078091C0
:1075F000320490913304A0913404B0913504BC015D
:10760000CD012AE030E040E050E00E943A9A309309
:107610008E0720938D078091C8079091C90790939A
:10762000900780938F0780918A0190918B019093AE
:10763000940780939307809120019091210190936A
:10764000960780939507809138049927909398071F
:10765000809397078091F8099091F90990939A0780
:10766000809399078091FE08992790939C078093B7
:107670009B0780910609992790939E0780939D0709
:1076800080910E0999279093A00780939F0780917E
:10769000160999279093A2078093A10780910A0366
:1076A00090910B039093AC078093AB0780911C04DF
:1076B00090911D049093AE078093AD078091DC0AF2
:1076C0009091DD0A9093B0078093AF078091E00A14
:1076D0009091E10A9093B2078093B10780912E04B4
:1076E00090912F04A0913004B0913104BC01CD01E0
:1076F0002AE030E040E050E00E943A9A3093B4072C
:107700002093B30780915004909151049093BA074D
:107710008093B9078091E20A99279093BE078093DE
:10772000BD0780910705909108059093C00780934D
:10773000BF0780910505909106059093C20780933D
:10774000C10780919D05882321F480919E0588239F
:1077500021F080918207816003C0809182078E7F33
:10776000809382071F910F91FF90EF900895EF9201
:10777000FF921F93CF93DF93182F7B0180913704E3
:10778000882391F5809102018C3010F0873111F43B
:10779000299801C0299A11501F3FE9F0F092120375
:1077A000E0921103E7018091110390911203892B5C
:1077B00011F4209781F3809115038823A1F310928F
:1077C00015038091110390911203892B09F42197DD
:1077D0000E942E97E8CF809102018C3010F0873103
:1077E00011F4299A01C02998DF91CF911F91FF9040
:1077F000EF900895CF93DF93809102018D3011F4C3
:107800000E94B11E10927A0080913403909135034A
:107810009093030A8093020A80913203909133037C
:107820009093F4098093F309809130039091310390
:107830009093460A8093450A20912C0330912D03A2
:10784000C901880F991F880F991F820F931F820FFC
:10785000931F9093410A8093400A20912E03309108
:107860002F03C901880F991F880F991F820F931F3B
:10787000820F931F9093510A8093500A8FEC80934C
:107880007A00A9E3B4E0CDE2D8E097E08991E82F4F
:10789000FF27EE0FFF1FE25AF64F0190F081E02D17
:1078A000E158FF4F1E161F061CF0E0E0F0E005C097
:1078B000EF3FF10514F0EFEFF0E08C91282F332724
:1078C000E217F30714F4815004C02E173F0714F495
:1078D0008F5F8C939150119697FFD8CF8091690854
:1078E0009927AA27BB27BC01CD0124EC39E040E051
:1078F00050E00E94C699DC01CB01809382019093F5
:107900008301A0938401B093850180916A0899272F
:10791000AA27BB27BC01CD010E94C699DC01CB017F
:1079200080937E0190937F01A0938001B0938101A9
:10793000DF91CF910895A0E0B0E0E1EAFCE30C9480
:10794000599A682EE1E07E2E00E010E068015801AF
:10795000E80110929D0510939F0400939E041093DC
:107960009D0400939C041093990400939804109232
:1079700097041093A9040093A8041093A7040093FC
:10798000A6041093A5040093A4041092640110921D
:107990006301109225030E94FA3B84E690E00E9466
:1079A000E0190E94FA3B8091350880FF10C0809159
:1079B000160190911701875B934038F4809116016E
:1079C000909117018E5E924010F40E942F1E7FE16D
:1079D000E72E8AE090E00E94E019809130039091B8
:1079E0003103080F191F8091340390913503C80E9D
:1079F000D91E8091320390913303A80EB91E809155
:107A0000C8079091C907C80FD91FEA94E7FEE1CFD4
:107A10009601205F3F4F36952795369527953093F1
:107A2000A9042093A804C50140969695879596953C
:107A300087959093A7048093A604005F1F4F45E0AD
:107A4000169507954A95E1F71093A5040093A404B1
:107A50006096B5E0D695C795BA95E1F7D0939904AD
:107A6000C09398049093A3048093A2043093A1043C
:107A70002093A00482E06816C9F58091400A909195
:107A8000410A97FF03C0909581959F4F6CE070E08D
:107A90000E94059A9B0170939F0460939E048091BD
:107AA000500A9091510A97FF03C0909581959F4F7E
:107AB0006CE070E00E94059A70939D0460939C04B2
:107AC000B90184E090E00E94933060919C04709131
:107AD0009D0486E090E00E9493306091980470913C
:107AE000990488E090E00E9493304FC084E090E0D9
:107AF0000E948E3090939F0480939E0486E090E0D5
:107B00000E948E309C0190939D0480939C048091F0
:107B10009E0490919F048150984018F42150384061
:107B2000A0F18CE499E09F938F9383EB95E19F9371
:107B30008F93E0918405F091850509958091400A25
:107B40009091410A97FF03C0909581959F4F6CE0FB
:107B500070E00E94059A70939F0460939E04809148
:107B6000500A9091510A97FF03C0909581959F4FBD
:107B70006CE070E00E94059A70939D0460939C04F1
:107B800077240F900F900F900F9012BC11BC1092A1
:107B9000030A1092020A1092F4091092F30910924B
:107BA000460A1092450A84E690E00E94E01980910E
:107BB0002C0390912D039C01220F331F220F331FA2
:107BC000280F391F280F391F3093410A2093400A8C
:107BD00080912E0390912F038C01000F111F000F35
:107BE000111F080F191F080F191F1093510A009336
:107BF000500A80914408C82EDD24EE24FF24442737
:107C000037FD4095542FC701B6010E94C6994B011C
:107C10005C01609392047093930480939404909316
:107C200095049801442737FD4095542FC701B601AC
:107C30000E94C699DC01CB0180938A0490938B0447
:107C4000A0938C04B0938D0480927204909273047C
:107C5000A0927404B092750480936A0490936B04AC
:107C6000A0936C04B0936D041092620410926304AC
:107C7000109264041092650480911801909119018A
:107C8000A0911A01B0911B018093CA079093CB0772
:107C9000A093CC07B093CD07109224031092230336
:107CA00010922603109227031092280310922903A2
:107CB00010925204109253041092540410925504DE
:107CC00000918A0110918B0110935104009350048C
:107CD00084E690E0909387018093860182E390E0B0
:107CE0009093120380931103809169089927AA2722
:107CF000BB27BC01CD0124EC39E040E050E00E94FC
:107D0000C699DC01CB018856954CAF4FBF4F80938D
:107D1000820190938301A0938401B09385018091A7
:107D20006A089927AA27BB27BC01CD010E94C699E2
:107D3000DC01CB018856954CAF4FBF4F80937E013D
:107D400090937F01A0938001B09381011092410133
:107D500010924001C801AA2797FDA095BA2F209143
:107D60003C0130913D0140913E0150913F01BC01E9
:107D7000CD010E94C699DC01CB0180934C0A9093FF
:107D80004D0AA0934E0AB0934F0A10924D041092E0
:107D90004C040E94AA748091FF0384608093FF03C7
:107DA0008FEF8093CC0A1092CD0A80E28093CE0AA6
:107DB000C9E3D4E0ADE2B8E0E7E0EE2E8D91E82F24
:107DC000FF27EE0FFF1FE25AF64F80819181815805
:107DD0008993EA94E7FEF2CF84E680933804809199
:107DE0000F03882311F0579A0DC080E091E1909322
:107DF00009018093080181E0809310010E94801A9C
:107E00000E94801A8091920490919304A09194040E
:107E1000B0919504E0903C01F0903D0100913E014D
:107E200010913F01BC01CD01A80197010E943A9A2F
:107E300059016A0180918A0490918B04A0918C046D
:107E4000B0918D04BC01CD01A80197010E943A9A1E
:107E5000B901C5010E944A8B8C010E94F4789C01F3
:107E600090930D0A80930C0A809198049091990444
:107E7000AA2797FDA095BA2F7DE0880F991FAA1F0A
:107E8000BB1F7A95D1F78050904FAF43B040442745
:107E900037FD4095542FBC01CD010E943A9AC9018B
:107EA00080509E4F9093990480939804053111055A
:107EB0000CF07724662079F08091F703882359F03D
:107EC000C90181599040C39730F080919D0580622F
:107ED00080939D0577248091A8049091A9048056F1
:107EE0009940815C9B4228F080919D058160809340
:107EF0009D058091A6049091A70480569940815CCD
:107F00009B4228F080919D05826080939D05809121
:107F1000A4049091A5048C5291408957954028F073
:107F200080919D05846080939D0580919E04909131
:107F30009F048C529140835C914028F080919D0574
:107F4000886080939D0580919C0490919D048C5243
:107F50009140835C914028F080919D0580618093E1
:107F60009D0580919804909199048050924083558A
:107F7000914028F080919D05806280939D058091BD
:107F80009D058111772486E4809379010E94D49223
:107F900082E00E943994872D9927EEE0CDB7DEB7B5
:107FA0000C94759AA3E1B0E0E8EDFFE30C94559AC8
:107FB0008091A4049091A504209130033091310365
:107FC000821B930B9093460A8093450A80913A0353
:107FD00090913B0397FD07969C0113E035952795FB
:107FE0001A95E1F73093030A2093020A809138032F
:107FF0009091390397FD0796B3E095958795BA95CB
:10800000E1F79093F4098093F30930930F0A2093DA
:108010000E0A9093060A8093050A8091400A909177
:10802000410AAC01440F551F480F591F20912C03E2
:1080300030912D03C901880F991F880F991F820F56
:10804000931F820F931F480F591F57FF02C04D5FA8
:108050005F4F55954795559547955093410A4093E5
:10806000400A8091500A9091510AAC01440F551F6B
:10807000480F591F20912E0330912F03C901880FFB
:10808000991F880F991F820F931F820F931F480F0C
:10809000591F57FF02C04D5F5F4F55954795559546
:1080A00047955093510A4093500A20912C033091E8
:1080B0002D03C901880F991F880F991F820F931FE5
:1080C000820F931F9C01442737FD4095542F8091C8
:1080D000820490918304A0918404B0918504820F5E
:1080E000931FA41FB51F8093820490938304A093D1
:1080F0008404B093850420912E0330912F03C9018D
:10810000880F991F880F991F820F931F820F931F4B
:108110009C01442737FD4095542F80917E04909117
:108120007F04A0918004B0918104820F931FA41F4B
:10813000B51F80937E0490937F04A0938004B09336
:1081400081048091180A9091190A20912C03309192
:108150002D03820F931F9093190A8093180A809120
:10816000480A9091490A20912E0330912F03820FE3
:10817000931F9093490A8093480A80919A049091A2
:108180009B04019690939B0480939A048091C80766
:108190009091C9072091980430919904821B930B08
:1081A0009C01442737FD4095542F80917A0490918B
:1081B0007B04A0917C04B0917D04820F931FA41FC7
:1081C000B51F80937A0490937B04A0937C04B093B2
:1081D0007D048FEC80937A001092120120916A0442
:1081E00030916B0440916C0450916D0429873A875B
:1081F0004B875C8729543B46414050402CF028E493
:108200003BE641E050E00DC089859A85AB85BC8591
:10821000885B9449AE4FBF4F4CF428EB34E94EEFE6
:108220005FEF2D833E834F83588708C089859A85E9
:10823000AB85BC858D839E83AF83B8872091720404
:108240003091730440917404509175042D873E87DA
:108250004F87588B29543B46414050402CF028E42E
:108260003BE641E050E00DC08D859E85AF85B88925
:10827000885B9449AE4FBF4F4CF428EB34E94EEF86
:108280005FEF29833A834B835C8308C08D859E858D
:10829000AF85B88989839A83AB83BC83A091450A53
:1082A000B091460ABB8BAA8BFD01CF01AA2797FD8F
:1082B000A095BA2FA0906204B0906304C0906404AB
:1082C000D0906504A80EB91ECA1EDB1EA0926204DF
:1082D000B0926304C0926404D0926504E0904C0AAA
:1082E000F0904D0A00914E0A10914F0AE80EF91EC7
:1082F0000A1F1B1FE0924C0AF0924D0A00934E0A8F
:1083000010934F0AF0911B04F98BFF2309F098C1D9
:1083100080911A04882309F093C180913C0A86FF5A
:108320008FC18091F3099091F409AA2797FDA09538
:10833000BA2FBC01CD0129813A814B815C810E9419
:10834000C6999B01AC0197FF04C02150384F4F4F95
:108350005F4FBBE05595479537952795BA95D1F76F
:1083600080916301682E772488249924CA01B90179
:10837000A40193010E94C699DC01CB018093B4044F
:108380009093B504A093B604B093B704B7FF04C0AC
:108390008150904FAF4FBF4F1C012D01ACE0559461
:1083A000479437942794AA95D1F72092B404309239
:1083B000B5044092B6045092B7048091020A90919D
:1083C000030AAA2797FDA095BA2FBC01CD012D81E4
:1083D0003E814F8158850E94C69997FF04C0615025
:1083E000784F8F4F9F4FFBE09595879577956795D1
:1083F000FA95D1F7A40193010E94C699DC01CB0143
:108400008093B8049093B904A093BA04B093BB04CA
:10841000B7FF04C08150904FAF4FBF4F9C01AD01DB
:10842000ECE05595479537952795EA95D1F7209338
:10843000B8043093B9044093BA045093BB048091BC
:10844000B4049091B5049093EB098093EA0980916C
:10845000B8049091B9049093EF098093EE09221922
:108460003309440955092093B8043093B904409363
:10847000BA045093BB04E20EF31E041F151FE092D2
:108480004C0AF0924D0A00934E0A10934F0A8091C5
:1084900062018823B1F457FF04C02F5F3F4F4F4F55
:1084A0005F4F5595479537952795A21AB30AC40A89
:1084B000D50AA0926204B0926304C0926404D09280
:1084C00065042A893B8979010027F7FC0095102F64
:1084D0008091B8049091B904A091BA04B091BB0402
:1084E000E80EF91E0A1F1B1FC801B70129813A8136
:1084F0004B815C810E94C6999B01AC0197FF04C02F
:108500002150384F4F4F5F4F6BE05595479537954A
:1085100027956A95D1F780916401A82EBB24CC24BD
:10852000DD24CA01B901A60195010E94C699DC01AA
:10853000CB018093AC049093AD04A093AE04B093B0
:10854000AF04B7FF04C08150904FAF4FBF4F3C0105
:108550004D013CE095948794779467943A95D1F7D0
:108560006092AC047092AD048092AE049092AF041D
:10857000C801B7012D813E814F8158850E94C6995F
:1085800097FF04C06150784F8F4F9F4F2BE0959518
:108590008795779567952A95D1F7A60195010E9451
:1085A000C699DC01CB018093B0049093B104A093F1
:1085B000B204B093B304B7FF04C08150904FAF4FE3
:1085C000BF4FAC01BD010CE0759567955795479578
:1085D0000A95D1F74093B0045093B1046093B2046C
:1085E0007093B3042A893B8937FF03C030952195E6
:1085F0003F4F21343105E4F1D401C30197FE07C098
:10860000B095A095909581959F4FAF4FBF4F813802
:108610009105A105B10584F4DB01CA0177FF07C00C
:10862000B095A095909581959F4FAF4FBF4F8138E2
:108630009105A105B105E4F081E080934E0418C0D6
:108640001092EF091092EE091092EB091092EA09CC
:108650001092B0041092B1041092B2041092B304BC
:108660001092AC041092AD041092AE041092AF04BC
:108670008091B0049091B104A091B204B091B30480
:10868000BC01CD0124E630E040E050E00E943A9A7F
:10869000E090AC04F090AD04E21AF30AF092010A03
:1086A000E092000A8091AC049091AD04A091AE04D8
:1086B000B091AF04BC01CD0124E630E040E050E0D1
:1086C0000E943A9ADA01C9012091B0043091B104B4
:1086D0008C01021B130B1093F6090093F50980918E
:1086E0003C0190913D01A0913E01B0913F01BC0140
:1086F000CD0128E631E040E050E00E94C69920918B
:108700004C0A30914D0A40914E0A50914F0A26175B
:1087100037074807590764F0261B370B480B590BDE
:1087200020934C0A30934D0A40934E0A50934F0ABF
:1087300020914C0A30914D0A40914E0A50914F0AB7
:1087400057FF0CC0260F371F481F591F20934C0A94
:1087500030934D0A40934E0A50934F0A6091F309AB
:108760007091F4096E0D7F1D9B01442737FD4095E4
:10877000542F8091660490916704A0916804B09191
:108780006904820F931FA41FB51F80936604909302
:108790006704A0936804B0936904809120049091C9
:1087A0002104681B790BCB01AA2797FDA095BA2F4E
:1087B00029853A854B855C85820F931FA41FB51FC1
:1087C00080936A0490936B04A0936C04B0936D043F
:1087D000C0907E01D0907F01E0908001F0908101F7
:1087E000C816D906EA06FB06C4F488EA91E6A0E0BA
:1087F000B0E08C199D09AE09BF0980936A0490937B
:108800006B04A0936C04B0936D0480936604909302
:108810006704A0936804B093690422273327A90151
:108820002C193D094E095F0980916A0490916B04EF
:10883000A0916C04B0916D0482179307A407B5074B
:10884000B4F4D701C601885A9146A040B040809345
:108850006A0490936B04A0936C04B0936D048093AE
:10886000660490936704A0936804B09369046091D0
:10887000020A7091030A600F711F9B01442737FDA4
:108880004095542F80916E0490916F04A0917004D4
:10889000B0917104820F931FA41FB51F80936E04C3
:1088A00090936F04A0937004B093710480911E04A0
:1088B00090911F04681B790BCB01AA2797FDA09507
:1088C000BA2F2D853E854F855889820F931FA41F8F
:1088D000B51F8093720490937304A0937404B093B3
:1088E0007504E0908201F090830100918401109161
:1088F0008501E816F9060A071B07C4F488EA91E621
:10890000A0E0B0E08E199F09A00BB10B8093720418
:1089100090937304A0937404B093750480936E04D1
:1089200090936F04A0937004B093710422273327AF
:10893000A9012E193F09400B510B809172049091AF
:108940007304A0917404B091750482179307A4076F
:10895000B507B4F4D801C701885A9146A040B04089
:108960008093720490937304A0937404B09375047D
:1089700080936E0490936F04A0937004B09371047D
:108980008091620490916304A0916404B0916504A5
:108990008093760490937704A0937804B09379043D
:1089A0008091720490917304A0917404B091750445
:1089B0008093920490939304A0939404B0939504AD
:1089C00080916A0490916B04A0916C04B0916D0445
:1089D00080938A0490938B04A0938C04B0938D04AD
:1089E00080916E0490916F04A0917004B091710415
:1089F00080938E0490938F04A0939004B09391047D
:108A00008091660490916704A0916804B091690414
:108A10008093860490938704A0938804B09389047C
:108A200080911E0190911F0197FD079613E0959587
:108A300087951A95E1F79093030A8093020A809133
:108A40001C0190911D0197FD0796B3E095958795C0
:108A5000BA95E1F79093F4098093F3098091340378
:108A6000909135030F9734F488E19CEF9093030ABB
:108A70008093020A8091340390913503079734F470
:108A800080E398EF9093030A8093020A20910201F9
:108A90002A30A9F48091340390913503835F934089
:108AA00034F088EE93E09093030A8093020A809159
:108AB0003403909135038A5F9340DCF014C08091B9
:108AC000340390913503815D974034F088EE93E054
:108AD0009093030A8093020A8091340390913503A6
:108AE000805E974034F080ED97E09093030A809386
:108AF000020A80913203909133030F9734F488E196
:108B00009CEF9093F4098093F30980913203909144
:108B10003303079734F480E398EF9093F40980933C
:108B2000F3092A30A9F48091320390913303835FD3
:108B3000934034F088EE93E09093F4098093F30926
:108B400080913203909133038A5F9340DCF014C02C
:108B50008091320390913303815D974034F088EE29
:108B600093E09093F4098093F309809132039091FC
:108B70003303805E974034F080ED97E09093F409E2
:108B80008093F30960917101662309F4AFC04091AD
:108B90001E0150911F018091BC049091BD04481B9F
:108BA000590B5093C3044093C20420911E0130918D
:108BB0001F01280F391F37FF02C02F5F3F4F359528
:108BC00027953093BD042093BC04413851051CF017
:108BD00080E890E005C040585F4F34F480E89FEF94
:108BE0009093C3048093C20440911C0150911D01D5
:108BF0008091BE049091BF04481B590B5093C1044F
:108C00004093C00420911C0130911D01280F391F91
:108C100037FF02C02F5F3F4F359527953093BF0434
:108C20002093BE04413851051CF080E890E005C057
:108C300040585F4F34F480E89FEF9093C1048093D5
:108C4000C004462F55278091C2049091C304849F8D
:108C5000B001859F700D949F700D11249B0177FFCB
:108C600002C0215F3F4FE4E035952795EA95E1F793
:108C70008091020A9091030A820F931F9093030A36
:108C80008093020A8091C0049091C104849FD00116
:108C9000859FB00D949FB00D1124AD019D01B7FFCC
:108CA00002C0215F3F4F94E0359527959A95E1F7F3
:108CB0008091F3099091F409820F931F9093F40926
:108CC0008093F30980911E0190911F01860F971FD9
:108CD00090931F0180931E0180911C0190911D01B2
:108CE000840F951F90931D0180931C010091050A2C
:108CF0001091060A8091EA099091EB09101611066D
:108D00005CF59C0197FF04C022273327281B390BF1
:108D1000C901AA2797FDA095BA2F20916201332798
:108D200044275527BC01CD010E94C6999B01AC0187
:108D300097FF04C0215C3F4F4F4F5F4F86E0559532
:108D40004795379527958A95D1F78091000A90919C
:108D5000010A820F931F27C097FF03C0909581954A
:108D60009F4FAA2797FDA095BA2F20916201332724
:108D700044275527BC01CD010E94C6999B01AC0137
:108D800097FF04C0215C3F4F4F4F5F4FB6E05595B2
:108D9000479537952795BA95D1F78091000A90911C
:108DA000010A821B930B9093010A8093000AE090C2
:108DB0000E0AF0900F0A8091EE099091EF091E14AF
:108DC0001F045CF59C0197FF04C022273327281B52
:108DD000390BC901AA2797FDA095BA2F20916201EE
:108DE000332744275527BC01CD010E94C6999B011A
:108DF000AC0197FF04C0215C3F4F4F4F5F4FA6E08F
:108E00005595479537952795AA95D1F78091F509FE
:108E10009091F609820F931F27C097FF03C090958A
:108E200081959F4FAA2797FDA095BA2F20916201A7
:108E3000332744275527BC01CD010E94C6999B01C9
:108E4000AC0197FF04C0215C3F4F4F4F5F4FF6E0EE
:108E50005595479537952795FA95D1F78091F5095E
:108E60009091F609821B930B9093F6098093F50974
:108E700080913C0A87FF44C0B989BB2309F040C0F8
:108E800080911A048823E1F5E1E0EE16E1E0FE06A8
:108E90004CF08091020A9091030A8E0D9F1D805024
:108EA00091400DC0F0E0EF16FFEFFF0664F48091F3
:108EB000020A9091030A8E0D9F1D80509F4F909340
:108EC000030A8093020A21E0013012074CF08091DE
:108ED000F3099091F409800F911F805091400CC0CC
:108EE0003FEF0030130764F48091F3099091F40987
:108EF000800F911F80509F4F9093F4098093F30946
:108F0000E2E1CD5E0C94719A80913704882329F5B3
:108F10008091FF038C7F8093FF038091FE038F7D00
:108F20008093FE03A2EAB5E0EDEFF8E09BE08091CC
:108F3000EF02882309F48C938D91818312829150E2
:108F4000389697FFF4CF8091EF02882359F08091F3
:108F5000EF0281508093EF0205C08091FF03816092
:108F60008093FF0380915C03882319F010925C03C7
:108F7000089580935E038093600380915A038E7FEF
:108F800080935A0385EA8093BC000895882319F4DE
:108F900080E090E00895E82FFF27EE0FFF1FE25AD0
:108FA000F64F8081918181589F4F8F3F910521F02D
:108FB0001CF08FEF90E004C097FF02C080E090E0CB
:108FC00099270895CF93DF93A9E3B4E0CDE2D8E0E9
:108FD00057E08991E82FFF27EE0FFF1FE25AF64F67
:108FE0000190F081E02DE158FF4FEF3FF10521F0B6
:108FF0001CF0EFEFF0E004C0F7FF02C0E0E0F0E0AB
:10900000893111F4EC931BC04C91242F3327E217C4
:10901000F307A9F0CF01821B930B97FD039695955B
:10902000879595958795242F280F2C93822F992724
:10903000E817F90714F4215001C02F5F2C93515009
:10904000119657FFC6CF80913708883F38F0EFEF71
:10905000F0E0E81BF109E75CFB4F8081809376012B
:1090600080917601882329F0843618F084E6809375
:10907000760180913908883F38F0EFEFF0E0E81B87
:10908000F109E75CFB4F8081809375018091750148
:10909000882329F0843618F084E680937501809146
:1090A0004608883F38F0EFEFF0E0E81BF109E75C95
:1090B000FB4F808180937001809170018B3010F4A0
:1090C0008AE002C08F3F11F4809370018091730891
:1090D000883F38F0EFEFF0E0E81BF109E75CFB4F69
:1090E000808180931A0A80911A0A863010F485E0F4
:1090F00002C08F3F11F480931A0A80917508883F4F
:1091000038F0EFEFF0E0E81BF109E75CFB4F8081FE
:109110008093430A8091430A863010F485E002C0B0
:109120008F3F11F48093430A80916008873F19F4C0
:10913000429905C006C0863F31F4439B02C08CE8CB
:1091400015C086E413C0883F38F0EFEFF0E0E81B6D
:10915000F109E75CFB4F80818093170A8091170A21
:10916000893110F488E102C08F3F11F48093170A0F
:1091700080916108873F19F4429905C006C0863F77
:1091800031F4439B02C08CE815C086E413C0883FCD
:1091900038F0EFEFF0E0E81BF109E75CFB4F80816E
:1091A0008093F0098091F009893110F488E102C0C0
:1091B0008F3F11F48093F00980916208883F38F066
:1091C000EFEFF0E0E81BF109E75CFB4F8081809353
:1091D000200A8091200A893110F488E102C08F3F73
:1091E00011F48093200A809138080E94C64780932A
:1091F000150480913B08883F38F0EFEFF0E0E81B62
:10920000F109E75CFB4F80818093740180913D08F8
:10921000883F38F0EFEFF0E0E81BF109E75CFB4F27
:1092200080818093720180914508883F38F0EFEF8C
:10923000F0E0E81BF109E75CFB4F8081809373014C
:1092400080914708883F38F0EFEFF0E0E81BF10924
:10925000E75CFB4F808180936F0180914808883FD5
:1092600038F0EFEFF0E0E81BF109E75CFB4F80819D
:109270008093710180914908883F38F0EFEFF0E06A
:10928000E81BF109E75CFB4F808180936E018091C0
:109290004A08883F38F0EFEFF0E0E81BF109E75C9F
:1092A000FB4F808180936D0180915008883F38F09A
:1092B000EFEFF0E0E81BF109E75CFB4F8081809362
:1092C0006B0180915108883F38F0EFEFF0E0E81B28
:1092D000F109E75CFB4F8081809314048091520870
:1092E000883F38F0EFEFF0E0E81BF109E75CFB4F57
:1092F00080818093130480915308883F38F0EFEF0A
:10930000F0E0E81BF109E75CFB4F808180931204D9
:1093100080915408883F38F0EFEFF0E0E81BF10946
:10932000E75CFB4F80818093110480916E08883F39
:1093300038F0EFEFF0E0E81BF109E75CFB4F8081CC
:109340008093100480916F08883F38F0EFEFF0E0D1
:10935000E81BF109E75CFB4F808180930F0480914B
:109360007008883F38F0EFEFF0E0E81BF109E75CA8
:10937000FB4F808180930E0480917108883F38F004
:10938000EFEFF0E0E81BF109E75CFB4F8081809391
:109390000D0480915508883F38F0EFEFF0E0E81BAE
:1093A000F109E75CFB4F8081809369018091590846
:1093B000883F38F0EFEFF0E0E81BF109E75CFB4F86
:1093C00080818093680180915608883F38F0EFEFE4
:1093D000F0E0E81BF109E75CFB4F808180936701B7
:1093E00080915A08883F38F0EFEFF0E0E81BF10970
:1093F000E75CFB4F80818093660180916308883F22
:1094000038F0EFEFF0E0E81BF109E75CFB4F8081FB
:109410008093650180916608883F38F0EFEFF0E0B7
:10942000E81BF109E75CFB4F808180936401809128
:109430006708883F38F0EFEFF0E0E81BF109E75CE0
:10944000FB4F80818093630180916808883F38F0EA
:10945000EFEFF0E0E81BF109E75CFB4F80818093C0
:10946000620180919008883F38F0EFEFF0E0E81B50
:10947000F109E75CFB4F80818093FF099091110512
:10948000992321F08091FF09981720F08091FF091E
:10949000882311F49093FF098091350880933C0A4A
:1094A0008091980880931F0A80916D08883F38F05A
:1094B000EFEFF0E0E81BF109E75CFB4F8081809360
:1094C000610180918908883F38F0EFEFF0E0E81BF8
:1094D000F109E75CFB4F80818093530A80916B0117
:1094E000282F33272F5F3F4F8CE398E2B9010E946A
:1094F000059A709378016093770180914308809377
:10950000440A809142088093070AE0918B08EE2379
:1095100009F449C081E080930C04FF27EE0FFF1F80
:10952000E25AF64F80819181805C9F4F14F4109233
:109530000C048091790120910C04821721F1833071
:10954000F8F43091A401222351F08CED95E0909332
:10955000120380931103332369F48EE209C088EC6F
:1095600090E09093120380931103332319F487E161
:109570008093A40185E0809322042093790103C0A5
:109580008150809379018091930A9091940A97FF7A
:109590000FC080910C04882359F080919D0580684C
:1095A00080939D0505C0E0930C048AE080937901C7
:1095B0008091930A9091940A97FF1DC0809137047F
:1095C0008823C9F080910C048823A9F080910A01B6
:1095D00090910B018F5F9F4F71F488E99AE390930C
:1095E00012038093110380E094EA90930B0180931F
:1095F0000A0110920C0480910C04882321F08091C0
:10960000FE03816003C08091FE038E7F8093FE0382
:10961000DF91CF910895A7E1B0E0E1E1FBE40C9484
:10962000559A0E94D23F8091FF03992784719070D0
:10963000892B91F58091990882FF27C080911C04A5
:1096400090911D040097F1F002E088359007D4F462
:109650009C0197FF02C02D5F3F4F359527953595AB
:10966000279580914D089927289FA001299F500D8B
:10967000389F500D1124CA0164E670E00E94059ADB
:10968000CB0106C08DE290E003C080914D08992780
:109690009093FD038093FC032091FA033091FB0328
:1096A00055E72033350759F41092430410924204D1
:1096B0008091070A99279093FD038093FC036091A2
:1096C0004204709143047A8369838091070A992741
:1096D0000A966817790714F49A838983809138046D
:1096E000843608F06AC08091FE0382FD66C08091D6
:1096F000D8049091D904009731F001979093D90440
:109700008093D8040BC01092370490930104809387
:1097100000048091FF038D7E8093FF0380910201FE
:109720008A3011F0843110F0289A01C02898809175
:10973000000490910104895E9340E0F18091E20A77
:109740008536C0F18091FC039091FD039A83898353
:109750008091FF0380618093FF0380912908A82FE7
:10976000BB27AA0FBB1FFD01EC55F64F11821082DB
:1097700080912A08282F3327220F331FC9018C55C7
:10978000964FFC0111821082A25AB64F11961C927C
:109790001E92225A364FD90111961C921E92809128
:1097A0002C08E82FFF27EE0FFF1FE25AF64F118219
:1097B000108277C51092370474C5809138048D38B3
:1097C00008F445C590919408992309F445C0809107
:1097D0009508882309F440C0E92FFF27EE0FFF1FEB
:1097E000E25AF64F80819181C397BCF080918E013F
:1097F000823361F48091FE0385FF08C08091FE03EF
:1098000080648093FE0380E38093A4018091FE0333
:109810008F778093FE0386E917C0808191818E5CEB
:109820009F4FACF480918E01863941F48091FE0304
:1098300080688093FE038FE28093A4018091FE03F1
:109840008F7B8093FE0382E380938E0105C080911D
:10985000FE038F738093FE038091FF038F7E8093BE
:10986000FF0390914E0882E3989FC00111249093CA
:10987000D9048093D804E981FA81B9978CF080915A
:109880003704882369F08091000490910104FFEF70
:109890008F3F9F0729F00196909301048093000465
:1098A00040910004509101044F3F510509F048F5E3
:1098B00010925A0410925B0410925C0410925D04A2
:1098C00010925604109257041092580410925904A2
:1098D0001092C4041092C5041092C6041092C704DA
:1098E0001092620410926304109264041092650452
:1098F0008091FE0380628093FE0384E680938E0154
:1099000035C18091FF0382608093FF038091FE0345
:1099100085FF98C08091120599279C0124703070B2
:1099200082FD04C08091FE0386FF2AC080913B0126
:109930008D3331F58091F703882311F180E5809311
:10994000270484EF91E0A0E0B0E080932804909396
:109950002904A0932A04B0932B0480932E0490939F
:109960002F04A0933004B093310488EE93E09093D9
:109970008D0180938C01232B19F08DE08093A4013D
:1099800080911D0390911E03A0911F03B0912003AD
:1099900087399105A105B1058CF48091320490912D
:1099A0003304A0913404B0913504825A9E4FAF4FD6
:1099B000BF4F24F080913C0A80FD21C088EE93E0E7
:1099C00090938D0180938C018091FE0386FF0FC0E0
:1099D000109227048CE291E0A0E0B0E080932E0486
:1099E00090932F04A0933004B093310403C080E31C
:1099F0008093A4018091FE038F718093FE031092E7
:109A00005A0410925B0410925C0410925D04109250
:109A10005604109257041092580410925904109250
:109A20006204109263041092640410926504495E0B
:109A3000534008F49BC088EE93E090930104809318
:109A4000000494C08091FE0387FF1AC080913B01FF
:109A5000863711F08D33A1F48091F703882381F0CC
:109A6000809195088093270480EE91EBAFEFBFEFD4
:109A70008093280490932904A0932A04B0932B0484
:109A800020918C0130918D0143E0283E340708F08D
:109A900048C02F5F3F4F30938D0120938C0110926F
:109AA0005A0410925B0410925C0410925D041092B0
:109AB00056041092570410925804109259041092B0
:109AC0006204109263041092640410926504809101
:109AD0001D0390911E03A0911F03B09120038C528F
:109AE0009140A040B04080932E0490932F04A09307
:109AF0003004B0933104285E3340C1F58091FE03F9
:109B000087FF34C080913B018B3281F18091FE034D
:109B10008F778093FE038091FE0380628093FE0323
:109B200025C08091F703882309F180913B01863796
:109B300011F08D32D9F48091320490913304A091C8
:109B40003404B0913504885E9340A040B04074F472
:109B50008091C8079091C9078D5A93403CF01092AC
:109B60008D0110928C018EE08093A40180912B08CE
:109B7000E82FFF27EE0FFF1FE25AF64F80819181F9
:109B8000813591050CF454C120913704222309F04A
:109B90004FC180912C08E82FFF27EE0FFF1FE25ADC
:109BA000F64F808191818C3491050CF411C1809124
:109BB000DA048F5F8093DA04893C08F439C120937A
:109BC000DA04109201041092000430912908E32F66
:109BD000FF27EE0FFF1FE25AF64F808191818734F5
:109BE0009105B4F480912A08E82FFF27EE0FFF1F9C
:109BF000E25AF64F808191810190F081E02DF7FFCC
:109C000003C0F095E195FF4FE734F1050CF478C0FF
:109C100041E020912A08A22FBB27AA0FBB1FA25AFE
:109C2000B64F8D919C9111978734910544F0E32FA5
:109C3000FF27EE0FFF1FE25AF64F808191818D9131
:109C40009C918734910574F080912908E82FFF27B3
:109C5000EE0FFF1FE25AF64F808191818734910504
:109C60000CF042E0E22FFF27EE0FFF1FE25AF64F03
:109C7000808191818634910574F480912908E82FC0
:109C8000FF27EE0FFF1FE25AF64F80819181873444
:109C900091050CF043E0E22FFF27EE0FFF1FE25A81
:109CA000F64F808191818A5B9F4F74F480912908DF
:109CB000E82FFF27EE0FFF1FE25AF64F80819181B8
:109CC000873491050CF044E0E22FFF27EE0FFF1FD1
:109CD000E25AF64F808191818A5B9F4F74F48091A4
:109CE0002908E82FFF27EE0FFF1FE25AF64F808169
:109CF0009181863491050CF445E0842F0E94ED306B
:109D000080912A08E82FFF27EE0FFF1FE25AF64F37
:109D1000808191810190F081E02DF7FF03C0F095E3
:109D2000E195FF4F7E97CCF480912908E82FFF271B
:109D3000EE0FFF1FE25AF64F808191818A5B9F4FA1
:109D400064F481E08093B8051092230488EE93E0D8
:109D500090931203809311036BC0809100010E94C5
:109D6000983080E00E94AA0980914F080E94AD952A
:109D700080913C0A80FF10C08091160190911701DC
:109D8000875B934038F480911601909117018E5EA5
:109D9000924010F40E942F1E81E00E949B3C982F5D
:109DA0008093230421E020930F03579A80919D050F
:109DB000882311F087E006C0992319F42093A401A9
:109DC00003C088E18093A40185E080933E0527C00D
:109DD00080819181855B9F4F4CF58091DA048F5F84
:109DE0008093DA04893C20F1209337042093DA042D
:109DF000109201041092000482E00E949B3C982F74
:109E00008093230480919D05882311F087E005C08D
:109E1000992311F481E001C088E18093A40168E7EF
:109E200070E0809100010E94B73B02C02093DA04E9
:109E300080912B08E82FFF27EE0FFF1FE25AF64F05
:109E4000808191818C599F4F0CF0FAC120918C0830
:109E5000E22FFF27EF77F070EE0FFF1FEC55F64F64
:109E600080819181069714F084E606C080819181FB
:109E70008B5F9F4F1CF48CE98093DD048091370445
:109E8000E0912C08882309F03EC1FF27EE0FFF1F49
:109E9000E25AF64F808191818C599F4F9CF48091BA
:109EA000990883FD0BC0E22FFF27EE0FFF1FE25A38
:109EB000F64F80819181855B9F4FDCF080918C080B
:109EC0008823B9F08091990883FF1AC180918C088A
:109ED000E82FFF27EE0FFF1FE25AF64F8081918196
:109EE000875F9F4F0CF40CC18091DD04843609F02C
:109EF00007C120912304222329F08091FF03886069
:109F00008093FF038091180190911901A0911A018B
:109F1000B0911B018093CA079093CB07A093CC0705
:109F2000B093CD0710921D0310921E0310921F03D1
:109F300010922003109232041092330410923404D1
:109F400010923504109226031092270310922803D2
:109F50001092290380912908E82FFF27EE0FFF1F99
:109F6000E25AF64F808191818D599F4FACF48091D8
:109F70002A08E82FFF27EE0FFF1FE25AF64F8081D5
:109F800091810190F081E02DF7FF03C0F095E195FC
:109F9000FF4FE436F10534F480918C08882311F4E6
:109FA0008093DB048091DB048F5F8093DB048E3F22
:109FB00008F438C11092DB0480919D05882309F0D4
:109FC00092C0222309F48FC080911605882309F0DE
:109FD0008AC081E090E0909301048093000481E0C6
:109FE000809337041092C4041092C5041092C604E2
:109FF0001092C704109262041092630410926404D9
:10A000001092650410925E0410925F041092600436
:10A010001092610480914408E82EFF240027112744
:10A020008091400A9091410A9C01442737FD409558
:10A03000542FC801B7010E94C699DC01CB0180935F
:10A04000720490937304A0937404B0937504809188
:10A05000500A9091510A9C01442737FD4095542F96
:10A06000C801B7010E94C699DC01CB0180936A0444
:10A0700090936B04A0936C04B0936D048091920450
:10A0800090919304A0919404B091950480936E04F0
:10A0900090936F04A0937004B093710480918A042C
:10A0A00090918B04A0918C04B0918D0480936604F0
:10A0B00090936704A0936804B093690410925A04C3
:10A0C00010925B0410925C0410925D04109256048E
:10A0D00010925704109258041092590484E6809309
:10A0E000220484E39AC08CED95E090931203809350
:10A0F000110380912304882309F094C081E08DC06E
:10A100001092DB048FC0FF27EE0FFF1FE25AF64FBD
:10A1100080819181853691059CF08091990883FD1D
:10A120000BC0E22FFF27EE0FFF1FE25AF64F808190
:10A130009181855B9F4FDCF080918C088823B9F07A
:10A140008091990883FF6CC080918C08E82FFF27CD
:10A15000EE0FFF1FE25AF64F808191818E5C9F4F78
:10A160000CF05EC08091DD048C3909F059C08091FB
:10A170002908E82FFF27EE0FFF1FE25AF64F8081D4
:10A1800091818D599F4FACF480912A08E82FFF27C9
:10A19000EE0FFF1FE25AF64F808191810190F0810E
:10A1A000E02DF7FF03C0F095E195FF4FE436F10590
:10A1B0003CF480918C08882319F48093DC0418C047
:10A1C00010925A0410925B0410925C0410925D0489
:10A1D0001092560410925704109258041092590489
:10A1E00010924904109248041092470410924604B9
:10A1F0008091DC048F5F8093DC048B3F98F0109299
:10A2000037041092DC041092010410920004809133
:10A21000FE038F718093FE0386E28093A40102C047
:10A220001092DC048091FA039091FB03F3E0883EE6
:10A230009F07B8F501969093FB038093FA0331C012
:10A240001092DD041092FB031092FA032AC02E5ED6
:10A25000324038F180915B0A90915C0A80599140BC
:10A2600000F58091320490913304A0913404B091B0
:10A2700035048C5D9540A040B0409CF480E395E7A8
:10A280009093FB038093FA03809100049091010462
:10A290008A5E934030F089EE93E0909301048093BE
:10A2A000000480913A01815080933A0180913A01F3
:10A2B0008F3F21F08091FF0384FFA9C30E94E247F2
:10A2C000B0903F088091E6049091E7049C01220F32
:10A2D000331F280F391FC0902908AC2DBB27AA0FA8
:10A2E000BB1FFD01E25AF64F4B2D5527808191810E
:10A2F000849FB001859F700D949F700D1124260FCF
:10A30000371F37FF02C02D5F3F4FB9017595679525
:10A3100075956795AC55B64F80914008082F112769
:10A320008D919C91809FD001819FB00D909FB00D29
:10A3300011246A0F7B1F7093E7046093E6048091F9
:10A34000E8049091E9049C01220F331F280F391F64
:10A35000D0902A08AD2DBB27AA0FBB1FFD01E25AE2
:10A36000F64F80819181849FF001859FF00D949F2D
:10A37000F00D11242E0F3F1F37FF02C02D5F3F4FFE
:10A38000A9015595479555954795AC55B64F8D9173
:10A390009C91809F7001819FF00C909FF00C112484
:10A3A0004E0D5F1D5093E9044093E80480910C0426
:10A3B000882309F448C0CB0177FD0396DC01B595ED
:10A3C000A795B595A795CA0157FD0396FC01F5958C
:10A3D000E795F595E79580919F01682F772767FDB1
:10A3E00070956A9F90016B9F300D7A9F300D1124FC
:10A3F00080911805482F552747FD50954E9FC00165
:10A400004F9F900D5E9F900D1124280F391F37FF2D
:10A4100002C0295F3F4F93E0359527959A95E1F764
:10A4200030934904209348046E9F90016F9F300D34
:10A430007E9F300D11244A9FC0014B9F900D5A9F63
:10A44000900D11243FC080918A08E82FFF27EE5B12
:10A45000FE4F868180939F01908190931805A82FCD
:10A46000BB27A7FDB095A69F9001A79F300DB69F73
:10A47000300D1124E92FFF27E7FDF095E49FC0017F
:10A48000E59F900DF49F900D1124280F391F37FF81
:10A4900002C0295F3F4F83E0359527958A95E1F704
:10A4A0003093490420934804A49F9001A59F300D48
:10A4B000B49F300D1124E69FC001E79F900DF69FD9
:10A4C000900D1124281B390B37FF02C0295F3F4F25
:10A4D00003E0359527950A95E1F7309347042093DB
:10A4E000460480912C08E82FFF27EE0FFF1FE25A49
:10A4F000F64F80819181909581959F4F909345046F
:10A50000809344048530910514F0049705C00FEF43
:10A510008C3F900734F40496909345048093440450
:10A5200004C01092450410924404809104058823CD
:10A5300009F43EC0282F33278091480490914904A4
:10A5400097FD079613E0959587951A95E1F7289F53
:10A55000A001299F500D389F500D1124CA0157FDAD
:10A560000F96B4E095958795BA95E1F790934904D5
:10A5700080934804809146049091470497FD079684
:10A58000A3E095958795AA95E1F7289FB001299FAB
:10A59000700D389F700D1124CB0177FD0F96F4E0FC
:10A5A00095958795FA95E1F7909347048093460433
:10A5B0008090480490904904809107059091080587
:10A5C000881A990A9092490480924804009146049E
:10A5D000109147048091050590910605081B190B01
:10A5E000109347040093460480912B08E82FFF271F
:10A5F000EE0FFF1FE25AF64FE080F1808FE790E008
:10A60000E80EF91EF0924304E0924204809170013A
:10A610009927AA2797FDA095BA2FBC01CD010E94CA
:10A620003A99DC01CB0120E030E040E251E4BC018A
:10A63000CD010E94A898DC01CB01BC01CD010E9494
:10A640000C99DC01CB0180934A0A80916F018093C1
:10A65000210A80916E019927AA2797FDA095BA2F0C
:10A66000BC01CD010E943A99DC01CB0120E030E031
:10A6700040E251E4BC01CD010E94A898DC01CB016D
:10A68000BC01CD010E940C99DC01CB018093FA0939
:10A6900080916D018093100A8091C40580FF59C09C
:10A6A0008091530A813808F454C08091BD059927E0
:10A6B00087FD90952B2D3327829FD001839FB00D6E
:10A6C000929FB00D11248A0E9B1E90924904809295
:10A6D00048048091BE05992787FD9095829FF001DF
:10A6E000839FF00D929FF00D11240E0F1F1F1093EA
:10A6F0004704009346048091BF05282F332727FD88
:10A7000030958091440490914504820F931F90935B
:10A710004504809344048091C105282F332727FDE9
:10A72000309580913A089927289F8001299F100D24
:10A73000389F100D11241093410100934001809126
:10A74000C00599278E159F0524F4909343048093A8
:10A750004204809142049091430497FF04C01092F8
:10A7600043041092420480913C0A82FF02C010927E
:10A77000210A4091480450914904CA0157FD0396AB
:10A780009C01359527953595279537FF03C0309562
:10A7900021953F4F809104049091050482179307FF
:10A7A000B4F4CA0157FF03C0909581959F4F97FD60
:10A7B0000396959587959595879590930504809335
:10A7C00004048536910544F084E690E001C00197C9
:10A7D00090930504809304044091460450914704EB
:10A7E000CA0157FD03969C01359527953595279508
:10A7F00037FF03C0309521953F4F8091020490911F
:10A80000030482179307B4F4CA0157FF03C090955D
:10A8100081959F4F97FD039695958795959587957B
:10A8200090930304809302048536910544F084E6F6
:10A8300090E001C0019790930304809302048091FB
:10A84000FF0384FF08C010920504109204041092C4
:10A85000030410920204ED2DFF27EE0FFF1FE25AB2
:10A86000F64F40916408242F332780819181281767
:10A87000390744F48091960882FF04C081E08093F8
:10A88000190413C0ED2DFF27EE0FFF1FE25AF64FFC
:10A89000842F992720916508821B9109208131819D
:10A8A0002817390714F41092190440912A08E42F4C
:10A8B000FF27EE0FFF1FE25AF64F50916408852FD5
:10A8C000992722273327281B390B808191818217F2
:10A8D000930744F48091960883FF04C081E080933D
:10A8E000180416C080911804882391F0E42FFF27E4
:10A8F000EE0FFF1FE25AF64F809165089927851BDE
:10A900009109208131818217930714F41092180461
:10A91000EC2DFF27EE0FFF1FE25AF64F409164081F
:10A92000242F3327808191812817390744F480919F
:10A93000960880FF04C081E08093160417C08091C0
:10A940001604882399F0EC2DFF27EE0FFF1FE25A23
:10A95000F64F842F992720916508821B9109208149
:10A9600031812817390714F41092160440912908F0
:10A97000E42FFF27EE0FFF1FE25AF64F50916408B5
:10A98000852F992722273327281B390B8081918116
:10A990008217930744F48091960881FF04C081E0F8
:10A9A0008093170416C080911704882391F0E42F38
:10A9B000FF27EE0FFF1FE25AF64F80916508992797
:10A9C000851B9109208131818217930714F410921D
:10A9D000170480911904882319F4809118048111B7
:10A9E00081E080931A0480911604882321F48091D9
:10A9F0001704882351F081E080931B0410921A04FD
:10AA0000109219041092180402C080931B048091C4
:10AA10001A04882321F480911B04882369F0809113
:10AA20006308992729813A818217930714F49A833E
:10AA3000898381E080934E048091FE0399279C01D5
:10AA40002470307082FF2DC0809107059091080519
:10AA5000909581959F4F90934904809348048091ED
:10AA6000050590910605909581959F4F9093470419
:10AA70008093460480917C0190917D0190934304E2
:10AA80008093420480913C0A8B778B6680933C0ACA
:10AA900080911F0A8C7B80931F0A88EC8093150499
:10AAA0001EC08091FF0384FF1AC030934504209399
:10AAB000440430934904209348043093470420937E
:10AAC00046049AE590934A0A88E78093210A909376
:10AAD000FA098093100A10921A0410921B048091B4
:10AAE000130A9091140AA091150AB091160A2091A8
:10AAF0009204309193044091940450919504820FF4
:10AB0000931FA41FB51F8093130A9093140AA09358
:10AB1000150AB093160A80911B0A90911C0AA09105
:10AB20001D0AB0911E0AE0908A04F0908B040091F7
:10AB30008C0410918D04EB82FC820D831E838E0D9C
:10AB40009F1DA01FB11F80931B0A90931C0AA09306
:10AB50001D0AB0931E0A8091080A9091090AA091DB
:10AB60000A0AB0910B0AE0908E04F0908F040091D5
:10AB7000900410919104EF82F88609871A878E0D50
:10AB80009F1DA01FB11F8093080A9093090AA093EC
:10AB90000A0AB0930B0A8091FB099091FC09A091DD
:10ABA000FD09B091FE09E0908604F09087040091C1
:10ABB000880410918904EB86FC860D871E878E0D14
:10ABC0009F1DA01FB11F8093FB099093FC09A093C8
:10ABD000FD09B093FE09F0901B04FF86FF2029F4C5
:10ABE00080911A04882309F460C0109282041092A4
:10ABF0008304109284041092850410927E041092B3
:10AC00007F0410928004109281041092130A109213
:10AC1000140A1092150A1092160A10921B0A10922A
:10AC20001C0A10921D0A10921E0A1092080A109215
:10AC3000090A10920A0A10920B0A1092FB0910924C
:10AC4000FC091092FD091092FE0980917204909106
:10AC50007304A0917404B091750480936E04909372
:10AC60006F04A0937004B093710480916A04909172
:10AC70006B04A0916C04B0916D0480936604909372
:10AC80006704A0936804B0936904109222031092A1
:10AC9000210310921F0410921E041092210410929E
:10ACA00020040F85002309F0D0C180911A04882365
:10ACB00009F0CBC18091C8079091C907815092409B
:10ACC0002CF480913704882309F4BFC19090CC0AFA
:10ACD000A09044082090400A3090410A4090500AC9
:10ACE0005090510A19140CF0BBC0BB24CC24DD24B5
:10ACF000CA01B901A60195010E943A9A79018A0117
:10AD00008091950A9091960A281A390AC101AA27BA
:10AD100097FDA095BA2FE81AF90A0A0B1B0B6B8155
:10AD20007C818D819E81A60195010E943A9A5901EC
:10AD30006A018091970A9091980A481A590AC201AB
:10AD4000AA2797FDA095BA2FA81AB90ACA0ADB0A42
:10AD5000292C332427FC3094432C532CC801B701F1
:10AD6000A20191010E94C69997FF04C061507E4FD5
:10AD70008F4F9F4F3B014C0109E095948794779446
:10AD800067940A95D1F7C601B501A20191010E940D
:10AD9000C69997FF04C061507E4F8F4F9F4F5B0154
:10ADA0006C0119E0D594C794B794A7941A95D1F77C
:10ADB0008091040490910504813491053CF48091C4
:10ADC00002049091030481349105D4F0D401C301AD
:10ADD00097FE03C00196A11DB11D3C014D01959444
:10ADE000879477946794D601C501D7FE03C0019676
:10ADF000A11DB11D5C016D01D594C794B794A794B2
:10AE00008091CE0A282F332727FD3095432F532FCB
:10AE1000261537054805590514F439014A019927C3
:10AE200087FD9095909581959F4FAA2797FDA095B6
:10AE3000BA2F681679068A069B0614F43C014D0168
:10AE40002A153B054C055D0514F459016A01A81645
:10AE5000B906CA06DB060CF0D0C05C016D01CDC09E
:10AE6000EA2CFF2400271127CA01B901A801970184
:10AE70000E943A9A39014A01C101AA2797FDA0957B
:10AE8000BA2F681A790A8A0A9B0A6B817C818D81A4
:10AE90009E81A80197010E943A9A59016A01C20154
:10AEA000AA2797FDA095BA2FA81AB90ACA0ADB0AE1
:10AEB000D401C30197FE03C00F96A11DB11D3C0133
:10AEC0004D01F4E09594879477946794FA95D1F7BF
:10AED000D601C501D7FE03C00F96A11DB11D5C01AF
:10AEE0006D01E4E0D594C794B794A794EA95D1F79F
:10AEF0008091040490910504813491053CF4809183
:10AF000002049091030481349105A4F0C401B301BB
:10AF100023E030E040E050E00E943A9A39014A01D3
:10AF2000C601B50123E030E040E050E00E943A9ACB
:10AF300059016A0180912C08E82FFF27EE0FFF1FAF
:10AF4000E25AF64F808191810190F081E02DF7FF68
:10AF500003C0F095E195FF4F7A97A4F0C401B301C7
:10AF600023E030E040E050E00E943A9A39014A0183
:10AF7000C601B50123E030E040E050E00E943A9A7B
:10AF800059016A0189E18093880121E26216710406
:10AF9000810491042CF070E2672E712C812C912C8D
:10AFA00030EE63163FEF73063FEF83063FEF9306E5
:10AFB00044F460EE662E6FEF762E6FEF862E6FEF05
:10AFC000962E41E2A416B104C104D1042CF050E243
:10AFD000A52EB12CC12CD12C50EEA5165FEFB506D5
:10AFE0005FEFC5065FEFD50644F440EEA42E4FEFA9
:10AFF000B42E4FEFC42E4FEFD42E80917204909157
:10B000007304A0917404B091750486199709A80976
:10B01000B9098093720490937304A0937404B0935D
:10B02000750480916A0490916B04A0916C04B091B6
:10B030006D048A199B09AC09BD0980936A04909339
:10B040006B04A0936C04B0936D04809121039091E4
:10B0500022038F3F910509F008F4C4C56F8566236C
:10B0600009F04EC580911A04882309F049C58091E2
:10B070004E04882309F044C570916C08788B7723BF
:10B0800009F43EC58091130A9091140AA091150A03
:10B09000B091160AB7FF04C081509F4FAF4FBF4F0A
:10B0A000E92EFA2E0B2F112707FD1A95E092130AAD
:10B0B000F092140A0093150A1093160A80911B0A45
:10B0C00090911C0AA0911D0AB0911E0AB7FF04C0FE
:10B0D00081509F4FAF4FBF4F892F9A2FAB2FBB2768
:10B0E000A7FDBA95898B9A8BAB8BBC8B80931B0A7F
:10B0F00090931C0AA0931D0AB0931E0A80914408E5
:10B10000A82EBB24CC24DD2420918204309183041A
:10B110004091840450918504C601B5010E94C699EE
:10B1200097FF04C061507F4F8F4F9F4F672E782E3F
:10B13000892E992487FC9A946092820470928304E9
:10B14000809284049092850420917E0430917F0443
:10B150004091800450918104C601B5010E94C699B6
:10B1600097FF04C061507F4F8F4F9F4F272E382E7F
:10B17000492E552447FC5A9420927E0430927F0435
:10B18000409280045092810480917A0490917B04D3
:10B19000A0917C04B0917D04B7FF04C081509F4F03
:10B1A000AF4FBF4F892F9A2FAB2FBB27A7FDBA9563
:10B1B00080937A0490937B04A0937C04B0937D04E5
:10B1C000D801C70186199709A809B9098093D00445
:10B1D0009093D104A093D204B093D30420916B0830
:10B1E000E22EFF2400271127BC01CD01A801970101
:10B1F0000E943A9A59016A012093DE043093DF04D9
:10B200004093E0045093E10489899A89AB89BC8911
:10B2100082199309A409B5098093D4049093D504A5
:10B22000A093D604B093D704BC01CD01A801970127
:10B230000E943A9A2093E2043093E3044093E4049A
:10B240005093E504D601C501D7FE04C081509F4F3D
:10B25000AF4FBF4F892F9A2FAB2FBB27A7FDBA95B2
:10B2600090931F0480931E0457FF04C021503F4F4A
:10B270004F4F5F4FBB2757FDBA95A52F942F832FB4
:10B2800090932104809320048091040490910504FC
:10B2900081349105DCF4809102049091030481349F
:10B2A0009105A4F480912C08E82FFF27EE0FFF1FD3
:10B2B000E25AF64F808191810190F081E02DF7FFF5
:10B2C00003C0F095E195FF4F7A97E4F08091CC0AA6
:10B2D0008F3FC1F480911E0490911F0497FD019649
:10B2E0009595879590931F0480931E048091200468
:10B2F0009091210497FD019695958795909321044F
:10B30000809320048091080A9091090AA0910A0A6A
:10B31000B0910B0AB7FF04C081509F4FAF4FBF4F92
:10B32000892F9A2FAB2FBB27A7FDBA958093080AC8
:10B330009093090AA0930A0AB0930B0A8091FB0923
:10B340009091FC09A091FD09B091FE09B7FF04C0DE
:10B3500081509F4FAF4FBF4F892F9A2FAB2FBB27E5
:10B36000A7FDBA958093FB099093FC09A093FD0972
:10B37000B093FE098091920490919304A09194045B
:10B38000B09195042F81388549855A85281B390B42
:10B390004A0B5B0B2093C8043093C9044093CA0442
:10B3A0005093CB0480918A0490918B04A0918C04DB
:10B3B000B0918D04EB84FC840D851E85E81AF90A92
:10B3C0000A0B1B0BE092CC04F092CD040093CE0448
:10B3D0001093CF042093D0043093D1044093D2042F
:10B3E0005093D304E092D404F092D5040093D60491
:10B3F0001093D70480916E0490916F04A091700413
:10B40000B0917104821B930BA40BB50B80936E0457
:10B4100090936F04A0937004B093710480916604BC
:10B4200090916704A0916804B09169048E199F09F6
:10B43000A00BB10B8093660490936704A0936804FB
:10B44000B093690488898823E1F020914C043091FD
:10B450004D04213831054CF08091A4049091A5044D
:10B4600001969093A5048093A40420583F4F4CF478
:10B470008091A4049091A50401979093A5048093D2
:10B48000A40410924D0410924C0481E090E090933B
:10B49000EB048093EA04E090D004F090D104009192
:10B4A000D2041091D304D801C70117FF07C0882721
:10B4B0009927DC018E199F09A00BB10B8150924096
:10B4C000A040B04034F084E090E09093EB0480938F
:10B4D000EA048091F0049091F104A091F204B091FB
:10B4E000F3042091130A3091140A4091150A5091E7
:10B4F000160A821B930BA40BB50B815E914BAF4FC9
:10B50000BF4F8F539C49A040B04028F08091CD0A96
:10B5100089310CF4FFC021E0E21620E1F20620E0C0
:10B52000020720E012070CF473C08091EC0488231A
:10B5300009F46AC0D801C70117FF07C088279927F7
:10B54000DC018E199F09A00BB10B9C01AD01B7FF67
:10B5500004C021503E4F4F4F5F4FF9E0559547953E
:10B5600037952795FA95D1F78091EA049091EB04ED
:10B57000820F931F9093EB048093EA04D801C701D4
:10B5800017FF03C00796A11DB11DE3E0B595A79570
:10B5900097958795EA95D1F78093DE049093DF0421
:10B5A000A093E004B093E10489589341A040B040D7
:10B5B00064F088E893E1A0E0B0E08093DE0490932B
:10B5C000DF04A093E004B093E1042091DE04309105
:10B5D000DF044091E0045091E10457FF04C0215082
:10B5E0003F4F4F4F5F4F232F342F452F552747FD98
:10B5F0005A9580911E0490911F04820F931F90937F
:10B600001F0480931E0406C081E08093EC0402C0F6
:10B610001092EC0440E0E41640EFF4064FEF04070C
:10B620004FEF14070CF073C08091ED04882309F4E8
:10B630006AC0D801C70117FF07C088279927DC0116
:10B640008E199F09A00BB10B9C01AD01B7FF04C07F
:10B6500021503E4F4F4F5F4F69E0559547953795C5
:10B6600027956A95D1F78091EA049091EB04820FB7
:10B67000931F9093EB048093EA04D801C70117FF4E
:10B6800003C00796A11DB11D23E0B595A795979519
:10B6900087952A95D1F78093DE049093DF04A093D9
:10B6A000E004B093E10488579C4EAF4FBF4F64F461
:10B6B00088E79CEEAFEFBFEF8093DE049093DF044A
:10B6C000A093E004B093E1042091DE043091DF0404
:10B6D0004091E0045091E10457FF04C021503F4FD6
:10B6E0004F4F5F4F232F342F452F552747FD5A9536
:10B6F00080911E0490911F04820F931F90931F044A
:10B7000080931E0411C081E08093ED040DC010925F
:10B71000ED040AC01092EB041092EA0484E690E073
:10B7200090938701809386016889262F3327809123
:10B73000EA049091EB042817390724F43093EB04C2
:10B740002093EA041091CD0A112379F0212F332799
:10B7500027FD30958091EA049091EB042817390772
:10B7600024F43093EB042093EA044091D0045091E8
:10B77000D1046091D2047091D30441385105610520
:10B78000710574F08091A8049091A9042091EA04B5
:10B790003091EB04820F931F9093A9048093A80427
:10B7A00040585F4F6F4F7F4F74F48091A804909181
:10B7B000A9042091EA043091EB04821B930B90932F
:10B7C000A9048093A80481E090E09093EB04809317
:10B7D000EA04C090D404D090D504E090D604F09050
:10B7E000D704D701C601F7FE07C088279927DC01D7
:10B7F0008C199D09AE09BF0981509240A040B0400C
:10B8000034F084E090E09093EB048093EA0480911C
:10B81000F4049091F504A091F604B091F7042091FE
:10B820001B0A30911C0A40911D0A50911E0A821B6E
:10B83000930BA40BB50B815E914BAF4FBF4F8F5352
:10B840009C49A040B04018F019310CF4FFC001E051
:10B85000C01600E1D00600E0E00600E0F0060CF4BF
:10B8600073C08091EE04882309F46AC0D701C60131
:10B87000F7FE07C088279927DC018C199D09AE09BE
:10B88000BF099C01AD01B7FF04C021503E4F4F4F8F
:10B890005F4F09E055954795379527950A95D1F75C
:10B8A0008091EA049091EB04820F931F9093EB0434
:10B8B0008093EA04D701C601F7FE03C00796A11DD5
:10B8C000B11D13E0B595A795979587951A95D1F772
:10B8D0008093E2049093E304A093E404B093E5041E
:10B8E00089589341A040B04064F088E893E1A0E01B
:10B8F000B0E08093E2049093E304A093E404B09357
:10B90000E5042091E2043091E3044091E404509175
:10B91000E50457FF04C021503F4F4F4F5F4F232F87
:10B92000342F452F552747FD5A958091200490913B
:10B930002104820F931F909321048093200406C05A
:10B9400081E08093EE0402C01092EE0420E0C21663
:10B9500020EFD2062FEFE2062FEFF2060CF073C0B5
:10B960008091EF04882309F46AC0D701C601F7FE6D
:10B9700007C088279927DC018C199D09AE09BF09EA
:10B980009C01AD01B7FF04C021503E4F4F4F5F4FA8
:10B99000E9E05595479537952795EA95D1F7809138
:10B9A000EA049091EB04820F931F9093EB04809331
:10B9B000EA04D701C601F7FE03C00796A11DB11D19
:10B9C00073E0B595A795979587957A95D1F780936C
:10B9D000E2049093E304A093E404B093E504885751
:10B9E0009C4EAF4FBF4F64F488E79CEEAFEFBFEFC4
:10B9F0008093E2049093E304A093E404B093E504FD
:10BA00002091E2043091E3044091E4045091E50474
:10BA100057FF04C021503F4F4F4F5F4F232F342F0C
:10BA2000452F552747FD5A95809120049091210478
:10BA3000820F931F909321048093200411C081E012
:10BA40008093EF040DC01092EF040AC01092EB0433
:10BA50001092EA0484E690E0909387018093860137
:10BA60004889242F33278091EA049091EB0428170A
:10BA7000390724F43093EB042093EA048091CD0A33
:10BA8000882379F0282F332727FD30958091EA0409
:10BA90009091EB042817390724F43093EB0420939A
:10BAA000EA044091D4045091D5046091D604709179
:10BAB000D704413851056105710574F08091A604E1
:10BAC0009091A7042091EA043091EB04820F931F18
:10BAD0009093A7048093A60440585F4F6F4F7F4F09
:10BAE000CCF48091A6049091A7042091EA043091AF
:10BAF000EB04821B930B9093A7048093A6040AC0C7
:10BB0000109221041092200410921F0410921E041F
:10BB100010924E048091210A882341F4109221044E
:10BB20001092200410921F0410921E048091130A98
:10BB30009091140AA091150AB091160A8093F0040E
:10BB40009093F104A093F204B093F30480911B0A44
:10BB500090911C0AA0911D0AB0911E0A8093F404D2
:10BB60009093F504A093F604B093F7041092820426
:10BB700010928304109284041092850410927E0423
:10BB800010927F04109280041092810410927A0423
:10BB900010927B0410927C0410927D041092130A80
:10BBA0001092140A1092150A1092160A10921B0A8B
:10BBB00010921C0A10921D0A10921E0A1092080A76
:10BBC0001092090A10920A0A10920B0A1092FB09AD
:10BBD0001092FC091092FD091092FE0910922203A6
:10BBE00010922103E0904404F0904504C701F7FE51
:10BBF00004C0882799278E199F0904973CF08091EB
:10BC00003C0A84FD03C082E3809322041091410822
:10BC1000A12EBB24CC24DD24B701882777FD809595
:10BC2000982F9701F7FE04C0222733272E193F09CA
:10BC3000442737FD4095542F0E94C6999B01AC01C3
:10BC4000C601B5010E94C69997FF04C061507E4F9E
:10BC50008F4F9F4F59E095958795779567955A95A2
:10BC6000D1F79B01812F99278E9DD0018F9DB00D1B
:10BC70009E9DB00D1124CD01B7FD03969595879536
:10BC800095958795280F391F8091FA039091FB03B2
:10BC90008150924010F020E030E080912404909197
:10BCA0002504280F391F442737FD4095542F209332
:10BCB000C4043093C5044093C6045093C7048091D4
:10BCC000620490916304A0916404B0916504821BA6
:10BCD000930BA40BB50B8093620490936304A09321
:10BCE0006404B09365048155934CA040B04064F067
:10BCF00080E593ECA0E0B0E080936204909363044D
:10BD0000A0936404B09365048091620490916304ED
:10BD1000A0916404B0916504805B9C43AF4FBF4F1A
:10BD200064F480EB9CE3AFEFBFEF809362049093E9
:10BD30006304A0936404B093650400918A01109198
:10BD40008B0117FDFCC080913C0A83FFF8C08091F5
:10BD50008901815080938901882309F0F4C08DE026
:10BD6000809389018091920490919304A09194040E
:10BD7000B0919504B7FF04C081509E4FAF4FBF4FA5
:10BD800039E0B595A795979587953A95D1F77C01B8
:10BD900097FF04C0F094E194F108F39480918A0431
:10BDA00090918B04A0918C04B0918D04B7FF04C0D6
:10BDB00081509E4FAF4FBF4F29E0B595A7959795FE
:10BDC00087952A95D1F79C0197FF03C0309521955F
:10BDD0003F4FE216F3060CF47901B701F7FE02C0FB
:10BDE000695F7F4F2B0183E0559447948A95E1F773
:10BDF00022E030E0420E531E60904C0A70904D0AD3
:10BE000080904E0A90904F0A20913C0130913D0164
:10BE100040913E0150913F01C401B3010E943A9A02
:10BE200059016A013093F9092093F809021B130B99
:10BE3000C801845E9D4F68E671E00E94059A9C01EE
:10BE4000245B30408091860190918701009731F00A
:10BE5000019790938701809386011BC049E1E41606
:10BE6000F104BCF480914C0490914D04820F931F17
:10BE700090934D0480934C0480912204882349F0D0
:10BE8000815080932204882321F4B0925104A0921F
:10BE900050048091860190918701892BF9F480915B
:10BEA00088019927289FB001299F700D389F700D38
:10BEB0001124CB01B2010E94059ACB01AA2797FD5C
:10BEC000A095BA2F680E791E8A1E9B1E60924C0A9E
:10BED00070924D0A80924E0A90924F0A80912204ED
:10BEE000882369F580915004909151042091F809BC
:10BEF0003091F909821B930B845E9D4F68E671E0D7
:10BF00000E94059A9C01245B3040809173018695C4
:10BF10009927289FD001299FB00D389FB00D11247B
:10BF20009D01B7FF02C0215F3F4F04E03595279583
:10BF30000A95E1F7309325042093240404C010925D
:10BF400025041092240480914E04882381F01092DD
:10BF500056041092570410925804109259041092EB
:10BF60005A0410925B0410925C0410925D04F090ED
:10BF70001B04FF20F1F48091210A282F3327442746
:10BF800055278091920490919304A0919404B091CC
:10BF90009504BC01CD010E94C699DC01CB01BC0116
:10BFA000CD0128EF3AE240E050E00E943A9A390190
:10BFB00002C066247724E0901A04EE20F1F4809108
:10BFC000210A282F33274427552780918A049091EE
:10BFD0008B04A0918C04B0918D04BC01CD010E9412
:10BFE000C699DC01CB01BC01CD0128EF3AE240E06B
:10BFF00050E00E943A9A290102C0442455248091BD
:10C00000F5099091F609893C91051CF088EC90E0C7
:10C0100005C088539F4F34F488E39FEF9093F6094F
:10C020008093F5098091000A9091010A893C91055D
:10C030001CF088EC90E005C088539F4F34F488E3EF
:10C040009FEF9093010A8093000A8091020A9091D9
:10C05000030AAA2797FDA095BA2F20914A0AA22E7B
:10C06000BB24CC24DD24BC01CD01A60195010E9496
:10C07000C6999B01AC018091F5099091F609AA2718
:10C0800097FDA095BA2F17E0880F991FAA1FBB1F15
:10C090001A95D1F7280F391F4A1F5B1F57FF04C09D
:10C0A000215C3F4F4F4F5F4FA6E055954795379521
:10C0B0002795AA95D1F78301020F131F1093030A46
:10C0C0000093020A8091F3099091F409AA2797FD41
:10C0D000A095BA2FBC01CD01A60195010E94C69979
:10C0E0009B01AC018091000A9091010AAA2797FD5B
:10C0F000A095BA2FF7E0880F991FAA1FBB1FFA95CA
:10C10000D1F7280F391F4A1F5B1F57FF04C0215C5E
:10C110003F4F4F4F5F4FE6E0559547953795279531
:10C12000EA95D1F74201820E931E9092F409809213
:10C13000F3098091450A9091460A880F991FAA2712
:10C1400097FDA095BA2F2091FA0933274427552748
:10C15000BC01CD010E94C6995B016C0197FF08C02C
:10C160002FE330E040E050E0A20EB31EC41ED51E07
:10C1700076E0D594C794B794A7947A95D1F7809137
:10C18000100A282F33274427552780917604909151
:10C190007704A0917804B0917904BC01CD010E948C
:10C1A000C699DC01CB01BC01CD0120EF35E540E0B3
:10C1B00050E00E943A9AB501620F731F7093460ACD
:10C1C0006093450A0150104134F080E090E1909373
:10C1D000030A8093020A8091020A9091030A805018
:10C1E000904F34F480E090EF9093030A8093020A1A
:10C1F00051E0851650E1950634F080E090E190938F
:10C20000F4098093F3098091F3099091F409805027
:10C21000904F34F480E090EF9093F4098093F30909
:10C220006150704134F080E090E19093460A809331
:10C23000450A8091450A9091460A8050904F34F407
:10C2400080E090EF9093460A8093450A8091010127
:10C25000482F5527809120019091210148175907B7
:10C2600094F4209120013091210109811A81049FC9
:10C27000C001059F900D149F900D1124B9010E94DB
:10C28000F1997A83698329813A81220F331F220F22
:10C29000331F3A83298380913C0A80FD02C00C94AD
:10C2A0008A6BEE2011F00C948A6BFF2011F00C9435
:10C2B0008A6B80919D0599278F779070009711F078
:10C2C0000C948A6B4C018091AA049091AB04892B49
:10C2D000D9F580911601909117018959934058F032
:10C2E00087B5803F20F480912503815011C081E003
:10C2F0008093030555C080911601909117018436F3
:10C300009105E8F487B58031B0F0809125038F5F07
:10C31000809325039FE08902900111248091D40726
:10C32000821B87BD8CE291E09093120380931103EE
:10C330008EE591E031C081E08093020531C0F0923A
:10C340000205F09203052CC09092240380922303EF
:10C350008091F703882321F081E00E94399417C06F
:10C360008091320490913304A0913404B09135044B
:10C3700054E0880F991FAA1FBB1F5A95D1F78093CD
:10C38000260390932703A0932803B0932903809159
:10C39000AA049091AB0401979093AB048093AA04F4
:10C3A00080913C0A2091150481FF3CC0223348F55E
:10C3B00080918F01815080938F018F3F09F052C08F
:10C3C0008091A401882339F480914F04882319F0C7
:10C3D00088E28093A40110924F04809132049091DE
:10C3E0003304A0913404B091350480932E049093CB
:10C3F0002F04A0933004B093310481E080938F0127
:10C4000031C0273478F18091A401882339F48091D8
:10C410004F04882319F487E28093A40188EC809369
:10C420008F011DC08091400190914101820F911DAB
:10C4300020913A083327829FA001839F500D929F3D
:10C44000500D1124CA01AA2797FDA095BA2F8093F9
:10C450002E0490932F04A0933004B093310481E014
:10C4600080934F048091920490919304A09194043E
:10C47000B0919504E0903C01F0903D0100913E01A7
:10C4800010913F01BC01CD01A80197010E943A9A89
:10C4900059016A0180918A0490918B04A0918C04C7
:10C4A000B0918D04BC01CD01A80197010E943A9A78
:10C4B000B901C5010E944A8B90930D0A80930C0A22
:10C4C000CC9734F08CE390E090930D0A80930C0AA3
:10C4D00080910C0A90910D0A0E94F47890930D0AB5
:10C4E00080930C0A80E280933B0110922D041092FD
:10C4F0002C0480914F04882309F470C78091FF03B6
:10C5000099279C012071307084FD68C78091FE03DB
:10C5100082608093FE0370911F0A872F992741E064
:10C52000C42ED12CC822D92280FD04C080913C0A9F
:10C5300081FD10C0E980FA803093F9042093F8045B
:10C5400030932D0420932C048091FF03806C809302
:10C55000FF03DFC28091FF0381FFAEC200917C0127
:10C5600010917D01C8010F96A0904204B090430441
:10C570008A159B050CF06EC080910205882309F096
:10C5800069C08091FA049091FB04459784F08091F2
:10C590001D0390911E03A0911F03B091200380936F
:10C5A0002E0490932F04A0933004B0933104809113
:10C5B000FF0387FF15C08091FF038F778093FF03F0
:10C5C00080911D0390911E03A0911F03B091200341
:10C5D00080932E0490932F04A0933004B0933104E1
:10C5E0008091FF0380648093FF03E090FF09EE20B9
:10C5F000F1F080912E0490912F04A0913004B0911D
:10C600003104BC01CD0124E630E040E050E00E945E
:10C610003A9A8E2D9927AA27BB2782179307A4073A
:10C62000B5072CF4D0922D04C0922C0410C0C50183
:10C63000801B910B0F9797FF03C0909581959F4F9B
:10C6400090932D0480932C048BE280933B011092F5
:10C65000260434C1C8010F97A816B906C4F5209165
:10C6600003052223A1F58091FF0386FF15C0809169
:10C67000FF038F7B8093FF0380911D0390911E0326
:10C68000A0911F03B091200380932E0490932F0458
:10C69000A0933004B09331048091FF0380688093AD
:10C6A000FF03C501801B910B0F9697FF03C0909568
:10C6B00081959F4F909581959F4F90932D048093E6
:10C6C0002C048DE280933B0120932604F7C08DE378
:10C6D00080933B0160912704662371F12091280427
:10C6E0003091290440912A0450912B0480912E040A
:10C6F00090912F04A0913004B091310482179307D8
:10C70000A407B507CCF48091FF0380648093FF03F6
:10C71000862F992790932D0480932C048AE0809390
:10C7200026048EE580933B018091FF0387FFC6C0FE
:10C730008091FF038F7733C0662309F443C02091B3
:10C7400028043091290440912A0450912B048091AF
:10C750002E0490912F04A0913004B0913104281739
:10C7600039074A075B0774F58091FF03806880935F
:10C77000FF03862F9927909581959F4F90932D04C5
:10C7800080932C0486EF8093260486E780933B01F8
:10C790008091FF0386FF92C08091FF038F7B80937F
:10C7A000FF0380911D0390911E03A0911F03B09180
:10C7B000200380932E0490932F04A0933004B09311
:10C7C00031047CC08091FF03807C09F477C08091A4
:10C7D0002604882309F04CC080911D0390911E030C
:10C7E000A0911F03B0912003885C9040A040B0400E
:10C7F00020912E0430912F04409130045091310447
:10C8000082179307A407B5076CF080911D039091E0
:10C810001E03A0911F03B0912003885C9040A040AC
:10C82000B0401DC080911D0390911E03A0911F0375
:10C83000B091200388539F4FAF4FBF4F2817390740
:10C840004A075B07BCF080911D0390911E03A091E5
:10C850001F03B091200388539F4FAF4FBF4F80936A
:10C860002E0490932F04A0933004B093310402C09F
:10C87000109226048091FF038F738093FF03109220
:10C88000F9041092F80471FF06C084EF91E09093D0
:10C8900012038093110380913604882379F48091E8
:10C8A000320490913304A0913404B0913504C397BD
:10C8B000A105B1051CF081E0809336046091F80475
:10C8C0007091F90480912C0490912D04680F791FC8
:10C8D0007093F9046093F804CB0177FF04C08827B4
:10C8E0009927861B970B855F91400CF4CEC0409131
:10C8F0002604442389F180912804909129042091F1
:10C900002E0430912F04821B930B0996439748F411
:10C910008091280490912904A0912A04B0912B04BD
:10C9200012C0242F332727FD3095432F532F80919A
:10C930002E0490912F04A0913004B0913104820F05
:10C94000931FA41FB51F80932E0490932F04A093D0
:10C950003004B093310424C020912E0430912F0470
:10C96000409130045091310480913A081616170610
:10C9700044F463E00E94E599280F311D411D511DCB
:10C9800007C063E00E94E599281B3109410951095C
:10C9900020932E0430932F0440933004509331049D
:10C9A0001092F9041092F804E0903204F0903304ED
:10C9B0000091340410913504D801C701805094408F
:10C9C000A040B04020912E0430912F0440913004BB
:10C9D0005091310482179307A407B5075CF4D8017E
:10C9E000C70180509C4FAF4FBF4F281739074A07E8
:10C9F0005B0744F080932E0490932F04A09330049F
:10CA0000B093310480911F0A81FF06C084E690E054
:10CA1000909312038093110380913E088823A9F517
:10CA200080912704882389F540911C0450911D04AE
:10CA300057FF02C04D5F5F4F5595479555954795F8
:10CA40008091200190912101209101013327489F7D
:10CA5000B001499F700D589F700D1124CB01B90191
:10CA60000E94059A70937D0160937C016634710584
:10CA70001CF486E490E005C06739710534F086E95E
:10CA800090E090937D0180937C018091AA04909125
:10CA9000AB04892BD1F180911D0390911E03A091CD
:10CAA0001F03B091200380932E0490932F04A09332
:10CAB0003004B093310429C0809132049091330442
:10CAC000A0913404B091350480599140A040B04009
:10CAD00080932E0490932F04A0933004B0933104DC
:10CAE00080913E08882311F0992702C088E790E0E2
:10CAF00090937D0180937C0189819A8190931D049C
:10CB000080931C048EE280933B01E0901C04F09023
:10CB10001D0480911D0390911E03A0911F03B091ED
:10CB2000200320912E0430912F0440913004509125
:10CB30003104281739074A075B0724F080911F0A40
:10CB400080FD98C48091F7036091AA047091AB04B2
:10CB5000882309F07CC2672B49F0E0901C04F09018
:10CB60001D041092FB041092FA04E1C080911D0391
:10CB700090911E03A0911F03B0912003821B930B81
:10CB8000A40BB50B8093C8049093C904A093CA0466
:10CB9000B093CB048230E0E89E07EFEFAE07EFEFF3
:10CBA000BE072CF481E090E8AFEFBFEF09C08F5FC4
:10CBB0009F47A040B04064F08FEF9FE7A0E0B0E057
:10CBC0008093C8049093C904A093CA04B093CB0483
:10CBD0008091C8049091C9049093FB048093FA0457
:10CBE00080917501282F3327442755278091C80449
:10CBF0009091C904A091CA04B091CB04BC01CD01AD
:10CC00000E94C69997FF04C0615E7F4F8F4F9F4F70
:10CC100025E095958795779567952A95D1F7609347
:10CC2000C8047093C9048093CA049093CB04653000
:10CC30000EEF70070FEF80070FEF90072CF484E0E2
:10CC40009EEFAFEFBFEF09C060507440804090404E
:10CC500064F080E094E0A0E0B0E08093C80490939A
:10CC6000C904A093CA04B093CB048090C8049090E8
:10CC7000C904209123033091240337FF02C0295FA8
:10CC80003F4F03E0359527950A95E1F74FEF22389E
:10CC900034071CF421E83FEF05C02038310514F0BB
:10CCA00020E830E0C901AA2797FDA095BA2F20916E
:10CCB0007601332744275527BC01CD010E94C69930
:10CCC00097FF04C06D5F7F4F8F4F9F4F12E0959588
:10CCD0008795779567951A95D1F79B015FEF61303E
:10CCE00075071CF420E03FEF06C06F3F710519F097
:10CCF00014F020E031E08091FF03807C49F0C9010D
:10CD000037FD03969C0135952795359527950DC0E0
:10CD100080911F0A80FF09C0C90137FD07969C0159
:10CD2000A3E035952795AA95E1F7820E931E2091F1
:10CD30007401222309F454C0609152047091530489
:10CD4000809154049091550497FF04C061587F4F1F
:10CD50008F4F9F4FF7E09595879577956795FA9553
:10CD6000D1F73327442755270E94C69997FF04C05F
:10CD7000615E7F4F8F4F9F4FE5E095958795779543
:10CD80006795EA95D1F76093C8047093C9048093BE
:10CD9000CA049093CB046138AFEF7A07AFEF8A07EC
:10CDA000AFEF9A072CF480E89FEFAFEFBFEF0AC018
:10CDB0006F3F71058105910569F064F080E091E0B5
:10CDC000A0E0B0E08093C8049093C904A093CA0483
:10CDD000B093CB048091C8049091C904880E991E29
:10CDE00080917201282F33278091D00A992787FDDF
:10CDF0009095289FF001299FF00D389FF00D112488
:10CE00009F01F7FF02C021583F4F220F232F221FFF
:10CE1000330BFFEF21383F071CF420E83FEF06C03B
:10CE20002F3F310519F014F020E031E0280D391DB5
:10CE3000C901AA2797FDA095BA2F00911C04109153
:10CE40001D049801442737FD4095542FBC01CD01A6
:10CE50000E94C69997FF04C061507E4F8F4F9F4F2D
:10CE600059E095958795779567955A95D1F7E61A84
:10CE7000F70A80912C0490912D04892B09F064C04D
:10CE8000101611060CF060C02091FA043091FB04DA
:10CE9000C90137FF03C0309521953F4F2D33310530
:10CEA00040F480914A0490914B048E159F0574F5CF
:10CEB00026C02C53304045E0369527954A95E1F73A
:10CEC0002031310510F02FE030E040914A045091BC
:10CED0004B0418161906E4F480E190E0821B930BD2
:10CEE000489F9001499F300D589F300D1124B4E0A8
:10CEF00036952795BA95E1F72E153F0520F58091D7
:10CF00007A0190917B01E816F906F4F07C011CC0CF
:10CF1000205F3F4F80917A0190917B01829FB00109
:10CF2000839F700D929F700D11249B01A4E0369594
:10CF30002795AA95E1F74E155F0514F07A0104C014
:10CF4000E216F30608F07901C701AA2797FDA0951C
:10CF5000BA2FFDE0880F991FAA1FBB1FFA95D1F7C2
:10CF600020910C0A30910D0A442737FD4095542F2B
:10CF7000BC01CD010E943A9A2093CC043093CD0499
:10CF80004093CE045093CF04E090CC04F090CD04B5
:10CF90008091FC049091FD049C01220F331F280F07
:10CFA000391F2E0D3F1D37FF02C02D5F3F4FA901D6
:10CFB00055954795559547955093FD044093FC042E
:10CFC00080913608282F3327220F331F220F331F5B
:10CFD000241735076CF48091440A282F3327220F39
:10CFE000331F220F331F205530404217530724F0C0
:10CFF0003093FD042093FC0480911F0A80FF14C02D
:10D000008091FC049091FD04A981BA818A179B0745
:10D0100024F0B093FD04A093FC04E091FC04F09193
:10D02000FD04FA83E98326C229813A81201B310B52
:10D0300037FF02C02D5F3F4F3595279535952795D2
:10D04000E090FC04F090FD04E20EF31EC1C1672BDA
:10D0500049F0E0901C04F0901D041092FB04109223
:10D06000FA0438C180911D0390911E03A0911F0303
:10D07000B0912003821B930BA40BB50B8093C804C3
:10D080009093C904A093CA04B093CB04823000E803
:10D0900090070FEFA0070FEFB0072CF481E090E8A6
:10D0A000AFEFBFEF09C08F5F9F47A040B04064F073
:10D0B0008FEF9FE7A0E0B0E08093C8049093C9048D
:10D0C000A093CA04B093CB048091C8049091C90482
:10D0D0009093FB048093FA0480917501282F3327E5
:10D0E000442755278091C8049091C904A091CA048F
:10D0F000B091CB04BC01CD010E94C69997FF04C03A
:10D10000615E7F4F8F4F9F4F05E09595879577958F
:10D1100067950A95D1F76093C8047093C90480930A
:10D12000CA049093CB04653028EF72072FEF820773
:10D130002FEF92072CF484E098EFAFEFBFEF09C018
:10D14000605078408040904064F080E098E0A0E03B
:10D15000B0E08093C8049093C904A093CA04B0932C
:10D16000CB048090C8049090C90480917401282F4A
:10D17000332780912A0390912B03829FA001839FE4
:10D18000500D929F500D11249A0157FF02C021505B
:10D190003F4F232F330F330B8091230390912403B0
:10D1A000820F931FAA2797FDA095BA2F8093C804DA
:10D1B0009093C904A093CA04B093CB048091260431
:10D1C00020912C0430912D04882331F0B3E0220FFC
:10D1D000331FBA95E1F71BC080913A089927289F21
:10D1E000B001299F700D389F700D11249B01A3E0A1
:10D1F000220F331FAA95E1F7260F371F37FF02C012
:10D20000215E3F4FF5E035952795FA95E1F730938C
:10D21000F9032093F8038091F8039091F9039C019E
:10D22000442737FD4095542F8091C8049091C9043C
:10D23000A091CA04B091CB04821B930BA40BB50B35
:10D240008093C8049093C904A093CA04B093CB04FC
:10D2500020917601332744275527BC01CD010E9438
:10D26000C69997FF04C0615E7F4F8F4F9F4FE5E0E7
:10D270009595879577956795EA95D1F76093C8045A
:10D280007093C9048093CA049093CB046530A8EFCF
:10D290007A07AFEF8A07AFEF9A072CF484E098EF94
:10D2A000AFEFBFEF09C0605078408040904064F01D
:10D2B00080E098E0A0E0B0E08093C8049093C904B7
:10D2C000A093CA04B093CB048091C8049091C90480
:10D2D000880E991EE818F90880914A0490914B0431
:10D2E0008E159F053CF480917A0190917B01E816A0
:10D2F000F9060CF07C01C701AA2797FDA095BA2F6B
:10D300005DE0880F991FAA1FBB1F5A95D1F7209186
:10D310000C0A30910D0A442737FD4095542FBC016B
:10D32000CD010E943A9A2093CC043093CD044093CF
:10D33000CE045093CF04E090CC04F090CD048091C3
:10D34000FC049091FD049C01220F331F280F391F0C
:10D350002E0D3F1D37FF02C02D5F3F4FA901559590
:10D360004795559547955093FD044093FC04809153
:10D370003608282F3327220F331F220F331F24177D
:10D3800035076CF48091440A282F3327220F331F6E
:10D39000220F331F205530404217530724F030939B
:10D3A000FD042093FC0480911F0A2091FC0430911D
:10D3B000FD0480FF10C0E981FA812E173F0724F099
:10D3C000F093FD04E093FC04E090FC04F090FD0475
:10D3D000FA82E9824FC03A8329834CC080913E088B
:10D3E000882301F560911C0470911D0477FF02C031
:10D3F0006D5F7F4F75956795759567954091200195
:10D400005091210180910101282F3327649FC00191
:10D41000659F900D749F900D1124B9010E94059A8B
:10D42000CB0101C0992790937D0180937C0180916D
:10D430007C0190917D01873491051CF486E490E095
:10D4400005C08639910534F086E990E090937D011E
:10D4500080937C0109811A811093FD040093FC04E0
:10D460008091FF03806C8093FF038091FE038D7F8A
:10D470008093FE038091FF0399279C0122703070F6
:10D4800081FF39C18091FE049091FF04A0910005B5
:10D49000B09101050097A105B10521F080913604F6
:10D4A0008130B9F480911C0490911D04AA2797FD46
:10D4B000A095BA2F1EE0880F991FAA1FBB1F1A95AF
:10D4C000D1F78093FE049093FF04A0930005B093DE
:10D4D000010580913604813019F482E0809336048E
:10D4E00029813A8179010027F7FC0095102F80915E
:10D4F0000C0A90910D0A9C01442737FD4095542F4A
:10D50000C801B7010E94C699DC01CB018093CC040D
:10D510009093CD04A093CE04B093CF04B7FF04C082
:10D520008150904EAF4FBF4F7C018D01ADE01595FE
:10D530000795F794E794AA95D1F7E092CC04F0927E
:10D54000CD040093CE041093CF0460910004709139
:10D5500001043FE0603A730750F58091FE0490911A
:10D56000FF04A0910005B09101059C01AD01FAE016
:10D570005695479537952795FA95D1F7821B930BCA
:10D58000A40BB50BA8019701E4E0220F331F441F41
:10D59000551FEA95D1F7820F931FA41FB51F8093E3
:10D5A000FE049093FF04A0930005B093010560541E
:10D5B0007F4118F58091FE049091FF04A091000531
:10D5C000B09101059C01AD016CE0569547953795EA
:10D5D00027956A95D1F7821B930BA40BB50BA80175
:10D5E0009701F2E0220F331F441F551FFA95D1F720
:10D5F000820F931FA41FB51F41C0809123039091F8
:10D600002403809123039091240397FF03C09095F6
:10D6100081959F4F84369105CCF580911D039091A3
:10D620001E03A0911F03B09120039C0180912E0442
:10D6300090912F04281B390B37FF03C0309521959B
:10D640003F4F2F3F310509F00CF58091FE0490917A
:10D65000FF04A0910005B09101059C01AD01EEE031
:10D660005695479537952795EA95D1F7821B930BE9
:10D67000A40BB50B8E0D9F1DA01FB11F8093FE0440
:10D680009093FF04A0930005B09301058091FE04E0
:10D690009091FF04A0910005B09101057EE0B69540
:10D6A000A795979587957A95D1F790931D048093C8
:10D6B0001C0440913C08442399F055279C01BA0171
:10D6C0000E94059AC901861B970B90934B04809387
:10D6D0004A04260F371F30937B0120937A011FC025
:10D6E00010924B0410924A048FEF93E090937B01C9
:10D6F00080937A0114C0109236041092FE041092A6
:10D70000FF04109200051092010530931D04209330
:10D710001C0405C08091FF03806C8093FF038091FF
:10D72000120581FF37C089819A8197FD03969595EF
:10D730008795959587952091FC033091FD032817D7
:10D74000390760F480911C0490911D04892B31F0FD
:10D75000220F331F220F331F3A83298380911D0329
:10D7600090911E03A0911F03B091200380932E047B
:10D7700090932F04A0933004B093310488E99AE386
:10D78000909312038093110380E09EE090930B012D
:10D7900080930A012091070A822F9927880F991FE9
:10D7A000880F991F889669817A818617970714F0E8
:10D7B0009A8389837091440A7D8B872F9927880FDC
:10D7C000991F880F991F80559040A981BA818A17A7
:10D7D0009B0714F49A83898380915B03882341F427
:10D7E0008091E20A8F3F21F4809116058823E9F0A9
:10D7F00080910004909101040297C097B0F4E981F0
:10D80000FA811E161F068CF481E090E090930104CB
:10D8100080930004E22EFF24EE0CFF1CEE0CFF1C94
:10D820008701085D1F4F1A83098329813A8130934C
:10D830009207209391078091C4049091C504A09110
:10D84000C604B091C70412E0880F991FAA1FBB1F1E
:10D850001A95D1F70091450A1091460A081B190B39
:10D86000213A31058CF0C90137FD019695958795D0
:10D87000801791070CF48C01909581959F4F0817A4
:10D8800019076CF48C010BC00135110514F000E58B
:10D8900010E03FEF003B130714F400EB1FEF4D893E
:10D8A000242F3327220F331F220F331FC901698111
:10D8B0007A81861B970B801791070CF48C01898164
:10D8C0009A81821B930B081719070CF48C01809125
:10D8D000020A9091030A6091480470914904861BE2
:10D8E000970B9093120A8093110AD090210A2091ED
:10D8F0005A0430915B0440915C0450915D04DD203A
:10D9000041F0661A770AC301AA2797FDA095BA2F9E
:10D9100004C0AA2797FDA095BA2F280F391F4A1FC8
:10D920005B1F20935A0430935B0440935C04509334
:10D930005D0480915A0490915B04A0915C04B091C5
:10D940005D0481509A4FA040B04064F080E09AEFAF
:10D95000A0E0B0E080935A0490935B04A0935C0431
:10D96000B0935D0480915A0490915B04A0915C0493
:10D97000B0915D0480509640AF4FBF4F64F480E09B
:10D9800096E0AFEFBFEF80935A0490935B04A093AF
:10D990005C04B0935D04C0904B082091110A309153
:10D9A000120A78E0E72EEC1498F08C2D9927829FCC
:10D9B000A001839F500D929F500D1124CA0157FD65
:10D9C00007967C0163E0F594E7946A95E1F712C04D
:10D9D0008C2D86959927829FB001839F700D929F11
:10D9E000700D1124CB0177FD03967C01F594E7942B
:10D9F000F594E794A0907701B090780195014427C1
:10DA000037FD4095542F80915A0490915B04A0916A
:10DA10005C04B0915D04BC01CD010E943A9AE20E13
:10DA2000F31E90906101692D772788279927980127
:10DA300017FF04C022273327201B310B37FF02C0FA
:10DA40002F5F3F4F35952795A981BA812A0F3B1F3C
:10DA5000442737FD4095542F0E94C69997FF04C074
:10DA6000615C7F4F8F4F9F4F26E095958795779507
:10DA700067952A95D1F79B016E157F050CF47B0104
:10DA8000309521953F4FE216F3060CF47901809111
:10DA9000F3099091F4096091460470914704861B44
:10DAA000970B9093F2098093F109209156043091DD
:10DAB00057044091580450915904DD2041F0461A12
:10DAC000570AC201AA2797FDA095BA2F04C0AA271A
:10DAD00097FDA095BA2F280F391F4A1F5B1F20936F
:10DAE000560430935704409358045093590480913E
:10DAF000560490915704A0915804B0915904815054
:10DB00009A4FA040B04064F080E09AEFA0E0B0E00F
:10DB10008093560490935704A0935804B0935904EB
:10DB20008091560490915704A0915804B0915904E3
:10DB300080509640AF4FBF4F64F480E096E0AFEF67
:10DB4000BFEF8093560490935704A0935804B0936A
:10DB500059042091F1093091F20948E04C1598F0F0
:10DB60008C2D9927829FB001839F700D929F700D1D
:10DB70001124CB0177FD07966C01B3E0D594C794CF
:10DB8000BA95E1F712C0C6948C2D9927829FD001D7
:10DB9000839FB00D929FB00D1124CD01B7FD039668
:10DBA0006C01D594C794D594C7949501442737FD4B
:10DBB0004095542F8091560490915704A091580499
:10DBC000B0915904BC01CD010E943A9AC20ED31EF5
:10DBD000692D772788279927980117FF04C02227E6
:10DBE0003327201B310B37FF02C02F5F3F4F359586
:10DBF0002795E981FA812E0F3F1F442737FD409575
:10DC0000542F0E94C69997FF04C0615C7F4F8F4FCD
:10DC10009F4FE6E09595879577956795EA95D1F7BB
:10DC20009B016C157D050CF46B01309521953F4FE0
:10DC3000C216D3060CF469018091070A282E3324FA
:10DC400050908D086DEF862E68E0962E54EBA52E31
:10DC500058E0B52E4BE0442E32E2632E3AE0732EAC
:10DC6000D5012C9112160CF029C1203429F4E98138
:10DC7000FA81FF8BEE8B1FC049815A81CA01AA2706
:10DC800097FDA095BA2F332727FD3095432F532FAB
:10DC9000BC01CD010E94C69997FF04C0615C7F4F13
:10DCA0008F4F9F4F26E095958795779567952A9595
:10DCB000D1F77F8B6E8BF5012181203439F42E89C9
:10DCC0003F892E0D3F1D3F8B2E8B2AC0203C39F4FF
:10DCD0004E895F894E195F095F8B4E8B21C0C7014A
:10DCE000AA2797FDA095BA2F332727FD3095432FFC
:10DCF000532FBC01CD010E94C69997FF04C0615CFF
:10DD00007F4F8F4F9F4FB6E0959587957795679595
:10DD1000BA95D1F7AE89BF89A60FB71FBF8BAE8B5F
:10DD2000F5012281203439F42E893F892C0D3D1DC7
:10DD30003F8B2E8B2AC0203C39F44E895F894C19C9
:10DD40005D095F8B4E8B21C0C601AA2797FDA09568
:10DD5000BA2F332727FD3095432F532FBC01CD0118
:10DD60000E94C69997FF04C0615C7F4F8F4F9F4F01
:10DD7000A6E09595879577956795AA95D1F7AE8991
:10DD8000BF89A60FB71FBF8BAE8BF501238120344F
:10DD900039F42E893F89200F311F3F8B2E8B2AC0EB
:10DDA000203C39F44E895F89401B510B5F8B4E8BB1
:10DDB00021C0C801AA2797FDA095BA2F332727FDB8
:10DDC0003095432F532FBC01CD010E94C69997FF78
:10DDD00004C0615C7F4F8F4F9F4FF6E0959587950C
:10DDE00077956795FA95D1F7AE89BF89A60FB71FCA
:10DDF000BF8BAE8BF301808191812E893F89821781
:10DE0000930764F4B901680F791F77FF02C06F5F51
:10DE10007F4F759567957F8B6E8B1DC0552049F49C
:10DE20004E895F89440F551F481B590B5F8B4E8BE2
:10DE300012C051E0551578F4252D33276E897F895E
:10DE4000861B970BB9010E94059AAE89BF89A60F60
:10DE5000B71FBF8BAE8BC101880F991F880F991F09
:10DE6000EE89FF898E179F0764F4FD898F2F99270C
:10DE7000880F991F880F991F2E893F892817390706
:10DE800014F09F8B8E8B8E899F8997FD03969595B5
:10DE9000879595958795F4018183880F991F880F41
:10DEA000991F2E893F89281B390BC901880F82834E
:10DEB000EE89FF89D301ED93FC9303C0F401118235
:10DEC00012824A9422E030E0620E731E44E050E079
:10DED000A40EB51E68E070E0860E971E47FEC0CE09
:10DEE000E2E1C95E0C94719A84B1806A84B93D9A6A
:10DEF00082E58CBD1DBC459A81E08093560A8AEA72
:10DF00008093670A83E88093680A8AE08093690AAD
:10DF100010926B0A10926A0A10926D0A10926C0AA3
:10DF20001092CF0A10928B0A08953091560A33232B
:10DF300009F070C00DB407FE6DC083E0809310033C
:10DF4000459A2EB58091190599278130910589F060
:10DF5000823091051CF4892B21F03EC00297B9F064
:10DF60003BC030938A0A20931A052138A9F581E035
:10DF700008C0253549F480911A05820F80931A054F
:10DF800082E08093190528C03093190525C080913F
:10DF90008A0AE82FFF27E455F54F20838F5F80938F
:10DFA0008A0A90911A058032A0F0291769F480E25C
:10DFB000ACEABAE0ECE8FAE00D9001928A95E1F75C
:10DFC00081E080938B0A02C030938B0A109219056E
:10DFD00003C0920F90931A052091660A2232A0F492
:10DFE00045980000000000000000E0915F0AF091F9
:10DFF000600AE20FF11D80818EBD8091880A9081B8
:10E00000890F8093880A03C081E08093560A2F5FAE
:10E010002093660A0895EF92FF920F931F938091C9
:10E0200044089927880F991F880F991F7C010027A2
:10E03000F7FC0095102F8091920490919304A09189
:10E040009404B0919504BC01CD01A80197010E94F0
:10E050003A9A30936B0A20936A0A80918A049091CD
:10E060008B04A0918C04B0918D04BC01CD01A8015A
:10E0700097010E943A9A30936D0A20936C0A20917E
:10E080004C0A30914D0A40914E0A50914F0ADA01E4
:10E09000C90173E0880F991FAA1FBB1F7A95D1F79A
:10E0A000820F931FA41FB51F820F931FA41FB51FBC
:10E0B00020913C0130913D0140913E0150913F0142
:10E0C000BC01CD010E943A9A3093730A2093720AE0
:10E0D0008091A4049091A5042091300330913103E4
:10E0E000821B930B9093790A8093780AE0919A04AB
:10E0F000F0919B048091180A9091190ABF010E9427
:10E10000059ACB019B01220F331F220F331F280FCB
:10E11000391F280F391F37FF02C02D5F3F4F35953C
:10E1200027953595279530936F0A20936E0A809135
:10E13000480A9091490ABF010E94059A9B01220F4B
:10E14000331F220F331F260F371F260F371F37FFAE
:10E1500002C02D5F3F4F3595279535952795309314
:10E16000710A2093700A10929B0410929A041092E4
:10E17000190A1092180A1092490A1092480A8091BE
:10E18000690A9927AA27BB27FC013A97E830F105CD
:10E1900008F029C2E058FF4F0C948C9A8091140427
:10E1A00080937C0A8091130480937D0A80911204ED
:10E1B00080937E0A8091110480937F0A80911004DD
:10E1C0008093800A80910F048093810A80910E04CD
:10E1D0008093820A80910D048093830A8091FF03CB
:10E1E0008093840A8091FF03837F8093FF03809153
:10E1F00000018093850A80918E088093860A809121
:10E20000FE038093870A4299EEC18091FE03877FC7
:10E210008093FE03E8C18091DC0A9091DD0A90931F
:10E220007D0A80937C0A8091E00A9091E10A9093A4
:10E230007F0A80937E0A8091200190912101809332
:10E24000800A809179080E94C6478093810A809154
:10E250003B018093820A90911B059093830AE92FDA
:10E26000FF2713E0EE0FFF1F1A95E1F7E350F74F7A
:10E2700086818093840A83818093850A8781809335
:10E28000860A85818093870A9F5F90931B05E92FFB
:10E29000FF27EE0FFF1FEE0FFF1FE955F74F858594
:10E2A000882309F0A0C1992309F49DC1892F9927DA
:10E2B00001966CE070E00E94059A9C01982FE82F6F
:10E2C000FF27EE0FFF1FEE0FFF1FE955F74F858564
:10E2D000882311F4222351F720931B0584C18091D8
:10E2E000010180937C0A80917A0880937D0A809155
:10E2F0007B0880937E0A80917C0880937F0A8091BE
:10E300007D088093800A809181088093810A8091A2
:10E3100082088093820A809183088093830A809187
:10E3200086088093840A809184088093850A80916E
:10E3300085088093860A8091870853C18091780868
:10E3400080937C0A80914F08863081F08091DC02B6
:10E35000823451F00E94367AE82FFF27E853FF4EAF
:10E3600084918093DC0202C00E94367A80913F053E
:10E3700080937D0A8091950880937E0A34C1F89439
:10E3800080912B08E82FFF27EE0FFF1FE25AF64F70
:10E390000190F081E02DE038F1051CF0EFE7F0E0AE
:10E3A00006C02FEFE138F20714F4E1E8FFEFE09345
:10E3B0007C0A80912C08E82FFF27EE0FFF1FE25AFE
:10E3C000F64F0190F081E02DE038F1051CF0EFE709
:10E3D000F0E006C07FEFE138F70714F4E1E8FFEF63
:10E3E000E0937D0A80912A08E82FFF27EE0FFF1F98
:10E3F000E25AF64F0190F081E02DE038F1051CF073
:10E40000EFE7F0E006C08FEFE138F80714F4E1E839
:10E41000FFEFE0937E0A80912908E82FFF27EE0F97
:10E42000FF1FE25AF64F0190F081E02DE038F10530
:10E430001CF0EFE7F0E006C02FEFE138F20714F42C
:10E44000E1E8FFEF7894E0937F0A809139048093AC
:10E45000800A80913A048093810A80913B048093E2
:10E46000820A80913C048093830A80913D048093CA
:10E47000840A80913E048093850A80913F048093B2
:10E48000860A80914004ADC08091B805863018F0AE
:10E490001092B80585E080937C0A8091880880936B
:10E4A0007D0A8091320490913304A0913404B0919C
:10E4B0003504BC01CD0125E030E040E050E00E9491
:10E4C0003A9A30937F0A20937E0A80912E0490918D
:10E4D0002F04A0913004B0913104BC01CD0125E09E
:10E4E00030E040E050E00E943A9A3093810A209355
:10E4F000800A80917E088093820A80917F088093B1
:10E50000830A809180088093840A809138048093E4
:10E51000850A1092860A809191079091920797FD43
:10E52000039695958795959587955BC082E0809336
:10E530007C0A10927D0A10927E0A87E380937F0AFC
:10E54000809102018093800A80919D058093810AC9
:10E5500090919E059093820A8F7780939D0590718C
:10E5600090939E051092830A80913C0A8093840ABE
:10E5700080911F0A8093850A80918A088093860A79
:10E58000809199082EC080915D0880937C0A8091CB
:10E59000970880937D0A8091690180937E0A80911B
:10E5A000560880937F0A809157088093800A809153
:10E5B00058088093810A809168018093820A809133
:10E5C0005A088093830A80915B088093840A809123
:10E5D0005C088093850A8091E20A8093860A809184
:10E5E000BB078093870A80918B0A882309F47DC139
:10E5F00060918C0A8091A001681719F08AEF8093CE
:10E600009E016093A00181E08093890140918D0A71
:10E6100050918E0ACA0181509E4F8F5F9340B0F493
:10E6200020918F0A3091900AC90181509E4F8F5FCF
:10E63000934060F48091350885FF08C05093080529
:10E640004093070530930605209305058091930AB2
:10E650009091940A21E08936920724F490938B01DB
:10E6600080938A0120919D0A30919E0A8091110326
:10E67000909112038217930740F48091E40288235B
:10E6800021F43093120320931103862F99278936A2
:10E69000910509F4A5C08A36910544F487369105A1
:10E6A00071F08836910509F462C027C18A36910558
:10E6B00009F414C18B36910509F4E2C01EC18091A2
:10E6C0009F0A8093CC0A8091A00A8093CE0A809101
:10E6D000A10A8093CD0A8091A20A8093880180913B
:10E6E000A30A8093D00A8091A40A80939F0180910D
:10E6F000A50A809318058091A60A8093040580914D
:10E700000C048823F9F02091A70A3091A80A37FD5C
:10E7100019C0309351042093500490915F089923BD
:10E7200089F08FE0989FC0011124281B390BC90183
:10E7300088599E4F68E671E00E94059A90935104B3
:10E740008093500420910F05309110058091A90A03
:10E750009091AA0A280F391F37FF02C02F5F3F4F41
:10E76000359527953093100520930F05C6C08091ED
:10E770009F0A8093610A8091A00A8093620A809127
:10E78000A10A8093630A8091A20A8093640A80910F
:10E79000A30A8093650A809181079091A40A892B2E
:10E7A000809381079091820793708091A50A8C7065
:10E7B000982B909382078091A60A809316058091EA
:10E7C000A70A809390018091A80A8093CF0A809134
:10E7D000A90A809312058091AA0A809311058DC021
:10E7E00080919F0A8093570A8091A00A8093580ACB
:10E7F0008091A10A8093590A8091A20A80935A0AB3
:10E800008091A30A9091A40A90935C0A80935B0A7A
:10E810008091A50A9091A60A90935E0A80935D0A62
:10E820008091A70A992787FD9095909399098093E5
:10E8300098098091A80A809327048091A90A909151
:10E84000AA0A9C01442737FD4095542FDA01C901DB
:10E8500063E0880F991FAA1FBB1F6A95D1F7820F2B
:10E86000931FA41FB51F820F931FA41FB51F809372
:10E87000280490932904A0932A04B0932B043DC04C
:10E8800080919F0A809315058091A00A80931405BA
:10E890008091A10A809313059091A20A992349F0CF
:10E8A0008091A401882319F08151833010F4909352
:10E8B000A4018091A30A809344058091A40A8093C7
:10E8C00043058091A50A9091A60A909341058093F3
:10E8D00040058091A70A809342050FC080914F08A0
:10E8E000863059F40E948F7A08C010920805109261
:10E8F000070510920605109205051F910F91FF90D4
:10E90000EF9008958091560A882319F1459887E67B
:10E910009AE09093600A80935F0A90911705E92F1F
:10E92000FF27EF56FE4F9F5F9093170580818093DE
:10E93000690A9D3010F0109217051092560A0E9435
:10E940000B7081E08093660A8091670A8093880A41
:10E950008EBD089587B18C6087B942984398109214
:10E960001D0580E88093A20110921C058093A101EF
:10E970000895809198099091990981589F4F39F095
:10E9800080919809909199098158809327058091E9
:10E9900022058150809322058F3F09F043C189E011
:10E9A000809322058091FF03992780739070892BB3
:10E9B00021F480919E0580FF1DC0809176088823F8
:10E9C00051F080912505882319F484E080931D057A
:10E9D00081E080932505809177088823B9F08091A4
:10E9E0002605882319F484E080931C0581E0809338
:10E9F00026050CC0109225051092260580917208FC
:10EA000080932305809174088093240580912505C7
:10EA1000882309F073C080919608282F332724FF9C
:10EA200007C080913704882319F425FD80C081C078
:10EA300090917308983F48F080911A0A8D3D28F014
:10EA40008091230588236CF00AC0983F68F080917C
:10EA50001A0A853049F48091230587FF02C0429845
:10EA600001C0429A81E032C080911D05815080939F
:10EA70001D058F3F09F05EC08091990885FF29C070
:10EA800090912705892F869580931D05992351F430
:10EA90008091230587FF02C0429801C0429A1092DC
:10EAA000A20148C08091A20190912305882341F4DE
:10EAB0008093270580E88093A2019923D4F137C081
:10EAC000982311F0429A01C0429886958093A20142
:10EAD00031C080911A0A869580931D058091A2010C
:10EAE000813021F41092270580E801C0869580933B
:10EAF000A2018091A2019091230517C080911D056C
:10EB0000815080931D058F3FA9F489E080931D05F6
:10EB10008091A201813011F480E801C08695809334
:10EB2000A2018091A20190917608892311F0429A66
:10EB300001C0429880912605882309F043C0909136
:10EB4000960897FF07C080913704882319F496FD33
:10EB500052C053C090917508983F48F08091430A85
:10EB60008D3D28F08091240588236CF00AC0983FE1
:10EB700078F08091430A853059F48091240587FF0D
:10EB800002C0439801C0439A81E08093A10136C03E
:10EB900080911C05815080931C058F3F79F58091F1
:10EBA000430A869580931C058091A101813011F460
:10EBB00080E801C086958093A1018091A101909188
:10EBC000240517C080911C05815080931C058F3F40
:10EBD000A9F489E080931C058091A101813011F492
:10EBE00080E801C086958093A1018091A101909158
:10EBF0007708892311F0439A01C04398429B05C0CE
:10EC00008091FE0388608093FE03439B06C0809141
:10EC1000FE0380618093FE0308958091FE038F7E42
:10EC20008093FE0308950F931F93CF93DF93482F94
:10EC3000EB0180913804E42FFF27843BD8F08F014B
:10EC40000E0F1F1FF801E25AF64F808191819B0140
:10EC5000281B390BC90163E070E00E94059ACB01C3
:10EC6000880F991F860F971F0C55164FF801918337
:10EC7000808306C0EE0FFF1FEC55F64F1182108205
:10EC8000E42FFF27EE0FFF1FE25AF64FD183C08318
:10EC9000DF91CF911F910F9108954FB724E130E09C
:10ECA000F8948091C9008F778093C9008091C90042
:10ECB0008F7B8093C9008091C9008F7D8093C900AC
:10ECC000832F99278093CD002093CC008091C8009A
:10ECD00082608093C80080E18093C9008091CA005F
:10ECE0008F778093CA008091CA008F7B8093CA007F
:10ECF0008091CA008F7D8093CA008091CA008F7E68
:10ED00008093CA008091CA00877F8093CA00809157
:10ED1000C9008B7F8093C9008091CA008460809372
:10ED2000CA008091CA0082608093CA008091C800A6
:10ED300087FF03C08091CE00F9CF8091C900806821
:10ED40008093C9004FBF0895EF92FF920F931F93D6
:10ED5000CF93DF93482F00E010E08091A301813032
:10ED600061F41092A30184E480932A0510922C058B
:10ED700010922B0510922D05E6C180912A0588235B
:10ED800019F421E030E001C0980190912B059923FE
:10ED900071F4232B11F081E010C084E480932A05E4
:10EDA00090932C0590932B0590932D05B5C1913030
:10EDB00069F4232B09F0A6C182E080932B05809192
:10EDC0002C058F5F80932C0583E0A4C19230D1F491
:10EDD000232B09F097C183E080932A0540932D05EA
:10EDE00090912C05923039F410922E0547FF03C004
:10EDF00081E080932E0583E080932B059F5F9093A5
:10EE00002C058AC1933009F07DC1232B09F07AC10A
:10EE100090932A0582E080932B0580912C058F5FCB
:10EE200080932C0520912D05822F9927782F662716
:10EE3000842F9927682B792B80914F08813051F4CA
:10EE40007370CB018050924063E070E00E94059A9D
:10EE5000EB0119C0823069F47770CB018050944087
:10EE600066E070E00E94059AEB01269526952695AE
:10EE70000CC0EB01D370C856D140CE01D7FD01962E
:10EE8000EC01D595C79526952695022F11270F7071
:10EE900010700F5F1F4F0D30110508F02CC10230AC
:10EEA000110519F404E010E005C00430110511F457
:10EEB00002E010E0D801A00FB11FFD01E25AF64FA9
:10EEC000808191819E01281B390BC90137FF03C046
:10EED000909581959F4F069704F5E0919108EE2358
:10EEE00051F0FF27EE0FFF1FE25AF64F808191810C
:10EEF0008436910594F480913804883C30F48091F4
:10EF00003804865F8093380408C088EC8093380406
:10EF100080916F008F7D80936F00A25AB64F8D91C4
:10EF20009C91BC01660F771F680F791F6C0F7D1FC6
:10EF300077FF02C06D5F7F4F7B01F594E794F594F6
:10EF4000E794CE0101968E159F0524F40894E108FC
:10EF5000F10808C0CE010197E816F9061CF40894E0
:10EF6000E11CF11C0630110509F0ABC0C536D10516
:10EF70000CF482C090912905E92FFF27EF52F54F3D
:10EF8000E081ED3729F4809128058095809328054C
:10EF9000993009F06DC080912805882319F4E33871
:10EFA00021F066C0ED3709F063C08091D20A8D3739
:10EFB00039F48091D30A833899F463E87FEF0DC068
:10EFC000833871F48091D30A833819F460E070E0DB
:10EFD00004C08D3729F46DE770E085E00E94137658
:10EFE0008091D40A8D3739F48091D70A833899F407
:10EFF0006DE770E00DC0833871F48091D70A8338D3
:10F0000019F460E070E004C08D3729F463E87FEF05
:10F0100086E00E9413768091D80A8D3739F480916A
:10F02000D90A833899F463E87FEF0DC0833871F40F
:10F030008091D90A833819F460E070E004C08D37FC
:10F0400029F46DE770E089E00E9413768091D60A7A
:10F05000992787FD9095BC018AE00E9413768091E4
:10F06000D50A992787FD9095BC018CE00E94137604
:10F070001092290510922805CA30D1055CF48091C0
:10F0800029058F5F80932905E82FFF27EF52F54F61
:10F0900083E88083809129058A3011F41092290534
:10F0A0003FEFCC39D3076CF480912905E82FFF2777
:10F0B000EF52F54F8DE780838091280580958093EE
:10F0C00028050530110518F4B701802F11C007304D
:10F0D000110519F4BE0187E00BC00530110519F4C4
:10F0E000BE0188E005C008301105B1F4BE018BE017
:10F0F0000E94137611C00231110570F081E08093F7
:10F10000A3010AC081E08093A30110922C05109204
:10F110002E0584E480932A0580912C05803198F097
:10F1200080912E05882331F48091A301882311F466
:10F1300080933A0110922C0510922E0510922B0507
:10F1400084E480932A05E6E0CDB7DEB70C947D9A7F
:10F15000CF93FC0197FF05C0CFEFF095E195FF4FEE
:10F1600001C0C1E028E631E0CF01B9010E94059A53
:10F17000FC018B35910554F08B5590408A359105F3
:10F1800038F484EB90E08E1B9F0BFC0141E00DC036
:10F19000CF01855B90408A35910518F4E45BF0401F
:10F1A00003C02E1B3F0BF9014FEFEE0FFF1FEC5971
:10F1B000F64F259134918C2F992787FD9095289FA4
:10F1C000B001299F700D389F700D1124842F99274D
:10F1D00087FD9095689FA001699F500D789F500D05
:10F1E0001124CA01CF9108952AE530E0281B390B7C
:10F1F000C9010E94A8780895089508950895089572
:10F20000089580E090E008951092DD0A1092DC0AE3
:10F210001092E10A1092E00A1092DF0A1092DE0AC0
:10F220001092E20A8AE090E00E94BE1990933005A5
:10F2300080932F050895CF93DF9380912F059091B0
:10F2400030050E94C719882309F4AFC080912F05AB
:10F25000909130050A969093300580932F05E0E059
:10F26000F0E09F0190E05FEFADEFB8E04BE0ED0123
:10F270008B8187FF0BC09F5F8D81E80FF11D898116
:10F28000280F311D8E81851708F4582F415018968C
:10F2900047FFEDCF5093E20A232B41F5209135052E
:10F2A000309136054091370550913805BB27A52F81
:10F2B000942F832F9093340580933305AA27BB277F
:10F2C000281B390B4A0B5B0BCF01AA27BB27280F42
:10F2D000391F4A1F5B1F2093350530933605409335
:10F2E000370550933805E5E0F0E013C02091330571
:10F2F000309134052E173F0718F4E21BF30B02C0C0
:10F30000E0E0F0E0892F9927880F991FE80FF91F97
:10F310003596F093DD0AE093DC0AEF3FF10578F4CF
:10F3200080912001909121018E9F90018F9F300D3F
:10F330009E9F300D1124C90164E670E013C0CF0117
:10F34000969587959695879520912001309121017A
:10F35000289FA001299F500D389F500D1124CA01EC
:10F3600069E170E00E94F1997093DF0A6093DE0A10
:10F3700020913105309132052E0F3F1F3093320519
:10F38000209331055EE02131350778F08091E00A65
:10F390009091E10A01969093E10A8093E00A20514E
:10F3A0003E403093320520933105DF91CF9108958F
:10F3B00030914505E32FFF2783E0EE0FFF1F8A956D
:10F3C000E1F7E350F74F2781422F552747FD50952E
:10F3D000809146059927841795072CF420934605BC
:10F3E000309348050AC0222341F0809147059927B0
:10F3F0004817590714F420934705832F8F5F809394
:10F4000045058D30D0F010924505809147058F3F1E
:10F4100019F080933A0502C010923A058091460592
:10F4200080933B0580914805809339058FEF809349
:10F4300047051092460510924805089595E1899F69
:10F44000802D11240E94CF928DEA9CE09F938F9390
:10F4500081EA92E99F938F93E0918405F09185056D
:10F4600009950F900F900F900F900895CF93C0E0E3
:10F470002091A40120933F058091FF0385FF02C0E6
:10F48000C0E123C0909116059923B1F08091370413
:10F49000882349F4E92FFF27EE0FFF1FE55EF54FA4
:10F4A0008491882349F4E92FFF27EE0FFF1FE65EC2
:10F4B000F54FC491CC2349F48091990886FD03C08F
:10F4C0001092A40104C0C22F02C0C0933F058091D6
:10F4D00049058C1771F480914A0590914B050E9463
:10F4E000C719882319F480E090E017C088E893E1F9
:10F4F00002C080ED97E00E94BE1990934B05809367
:10F500004A05CC2331F08091A401C81711F4109260
:10F51000A401C09349058C2F9927CF91089540E00D
:10F5200050E030E08091AA0A99278A38910589F045
:10F530008B38910524F48938910541F013C08D383A
:10F54000910569F08E38910539F00CC04BE35BE012
:10F5500008C043E15CE005C043EE5AE002C04FE062
:10F560005BE03CE290919F0A20E08091A00A28177E
:10F5700070F4931760F4DA01A90FB11DE22FFF2791
:10F58000E457F54F85898C939F5F2F5FEECF0895E9
:10F5900020E335E780913B018B3211F08D32F9F495
:10F5A00080913A08282F332780912C0490912D04C4
:10F5B000829FA001839F500D929F500D1124CA017C
:10F5C00063E070E00E94059ACB019B01205D3A4800
:10F5D000C196C19708F03FC02EEF34E73CC080329F
:10F5E00029F58091FF0381FF36C020913C053091C1
:10F5F0003D05205D3A4855E72133350748F085E75A
:10F600002439380718F420E335E702C02456304087
:10F6100045E720333407F8F454E72D3C350718F05C
:10F6200020E335E718C02C593F4F15C08E3549F4FB
:10F63000909127048AE0989F90011124205D3A4818
:10F640000AC0863741F4909127048AE0989FC00150
:10F650001124281B390BC9010895EF92FF920F93D3
:10F660001F9399278A38910509F494C18B38910525
:10F6700024F48938910551F03FC38D38910509F480
:10F680007EC28E38910509F4D9C136C30E94367AFC
:10F69000182F8093150C8091320490913304A0911F
:10F6A0003404B0913504BC01CD0124E630E040E0E3
:10F6B00050E00E943A9ADA01C9018C509E4F909313
:10F6C000410B8093400B112319F40E94C87A02C0A9
:10F6D00080E395E79093470B8093460B8091460B10
:10F6E0009091470B9093490B8093480B90934B0B51
:10F6F00080934A0B2091400B3091410B8091440B39
:10F700009091450B2817390724F43093450B20932B
:10F71000440B8091420B9091430B8217930724F482
:10F720003093430B2093420B10923D0B8BE39BE0F5
:10F7300090935C0580935B0580913B018093610B06
:10F740008091FE0380FF02C083E401C080E28093C9
:10F75000620B20911605222309F1822F6AE00E9494
:10F76000E599805D80934C0B822F0E94E599892F4B
:10F77000805D80934D0B8AE380934E0B81E1289F3F
:10F78000F0011124AFE4BBE0E65AF54F9FE084910D
:10F790008D939150319697FFFACFABC28091FF03C2
:10F7A00085FF0CC0ACE4BBE0E1E8FCE094E18491AF
:10F7B0008D939150319697FFFACF9BC280913E0571
:10F7C000882301F1ACE4BBE0EAE7FCE096E0849139
:10F7D0008D939150319697FFFACF80910001805D13
:10F7E0008093500BA3E5BBE0EAE9F8E09BE0819150
:10F7F0008D93915097FFFBCF80E280935E0B8093B7
:10F800005F0BB9C030914305332309F499C087E5F4
:10F8100080934C0B80E580934D0B40E240934E0B60
:10F8200020914405822F6AE00E94E599805D8093D3
:10F830004F0B822F0E94E599892F805D8093500B9A
:10F840008FE28093510B832F0E94E599805D809316
:10F85000520B832F0E94E599892F805D8093530B73
:10F860004093540B209140053091410583E0293E9F
:10F87000380780F0C90168EE73E00E94F199CB016E
:10F88000805D8093550BC90168EE73E00E94F19989
:10F890009C0102C04093550B2536310580F0C9010B
:10F8A00064E670E00E94F199CB01805D8093560B75
:10F8B000C90164E670E00E94F1999C0103C080E2F6
:10F8C0008093560BC9016AE070E00E94F199CB0168
:10F8D000805D8093570BC9016AE070E00E94F19946
:10F8E000805D8093580B8DE68093590B80E2809366
:10F8F0005A0B20914205253660F0822F64E60E9463
:10F90000E599805D80935B0B822F0E94E599292FFA
:10F9100002C080935B0B822F6AE00E94E599805DB4
:10F9200080935C0B822F0E94E599892F805D8093E4
:10F930005D0B83E780935E0B80E280935F0BD9C100
:10F94000809123048823D1F4ACE4BBE0E9E9FCE036
:10F9500090E184918D939150319697FFFACF82E395
:10F9600080935C0B8EE280935D0B80E380935E0B53
:10F9700080935F0B81E68093600BBBC1ACE4BBE07E
:10F98000E7E9FCE094E184918D939150319697FFE3
:10F99000FACFAFC18091320490913304A091340426
:10F9A000B0913504BC01CD0124E630E040E050E0E8
:10F9B0000E943A9ADA01C9018C509E4F9093290C0B
:10F9C0008093280C8091150C882319F40E94C87A22
:10F9D00002C080E395E790932B0C80932A0C88E774
:10F9E00080932C0C8091580A80932D0C8091570A9B
:10F9F00081FF02C084E407C08091590A833011F46A
:10FA000080E201C081E280932E0C83E19CE0909320
:10FA10005C0580935B058091900180933A0C809106
:10FA20002E0C80933C0C80915D0A90915E0A97FDAC
:10FA300001969595879580932F0C5BC10E94D8798C
:10FA40008091320490913304A0913404B091350434
:10FA5000BC01CD0124E630E040E050E00E943A9A3B
:10FA6000DA01C9018C509E4F9093FE0A8093FD0AE3
:10FA700080912001909121019093F80A8093F70AD8
:10FA800080912001909121019093FA0A8093F90AC4
:10FA90008091F8099091F90997FD019695958795C0
:10FAA0008093E90A8093F00A20915D0A30915E0A02
:10FAB00037FF02C02F5F3F4F359527952093EE0A01
:10FAC00080915B0A90915C0A64E170E00E94F19978
:10FAD0006093EF0A2093F50A6093F60A8091150C63
:10FAE000882319F40E94C87A02C080E395E79093B6
:10FAF000060B8093050B88E78093070B809120010C
:10FB0000909121019093020B8093010B80913A0513
:10FB10008C5E8093FB0A80913B058C5E8093FC0A8F
:10FB20008091E00A9091E10A6AE070E00E94F19908
:10FB30007093040B6093030B1092E50A8091DC0A2A
:10FB40009091DD0A9093000B8093FF0A83EE9AE078
:10FB500090935C0580935B052091DE023091DF027B
:10FB6000C9016CE370E00E94F19960930A0BC9012E
:10FB70006CE370E00E94F19980930B0BBAC00E9475
:10FB8000D87980915B0A90915C0A64E670E00E94EB
:10FB9000F1997093250B6093240B8091F809909153
:10FBA000F90997FD0196959587958093150B80919E
:10FBB0005D0A90915E0A97FD0196959587958093D1
:10FBC0001A0B80910101482F55279A012B5F3F4F57
:10FBD00080912001909121012817390784F48091A8
:10FBE000200190912101841B950B9C01220F331F52
:10FBF000280F391F822F82518093210B02C010924F
:10FC0000210BE0903204F090330400913404109101
:10FC10003504C801B70124E630E040E050E00E941E
:10FC20003A9A3093230B2093220B37FF04C0109293
:10FC3000230B1092220BC801B70124E630E040E00C
:10FC400050E00E943A9ADA01C9018C509E4F90937D
:10FC5000270B8093260B8091200190912101909396
:10FC60001C0B80931B0B809120019091210190939C
:10FC70001E0B80931D0B8091150C882319F40E9494
:10FC8000C87A02C080E395E79093290B8093280BF4
:10FC900088E780932A0B8091200190912101909315
:10FCA0002E0B80932D0B80913A058C5E80931F0B59
:10FCB00080913B058C5E8093200B8091E00A9091AF
:10FCC000E10A6AE070E00E94F1997093300B609352
:10FCD0002F0B1092110B8091DC0A9091DD0A90930A
:10FCE0002C0B80932B0B8FE09BE090935C05809313
:10FCF0005B052CE230E002C020E030E0C9011F913A
:10FD00000F91FF90EF900895EF92FF920F931F9342
:10FD1000CF93DF9380913C0590913D059C0153E08A
:10FD2000220F331F5A95E1F7281B390B80912303CB
:10FD300090912403280F391F37FF02C0295F3F4FDE
:10FD400043E0359527954A95E1F730933D0520939B
:10FD50003C0590914D05992309F026C380914C05EF
:10FD6000282F3327442755278F5F80934C05F901AF
:10FD70002131310508F015C3E857FF4F0C948C9AD8
:10FD80008091FF0385FF2AC080E00E94CF9280917E
:10FD90002001909121016AE070E00E94059A9F93F2
:10FDA0008F9380912001909121016AE070E00E9480
:10FDB000059A7F936F9383EC9CE09F938F9382ECE3
:10FDC00092E99F938F93E0918405F09185050995C1
:10FDD0002DB73EB7285F3F4F2DBF28C080E00E945F
:10FDE000CF9280912001909121016AE070E00E9401
:10FDF000059A9F938F9380912001909121016AE051
:10FE000070E00E94059A7F936F9380ED9CE09F9332
:10FE10008F9381EA92E99F938F93E0918405F0910B
:10FE2000850509958DB79EB708968DBF80913C0AD0
:10FE300080FF3FC080914F048823E9F08AE00E9450
:10FE4000CF9280913B0199279F938F9380913204A9
:10FE500090913304A0913404B0913504BC01CD01DC
:10FE600024E630E040E050E00E943A9A3F932F931E
:10FE70008DED9CE09BC68AE00E94CF928091320477
:10FE800090913304A0913404B0913504BC01CD01AC
:10FE900024E630E040E050E00E943A9A3F932F93EE
:10FEA00089EE9CE09F938F9381EA92E99F938F93D1
:10FEB000A4C78AE00E94CF9284EF9CE09F938F9327
:10FEC00081EA92E90C9428888091FF0385FF2AC07B
:10FED00085E10E94CF928091DE029091DF026CE377
:10FEE00070E00E94F1999F938F938091DE02909130
:10FEF000DF026CE370E00E94F1997F936F938EEFC5
:10FF00009CE09F938F9382EC92E99F938F93E09173
:10FF10008405F091850509952DB73EB7285F3F4FC1
:10FF20002DBF28C085E10E94CF928091DE02909182
:10FF3000DF026CE370E00E94F1999F938F938091B0
:10FF4000DE029091DF026CE370E00E94F1997F93F2
:10FF50006F938BE09DE09F938F9381EA92E99F934B
:10FF60008F93E0918405F091850509958DB79EB733
:10FF700008968DBF8FE10E94CF9280E690E09F931C
:10FF80008F938091F8099091F9099F938F9388E15D
:10FF90009DE09F938F93C1EAD2E9DF93CF93E091E5
:10FFA0008405F091850509958091FE032DB73EB734
:10FFB000285F3F4F2DBF80FF06C089E20E94CF928D
:10FFC00083E29DE06FC389E20E94CF9285E29DE0CB
:10FFD000B5C68091FF0385FF1BC08AE20E94CF92C5
:10FFE0008091E00A9091E10A9F938F9387E29DE0D0
:10FFF0009F938F9382EC92E99F938F93E091840576
:020000021000EC
:10000000F091850509958DB79EB706968DBF1BC0EB
:100010008AE20E94CF928091E00A9091E10A9F9338
:100020008F938FE29DE09F938F9381EA92E99F9354
:100030008F93E0918405F091850509952DB73EB722
:100040002A5F3F4F2DBF86E30E94CF928091DC0A4A
:100050009091DD0A6AE070E00E94F1999F938F937E
:100060008091DC0A9091DD0A6AE070E00E94F199CB
:100070007F936F9387E39DE09F938F9381EA92E94B
:100080009F938F93E0918405F091850509958DB735
:100090009EB70896BAC689E00E94CF9283E49DE09D
:1000A0009F938F9301EA12E91F930F93E0918405C8
:1000B000F091850509958EE10E94CF920F900F90E7
:1000C0000F900F9085E49DE09F938F931F930F9364
:1000D000E0918405F0918505099583E30E94CF9214
:1000E0000F900F900F900F9087E49DE09F938F9358
:1000F0001F930F93E0918405F091850509958FE397
:100100000E94CF920F900F900F900F9089E49DE086
:100110009F938F931F930F93E0918405F091850532
:1001200009958EE70E94CF920F900F900F900F903D
:100130008FE59DE09F938F931F930F938BC78091C3
:100140009E01882309F462C08DE50E94CF9285E765
:100150009DE09F938F93C1EAD2E9DF93CF93E09123
:100160008405F0918505099584E50E94CF920F9052
:100170000F900F900F908091580A99279F938F931B
:1001800087E79DE09F938F93DF93CF93E091840562
:10019000F091850509958EE50E94CF922DB73EB767
:1001A0002A5F3F4F2DBF80915B0A90915C0A6AE005
:1001B00070E00E94F1997F936F9380E89DE09F9398
:1001C0008F93DF93CF93E0918405F0918505099596
:1001D0008DB79EB706968DBF8091590A833081F402
:1001E0008091570A81FF06C08BE50E94CF928AE872
:1001F0009DE0A4C58BE50E94CF928DE89DE09EC551
:100200008BE50E94CF9280E99DE01EC784E0CFC3BA
:1002100080919E01882309F47AC080914F0591EA6C
:10022000E92E92E9F92E882309F44BC089E60E9451
:10023000CF928091150599279F938F9383E99DE035
:100240009F938F93FF92EF92E0918405F091850543
:10025000099585E70E94CF922DB73EB72A5F3F4FA1
:100260002DBF8091900199279F938F9300E610E016
:100270001F930F9380915D0A90915E0A9F938F93D5
:100280008EE99DE09F938F93FF92EF92E09184051A
:10029000F0918505099582E70E94CF928DB79EB7B0
:1002A0000A968DBF8091130599279F938F931F9373
:1002B0000F938091140599279F938F938AEA9DE06D
:1002C00064C689E60E94CF928091900199279F93FE
:1002D0008F9380E690E09F938F9380915D0A909139
:1002E0005E0A9F938F9380915A0A99279F938F93C9
:1002F0008AEB9DE09F938F93FF92EF92E0918405AC
:10030000F091850509958DB79EB70C967EC585E061
:100310004EC3909116059923D1F0809158058823FA
:1003200081F0903270F487E00E941E7A83E90E9487
:10033000CF928091160599279F938F9383ED9DE02F
:10034000A0C383E90E94CF928EED9DE0AFC3809160
:10035000FF0301EAE02E02E9F02E85FF06C084E9E2
:100360000E94CF9284EE9DE0D6C383E90E94CF9293
:1003700087EF9DE0D0C38091780C863059F480914E
:100380004F05882319F010924F058BC681E08093AA
:100390004F0587C6883009F084C60E94D49281E058
:1003A000D7C390934C0585C6913009F0DCC380918A
:1003B0004C05282F3327442755278F5F80934C0502
:1003C000F9012131310508F06FC6E756FF4F0C9453
:1003D0008C9A8091FF0385FF43C080E00E94CF92FA
:1003E0008091E00A9091E10A9F938F938091200180
:1003F000909121016AE070E00E94059A9F938F938B
:1004000080912001909121016AE070E00E94059A9C
:100410007F936F938091DE029091DF026CE370E036
:100420000E94F1999F938F938091DE029091DF0259
:100430006CE370E00E94F1997F936F938DE09EE0F2
:100440009F938F9382EC92E99F938F93E091840521
:10045000F091850509952DB73EB7225F3F4FA2C5A4
:1004600080E00E94CF928091E00A9091E10A9F93F0
:100470008F9380912001909121016AE070E00E94A9
:10048000059A9F938F9380912001909121016AE0BA
:1004900070E00E94059A7F936F938091DE029091A5
:1004A000DF026CE370E00E94F1999F938F9380913B
:1004B000DE029091DF026CE370E00E94F1997F937D
:1004C0006F9388E29EE0BEC285E10E94CF9280E6F3
:1004D00090E09F938F9380918A0190918B019F93DD
:1004E0008F9383E49EE09F938F93C1EAD2E9DF93D9
:1004F000CF93E0918405F0918505099580913C0AA0
:100500002DB73EB7285F3F4F2DBF80FF51C0809170
:100510004F04882339F18FE10E94CF9280913204F9
:1005200090913304A0913404B0913504BC01CD0105
:1005300024E630E040E050E00E943A9A3F932F9347
:100540008DE49EE09F938F9381EB92E99F938F932D
:10055000E0918405F091850509958DB79EB70696C3
:100560008DBF38C08FE10E94CF928091320490916C
:100570003304A0913404B0913504BC01CD0124E6CC
:1005800030E040E050E00E943A9A3F932F9386E596
:100590009EE09F938F93DF93CF93E0918405F0913A
:1005A000850509952DB73EB72A5F3F4F2DBF12C075
:1005B0008FE10E94CF928FE59EE09F938F93DF9310
:1005C000CF93E0918405F091850509950F900F90E8
:1005D0000F900F9089E20E94CF9280913B01992762
:1005E0009F938F9389E69EE004C480919E018823A7
:1005F000F9F08BE20E94CF928091900199279F930E
:100600008F9380915B0A90915C0A6AE070E00E948F
:10061000F1997F936F9380E690E09F938F93809101
:100620005D0A90915E0A9F938F938CE69EE058C17D
:1006300082E0BDC18FE30E94CF928091DE0A90914B
:10064000DF0A9F938F938091DC0A9091DD0A6AE024
:1006500070E00E94F1999F938F938091DC0A9091B2
:10066000DD0A6AE070E00E94F1997F936F9383E85E
:100670009EE09F938F93C1EAD2E9DF93CF93E091FD
:100680008405F091850509958091FE032DB73EB74D
:10069000265F3F4F2DBF80FF0AC082E50E94CF92A8
:1006A00087E99EE09F938F9381EB92E9D1C482E525
:1006B0000E94CF928AE99EE041C380919E0111EA97
:1006C000E12E12E9F12E882309F449C084E50E9445
:1006D000CF928091580A99279F938F9380915A0ABD
:1006E00099279F938F938DE99EE09F938F93E701C6
:1006F000FF92EF92E0918405F091850509958DB701
:100700009EB708968DBF8091590A833051F484E6D4
:100710000E94CF9280EB9EE09F938F93FF92EF9287
:100720000BC084E60E94CF9286EB9EE09F938F934E
:1007300082EC92E99F938F93E0918405F091850577
:1007400009950F900F900F900F908091570A81FF9D
:10075000B0C484E60E94CF928CEB9EE0EFC284E5A9
:100760000E94CF9282EC9EE0D6C180914E05C1EAF4
:10077000EC2EC2E9FC2E882309F450C089E60E94C1
:10078000CF9280911A096AE00E94E599892F9927F2
:100790009F938F9380911A090E94E59999279F93BF
:1007A0008F93809112090E94E599892F99279F9331
:1007B0008F93809112090E94E59999279F938F93B7
:1007C00080910A090E94E599892F99279F938F9319
:1007D00080910A090E94E59999279F938F938091B0
:1007E00002090E94E599892F99279F938F93809101
:1007F00002090E94E59999279F938F9388ED9EE0C7
:100800009F938F93FF92EF92E0918405F09185057D
:1008100009952DB73EB72C5E3F4FC4C389E60E94B1
:10082000CF9280E690E09F938F9380911C09992747
:1008300087FD90959F938F9380911409992787FD49
:1008400090959F938F9380910C09992787FD9095A0
:100850009F938F9380910409992787FD90959F938B
:100860008F9385EF9EE09F938F93FF92EF92E0919D
:100870008405F091850509958DB79EB70E96C5C282
:1008800080914E0590912708882309F48DC09430FB
:1008900009F48CC09630A1F58EE70E94CF9280912A
:1008A0002A096AE00E94E599892F99279F938F93DF
:1008B00080912A090E94E59999279F938F938091AF
:1008C00022090E94E599892F99279F938F93809100
:1008D00022090E94E59999279F938F9388E09FE0D2
:1008E0009F938F9381EA92E99F938F93E091840580
:1008F000F091850509952DB73EB7245F3F4F52C350
:10090000973008F4D6C38EE70E94CF9280913A09BF
:100910006AE00E94E599892F99279F938F93809190
:100920003A090E94E59999279F938F938091320904
:100930000E94E599892F99279F938F93809132097F
:100940000E94E59999279F938F9380912A090E948D
:10095000E599892F99279F938F9380912A090E9467
:10096000E59999279F938F93809122090E94E59999
:10097000892F99279F938F93809122090E94E5994F
:1009800099279F938F9387E19FE09F938F9381EAAD
:1009900092E99F938F93E0918405F09185050995E5
:1009A0008DB79EB7449631C2943021F486E00E9400
:1009B0001E7A7FC39630F1F48EE70E94CF9280E6D4
:1009C00090E09F938F9380912C09992787FD9095B4
:1009D0009F938F9380912409992787FD90959F93EA
:1009E0008F9384E39FE09F938F9381EA92E99F9393
:1009F0008F93CFC2973008F45CC38EE70E94CF92EA
:100A000080E690E09F938F9380913C09992787FD22
:100A100090959F938F9380913409992787FD9095A6
:100A20009F938F9380912C09992787FD90959F9391
:100A30008F9380912409992787FD90959F938F9399
:100A400087E49FE09F938F9381EA92E99F938F932E
:100A50000ECF90911605992309F44AC0809158054C
:100A60008823F9F09032E8F487E00E941E7A83E947
:100A70000E94CF928091160599279F938F938AE5C4
:100A80009FE09F938F9381EB92E99F938F93E091E7
:100A90008405F091850509952DB73EB72A5F3F4F34
:100AA00081C283E90E94CF9285E69FE09F938F9356
:100AB00001EA12E91F930F93E0918405F0918505F7
:100AC00009951F921F929091160581E1989FC00190
:100AD0001124865A954F9F938F931F930F93E09104
:100AE0008405F091850509958DB79EB70A968DC14D
:100AF0008091FF03B1EAEB2EB2E9FB2E85FF06C021
:100B000084E90E94CF928BE69FE005C083E90E94B2
:100B1000CF928EE79FE09F938F93FF92EF929AC2BE
:100B20008091780C863079F480914E05882319F0F5
:100B300010924E0503C081E080934E0585E00E942F
:100B40001E7A86E0A3C2883031F40E94D49282E0FB
:100B500080934D05A4C2813009F0A3C20E94D492B3
:100B600010924D059CC2923009F0A1C280914C05B3
:100B7000282F3327442755278F5F80934C05F90191
:100B80002131310508F090C2E655FF4F0C948C9A44
:100B900080E00E94CF928AE998E09F938F938091A2
:100BA000000199279F938F9384E99FE09F938F93F0
:100BB00081EB92E99F938F93E0918405F0918505F5
:100BC00009952DB73EB7285F3F4FECC185E10E94E4
:100BD000CF9288EA98E09F938F93809101016AE019
:100BE0000E94E599892F99279F938F938091010106
:100BF0000E94E59999279F938F9383EA9FE09F93A3
:100C00008F9381EA92E99F938F93E0918405F0910D
:100C10008505099569CF8AE20E94CF9284EB9FE017
:100C20009F938F93C1EAD2E9DF93CF93E09184053C
:100C3000F0918505099580913C0A0F900F900F90D7
:100C40000F9080FF41C0809135089091150481FD7F
:100C50000BC0892F99279F938F9389EB9FE09F93D8
:100C60008F93DF93CF9313CFE0918405F0918505A7
:100C7000933318F083EC9FE002C08AEC9FE09F93CF
:100C80008F93DF93CF9309950F900F900F900F9054
:100C900080911F0AE0918405F091850590911504DB
:100CA00080FF0BC0892F99279F938F9381ED9FE041
:100CB0009F938F93DF93CF93A4C0892F99279F93FE
:100CC0008F9387ED9FE0C4C08DED9FE037C08FE329
:100CD0000E94CF9286EE9FE09F938F93C1EAD2E964
:100CE000DF93CF93E0918405F091850509950F90EE
:100CF0000F900F900F9080918B08882319F48AEE43
:100D00009FE01CC080910C04E0918405F091850562
:100D1000882319F083EF9FE002C08AEF9FE09F9342
:100D20008F93DF93CF9309950F900F900F900F90B3
:100D30008091980886FFBDC181E090E19F938F93D9
:100D4000DF93CF9387C184E50E94CF9288E090E142
:100D50009F938F93C1EAD2E9DF93CF93E09184050B
:100D6000F0918505099580913C0A0F900F900F90A6
:100D70000F9085FD03C08DE090E108C08091790857
:100D80000E94C647823358F486E190E19F938F9387
:100D9000DF93CF93E0918405F091850516C0843BE5
:100DA00018F08DE190E1F2CF80919808E0918405F0
:100DB000F091850585FF03C084E290E102C08BE2DB
:100DC00090E19F938F93DF93CF9309950F900F90AE
:100DD0000F900F9080918F08882309F46AC18EE5E7
:100DE0000E94CF9280918F0899279F938F9382E3DF
:100DF00090E19F938F93DF93CF93E0918405F091DF
:100E0000850509958DB79EB706968DBF52C189E6B7
:100E10000E94CF928DE390E19F938F93C1EAD2E934
:100E2000DF93CF93E0918405F091850509950F90AC
:100E30000F900F900F9080918E08E0918405F091B3
:100E40008505882351F099279F938F9387E490E13C
:100E50009F938F93DF93CF931ECE8BE490E19F936C
:100E60008F93DF93CF93FAC080915005A1EAEA2EC9
:100E7000A2E9FA2E882309F053C08EE70E94CF9290
:100E80008091690199279F938F9380912A08E82F79
:100E9000FF27EE0FFF1FE25AF64F808191819F934B
:100EA0008F9380912908E82FFF27EE0FFF1FE25A4A
:100EB000F64F808191819F938F9381E590E19F937D
:100EC0008F93FF92EF92E0918405F091850509954B
:100ED00083E90E94CF928DB79EB70A968DBF80910D
:100EE0002C08E82FFF27EE0FFF1FE25AF64F8081F4
:100EF00091819F938F9380912B08E82FFF27EE0F0E
:100F0000FF1FE25AF64F8081918181589F4F9F9336
:100F10008F9385E690E19F938F93FF92EF924CCE53
:100F20008EE70E94CF9280913B0499279F938F93E5
:100F300080913A0499279F938F9380913904992740
:100F40009F938F9384E790E19F938F93FF92EF920B
:100F5000E0918405F0918505099583E90E94CF927F
:100F60008DB79EB70A968DBF80913E0499279F93B7
:100F70008F9380913D0499279F938F9380913C0498
:100F800099279F938F9388E890E19F938F93FF9287
:100F9000EF92E0918405F091850509952DB73EB754
:100FA000265F3F4F2DBF85C080915805882309F4E7
:100FB00080C08EE70E94CF9280913C0A86FD11C0CE
:100FC0008CE990E19F938F9382EC92E99F938F93AA
:100FD000E0918405F091850509950F900F900F9091
:100FE0000F908091960899278F709070892B89F0C7
:100FF0008BEA90E19F938F9382EC92E99F938F937A
:10100000E0918405F091850509950F900F900F9060
:101010000F9080913C0A82FF11C085EB90E19F9375
:101020008F9382EC92E99F938F93E0918405F091E6
:10103000850509950F900F900F900F9080913C0AB5
:1010400083FD37C08AEB90E19F938F9382EC92E906
:101050009F938F93E0918405F091850509950F90FA
:101060000F900F900F9025C00091780C063089F4F6
:1010700080915005882319F01092500503C081E03B
:101080008093500586E00E941E7A87E00E941E7AB7
:1010900008C0013031F40E94D49200934D051092A3
:1010A0004C051092780C05C010924C0502C01092AD
:1010B0004D05E6E0CDB7DEB70C947D9A4FB728E139
:1010C00030E0F8948091C9008F778093C9008091B7
:1010D000C9008F7B8093C9008091C9008F7D809368
:1010E000C900832F99278093CD002093CC00809155
:1010F000C80082608093C80080E18093C90080911D
:10110000CA008F778093CA008091CA008F7B80933A
:10111000CA008091CA008091CA008F7E8093CA0065
:101120008091CA0088608093CA008091C9008B7F3B
:101130008093C9008091CA0084608093CA00809126
:10114000CA0082608093CA008091C80087FF03C0F4
:101150008091CE00F9CF8091C90080688093C9004A
:101160008091560C84608093560C4FBF08959091E7
:101170002A05992341F48F3031F49093520580E58C
:1011800080932A050895E0915205EF5FE0935205A0
:10119000E83121F481E0809351050895E93120F090
:1011A00089E1809352050895FF27E15CF34F808326
:1011B0000895A0E0B0E0EFEDF8E80C945D9A91E0BE
:1011C000D92E82E0A82EBD2CE12C01E0F02E8091DA
:1011D000560C82FDB5C080916F008F7D80936F00AB
:1011E000E0919108EE2351F0FF27EE0FFF1FE25A26
:1011F000F64F80819181843691055CF480913804AA
:10120000883C20F4809138048C5E01C088EC809387
:1012100038048091400C682F7727809153058150C6
:10122000809353058F3F31F41CE7C12E82E08093F9
:10123000530502C0C4E2CC2E40E04C1508F07EC03D
:10124000EA2DFF27E15CF34F80818D2111F06E299B
:101250007F298D2D9927880F991FD82E882319F45F
:10126000B1E0DB2EAD0CEE0CFF1C20E0E21628E016
:10127000F20609F061C0A1E0EA2EF12CCB0180500A
:10128000944065E070E00E94059AAB2DBB27FD01FC
:10129000EA0FFB1FE25AF64F808191819C01220FD9
:1012A000331F280F391F260F371F37FF02C02D5F4E
:1012B0003F4FE901D595C795D595C795CB010196C7
:1012C0008C179D0714F4219706C061507040C61713
:1012D000D7070CF4219680913804833CD8F08D0117
:1012E0000A0F1B1FF801E25AF64F80819181FE011F
:1012F000E81BF90BCF0163E070E00E94059ACB0177
:10130000880F991F860F971F0C55164FF801918370
:10131000808307C0AA0FBB1FAC55B64F11961C9215
:101320001E92EB2DFF27EE0FFF1FE25AF64FD183DF
:10133000C08360E070E0B3944F5F7FCF10923A01BA
:1013400010925105EAE0CDB7DEB70C94799A089572
:10135000089540E050E080915405909155059C011E
:10136000220F331F280F391F8091230390912403EC
:10137000280F391F37FF02C02D5F3F4F3595279546
:1013800035952795309355052093540580913B0161
:101390008B32D9F480913A08282F332780912C047E
:1013A00090912D04829FA001839F500D929F500D1C
:1013B0001124CA0157FD4F96AC0125E0559547957C
:1013C0002A95E1F74B5F5F4F3DC08D32D9F4809194
:1013D0003A08282F332780912C0490912D04829F66
:1013E000A001839F500D929F500D1124CA0157FDFB
:1013F0004F96AC0195E0559547959A95E1F7455084
:10140000504020C0803271F48091FF0381FF1AC0E8
:10141000C90137FD4F96AC0185E0559547958A95F2
:10142000E1F710C08E3529F480912704482F552705
:1014300009C0863739F48091270499274427552716
:10144000481B590BCA01AA2797FDA095BA2F809374
:10145000970290939802A0939902B0939A020895EC
:101460000F931F930E94D8798091200190912101C0
:10147000AA2797FDA095BA2F8093C6019093C70124
:10148000A093C801B093C9018091DC0A9091DD0A54
:10149000AA27BB278093D9019093DA01A093DB019F
:1014A000B093DC010AE010E08091E00A9091E10A3B
:1014B000B8010E94F199CB01AA27BB278093EC01C8
:1014C0009093ED01A093EE01B093EF01809132046F
:1014D00090913304A0913404B0913504BC01CD0146
:1014E00024E630E040E050E00E943A9A2093FF0169
:1014F00030930002409301025093020280918A01CE
:1015000090918B01AA2797FDA095BA2F8093120284
:1015100090931302A0931402B09315028091580A7D
:101520009927AA27BB278093250290932602A09390
:101530002702B093280280915A0A9927AA27BB272D
:101540008093380290933902A0933A02B0933B0201
:1015500080915B0A90915C0AB8010E94F199CB01DD
:10156000AA27BB2780934B0290934C02A0934D0275
:10157000B0934E0280915D0A90915E0AAA2797FD72
:10158000A095BA2F80935E0290935F02A0936002B1
:10159000B093610280913B059927AA27BB278093CE
:1015A000710290937202A0937302B09374028091BF
:1015B00015059927AA27BB2780938402909385025B
:1015C000A0938602B0938702809116059927AA27D7
:1015D000BB278093AA029093AB02A093AC02B09376
:1015E000AD021F910F91089500242227332744272D
:1015F00051E0BB27EE27FF27A0E1660F771F881F6A
:10160000991F001C221F331F441F660F771F881F5E
:10161000991F001C221F331F441F2AF4050E2B1F85
:101620003E1F4F1F04C0051A2B0B3E0B4F0B550FCF
:10163000BB1FEE1F587F556047FD5250AA95E9F633
:10164000E695B7955795E695B7955795852F9B2FB6
:1016500008952227332741E0552768E0880F991F16
:10166000221F331F880F991F221F331F1AF4240FC4
:10167000351F02C0241B350B440F551F487F4560A2
:1016800037FD42506A9551F75695479556954795BF
:10169000842F0895AA2797FF04C0809590958A1FEC
:1016A0009A1F77FF04C0609570956A1F7A1F669F26
:1016B0009001779FA001679F300D411D5A1F300D8B
:1016C000411D5A1F889FF001999F2E0F3F1F401DFB
:1016D000511D899F300D411D5A1F300D411D5A1F4C
:1016E000CA01B901112480CF4FB720E430E0F8944B
:1016F0008091C9008F778093C9008091C9008F7B4A
:101700008093C9008091C9008F7D8093C900832F89
:1017100099278093CD002093CC008091C8008260EF
:101720008093C80088E18093C9008091CA008F77B8
:101730008093CA008091CA008F7B8093CA008091F9
:10174000CA008F7D8093CA008091CA008F7E8093EB
:10175000CA008091CA00877F8093CA008091C90027
:101760008B7F8093C9008091CA0084608093CA00F7
:101770008091CA0082608093CA008091C80087FF70
:1017800003C08091CE00F9CF8091C900806880931A
:10179000C9004FBF08950F931F93CF93DF93482F36
:1017A0004F5F893108F08BC080915D09841720F468
:1017B0004F5F40935D094150CB0183539B4268E1E9
:1017C00070E00E94059AA42FBB27FD01EA0FFB1FC2
:1017D000E25AF64F808191819B01281B390BC90188
:1017E00037FF03C0909581959F4F069794F48091A1
:1017F0003804883C30F480913804865F8093380444
:1018000008C088EC8093380480916F008F7D8093AE
:101810006F00FD01EA0FFB1FE25AF64F80819181B4
:101820009C01220F331F280F391F260F371F37FF48
:1018300002C02D5F3F4FE901D595C795D595C79556
:10184000CB0101968C179D0714F4219706C06150B7
:101850007040C617D7070CF4219680913804843B5A
:10186000D8F08D010A0F1B1FF801E25AF64F808154
:101870009181FE01E81BF90BCF0163E070E00E944B
:10188000059ACB01880F991F860F971F0C55164F8D
:10189000F8019183808307C0AA0FBB1FAC55B64FD8
:1018A00011961C921E92E42FFF27EE0FFF1FE25AA3
:1018B000F64FD183C083443011F410923A01DF9186
:1018C000CF911F910F910895CF93DF932091790CC1
:1018D000822F9927807F9070409709F066C02F3142
:1018E00009F040C080917A0C80935F0590917C0C48
:1018F0009093610580917D0C80936005992309F098
:1019000054C080912908282F3327220F331FF90153
:10191000EC55F64F1182108280912A08A82FBB2720
:10192000AA0FBB1FFD01EC55F64F1182108280916A
:101930002C08E82FFF27EE0FFF1FCF018C55964F85
:10194000EC0119821882225A364FE9011982188255
:10195000A25AB64F11961C921E92E25AF64F11826D
:10196000108223C0C22FCF70CA30F8F480917A0C55
:101970008093A50C80917B0C8093A40C80917C0CAF
:101980008093A70C80917D0C8093A60C6091A40C91
:101990007091A50C8C2F0E94CB8B6091A60C70913E
:1019A000A70C8C2F8F5F0E94CB8BDF91CF91089576
:1019B000CF93C82F8F3F49F4809162058F3F29F460
:1019C000109264051092630532C0209164052223B1
:1019D00039F4CF3111F485E001C084E080936505CE
:1019E00080916505909163058217A0F4892F8095F9
:1019F000809363058F3F19F48EEF80936305809188
:101A00006305C81711F40E94648C1092640510924B
:101A100063050BC0E22FFF27E758F34FC0832F5F0A
:101A2000209364059C0F90936305C0936205CF914A
:101A3000089590915E05933240F4E92FFF27EF5708
:101A4000F34F80839F5F90935E050895833218F46F
:101A50008D5F80935E05089590E2E4E8FCE08FE1FD
:101A60009193815087FFFCCF0895CF93CFB723E0A8
:101A700031E0F8948091C9008F778093C9008091FC
:101A8000C9008F7B8093C9008091C9008F7D8093AE
:101A9000C900832F99278093CD002093CC0080919B
:101AA000C80082608093C80088E18093C90080915B
:101AB000CA008F778093CA008091CA008F7B809381
:101AC000CA008091CA0080628093CA008091CA00D7
:101AD00080618093CA008091CA0088608093CA00A8
:101AE0008091C90084608093C9008091CA0084609D
:101AF0008093CA008091CA0082608093CA0080915E
:101B0000C80087FF03C08091CE00F9CF8091C90043
:101B100080688093C9008091C90080648093C90067
:101B20000E942C8DCFBFCF910895282F99278F70B9
:101B30009070892B31F4209580915D05822B8093E4
:101B40005D0508951F920F920FB60F9211248F9387
:101B5000EF93FF938091D702882309F068C0E0914A
:101B60006705EE2389F480916605882369F48091E6
:101B7000810C882321F081E08093680505C0809165
:101B8000C90081608093C90080916805882379F439
:101B9000EF5FE09367058091580C8E1720F481E089
:101BA000809368051CC0FF27E85AF34F3CC0809122
:101BB0006605882361F48091810C882311F483E009
:101BC00003C0813999F481E0809366050FC08330AA
:101BD00099F48091810C882349F01092810C8091B6
:101BE000C9008E7F8093C9008EEF1EC08091C9000E
:101BF00081608093C9000EC0833261F48091C90076
:101C00008E7F8093C9008FEF8093CE0081E0809318
